:020000040800F2
:1000000000060020E1020008E3020008E302000805
:10001000E3020008E3020008E3020008E30200082C
:10002000E3020008E3020008E30200086931000867
:10003000E3020008E3020008E3020008E30200080C
:10004000E3020008E3020008E3020008E3020008FC
:10005000E3020008E30200084D490008794900085E
:10006000A5490008D1490008FD490008D911000838
:10007000011200082D12000859120008851200080C
:10008000AD120008D9120008E3020008E3020008DC
:10009000E3020008E3020008E3020008294A00081E
:1000A000E3020008E3020008E3020008E30200089C
:1000B000E3020008E3020008E3020008E30200088C
:1000C000E3020008E3020008E3020008E30200087C
:1000D000E3020008014B0008E3020008E302000805
:1000E0008D4A0008E3020008E3020008E30200086A
:1000F000E3020008E3020008E30200080513000819
:10010000E3020008E3020008154B0008E3020008C0
:10011000E3020008E3020008E3020008E30200082B
:10012000311300085913000885130008B1130008A3
:10013000DD130008E3020008E3020008E302000800
:10014000E3020008E3020008E3020008E3020008FB
:1001500005140008311400085D140008E3020008CB
:10016000E3020008E3020008E3020008E3020008DB
:10017000E3020008553D0008E3020008E30200081E
:10018000E3020008E3020008E3020008E3020008BB
:10019000E3020008E3020008E3020008E3020008AB
:1001A000E3020008E3020008E3020008E30200089B
:1001B000E3020008E3020008E3020008E30200088B
:1001C000E3020008E3020008E3020008E30200087B
:1001D000E3020008413D0008E3020008E3020008D2
:1001E000E3020008E3020008E3020008E30200085B
:1001F000E3020008E3020008E3020008E30200084B
:10020000E3020008E3020008E3020008E30200083A
:10021000E3020008E3020008E3020008E30200082A
:10022000E3020008E3020008E3020008E30200081A
:10023000E3020008E3020008E3020008E30200080A
:10024000E3020008E3020008E3020008E3020008FA
:10025000E3020008E3020008E3020008E3020008EA
:10026000E3020008E3020008E3020008E3020008DA
:10027000E3020008E3020008E3020008E3020008CA
:10028000E3020008E3020008E3020008E3020008BA
:10029000E3020008E3020008E3020008E3020008AA
:1002A000E3020008E3020008E3020008E30200089A
:1002B000E3020008E3020008E3020008E30200088A
:1002C000E3020008E3020008E3020008E30200087A
:1002D000E3020008E3020008E3020008E30200086A
:1002E00002E000F000F8FEE772B6374880F30888B5
:1002F000364880F3098836483649086040F20000E5
:10030000CCF200004EF63471CEF200010860BFF36B
:100310004F8FBFF36F8F40F20000C0F2F0004EF637
:100320008851CEF200010860BFF34F8FBFF36F8F8B
:100330004FF00000E1EE100A4EF63C71CEF20001E3
:100340000860062080F31488BFF36F8F02F06EFF01
:1003500004F0B6F84FF055301F491B4A91423CBF9C
:1003600041F8040BFAE71D49184A91423CBF41F895
:10037000040BFAE71A491B4A1B4B9A423EBF51F83D
:10038000040B42F8040BF8E700201849184A914280
:100390003CBF41F8040BFAE702F086FF04F014F9C1
:1003A000144C154DAC4203DA54F8041B8847F9E7A6
:1003B00000F042F8114C124DAC4203DA54F8041B21
:1003C0008847F9E702F06EBF0006002000220020F7
:1003D0000000000808ED00E00000002000060020FA
:1003E000885000080022002064220020682200209B
:1003F0000C490020E0020008E0020008E0020008CA
:10040000E00200082DE9F04F2DED108AC1F80CD064
:10041000D0F80CD0BDEC108ABDE8F08F002383F338
:1004200011882846A047002002F054F9FEE702F0A8
:10043000DFF800DFFEE7000038B500F0D3FC00F085
:10044000A3FE02F051FE054602F084FE0446C0B948
:100450000E4B9D4217D001339D4241F2883512BFA9
:10046000044600250124002002F048FE0CB100F0F3
:1004700075F800F027FE284600F01EF900F06EF82F
:10048000F9E70025EFE70546EDE700BF010007B0FB
:1004900008B500F073FCA0F120035842584108BD94
:1004A00007B541F21203022101A8ADF8043000F0B3
:1004B00083FC03B05DF804FB38B5302383F3118867
:1004C000174803680BB102F0D1F90023154A4FF425
:1004D0007A71134802F0C0F9002383F31188124C9B
:1004E000236813B12368013B2360636813B1636819
:1004F000013B63600D4D2B7833B963687BB90220F3
:1005000000F042FD322363602B78032B07D1636830
:100510002BB9022000F038FD4FF47A73636038BDC8
:1005200068220020B90400088823002080220020CF
:10053000084B187003280CD8DFE800F00805020803
:10054000022000F013BD022000F000BD024B00228B
:100550005A6070478022002088230020F8B5504B55
:10056000504A1C461968013100F0998004339342C7
:10057000F8D162684C4B9A4240F291804B4B9B6899
:1005800003F1006303F500339A4280F08880002075
:1005900000F04EFC0220FFF7CBFF454B0021D3F8C3
:1005A000E820C3F8E810D3F81021C3F81011D3F8ED
:1005B0001021D3F8EC20C3F8EC10D3F81421C3F8C1
:1005C0001411D3F81421D3F8F020C3F8F010D3F8A5
:1005D0001821C3F81811D3F81821D3F8802042F05D
:1005E0000062C3F88020D3F8802022F00062C3F8B4
:1005F0008020D3F88020D3F8802042F00072C3F826
:100600008020D3F8802022F00072C3F88020D3F835
:10061000803072B64FF0E023C3F8084DD4E90004EF
:10062000BFF34F8FBFF36F8F224AC2F88410BFF31E
:100630004F8F536923F480335361BFF34F8FD2F848
:10064000803043F6E076C3F3C905C3F34E335B0154
:1006500003EA060C29464CEA81770139C2F8747224
:10066000F9D2203B13F1200FF2D1BFF34F8FBFF32C
:100670006F8FBFF34F8FBFF36F8F536923F4003336
:1006800053610023C2F85032BFF34F8FBFF36F8F17
:10069000302383F31188854680F308882047F8BD0E
:1006A0000000020820000208FFFF010800220020CD
:1006B0000044025800ED00E02DE9F04F93B0B44B38
:1006C0002022FF2100900AA89D6800F0A5FCB14AF5
:1006D0001378A3B90121B04811700360302383F36C
:1006E000118803680BB102F0C1F80023AB4A4FF444
:1006F0007A71A94802F0B0F8002383F31188009BB7
:1007000013B1A74B009A1A60A64A1378032B03D0A3
:1007100000231370A24A53604FF0000A009CD34696
:100720005646D146012000F021FC24B19C4B1B68A9
:10073000002B00F02682002000F020FB0390039B9A
:10074000002BF2DB012000F001FC039B213B1F2B5F
:10075000E8D801A252F823F0D907000801080008E0
:100760009508000825070008250700082507000848
:1007700027090008F70A0008110A0008730A000890
:100780009B0A0008C10A000825070008D30A0008D0
:1007900025070008450B0008790800082507000810
:1007A000890B0008E50700087908000825070008FC
:1007B000730A000825070008250700082507000818
:1007C0002507000825070008250700082507000859
:1007D00025070008950800080220FFF759FE0028A9
:1007E00040F0F981009B022105A8BAF1000F08BF73
:1007F0001C4641F21233ADF8143000F0DDFA91E7F7
:100800004FF47A7000F0BAFA071EEBDB0220FFF714
:100810003FFE0028E6D0013F052F00F2DE81DFE831
:1008200007F0030A0D1013360523042105A80593CC
:1008300000F0C2FA17E004215548F9E704215A48AC
:10084000F6E704215948F3E74FF01C08404608F149
:10085000040800F0EFFA0421059005A800F0ACFAB6
:10086000B8F12C0FF2D101204FF0000900FA07F780
:1008700047EA0B0B5FFA8BFB00F01AFC26B10BF07A
:100880000B030B2B08BF0024FFF70AFE4AE70421E5
:100890004748CDE7002EA5D00BF00B030B2BA1D1C1
:1008A0000220FFF7F5FD074600289BD00120002617
:1008B00000F0BEFA0220FFF73BFE1FFA86F8404622
:1008C00000F0C6FA0446B0B1039940460136A1F1E2
:1008D00040025142514100F0CBFA0028EDD1BA4616
:1008E000044641F21213022105A83E46ADF8143029
:1008F00000F062FA16E725460120FFF719FE244BA7
:100900009B68AB4207D9284600F094FA013040F0CA
:1009100067810435F3E70025224BBA463E461D7039
:100920001F4B5D60A8E7002E3FF45CAF0BF00B039C
:100930000B2B7FF457AF0220FFF7FAFD322000F0B7
:100940001DFAB0F10008FFF64DAF18F003077FF471
:1009500049AF0F4A08EB0503926893423FF642AF56
:10096000B8F5807F3FF73EAF124BB845019323DDCA
:100970004FF47A7000F002FA0390039A002AFFF60F
:1009800031AF039A0137019B03F8012BEDE700BF5C
:10099000002200208423002068220020B9040008DF
:1009A000882300208022002004220020082200202A
:1009B0000C22002084220020C820FFF769FD074692
:1009C00000283FF40FAF1F2D11D8C5F120020AAB4C
:1009D00025F0030084494245184428BF424601924D
:1009E00000F0F4FA019AFF217F4800F015FB4FEA6E
:1009F000A803C8F387027C492846019300F014FB42
:100A0000064600283FF46DAF019B05EB830533E7F5
:100A10000220FFF73DFD00283FF4E4AE00F046FA67
:100A200000283FF4DFAE0027B846704B9B68BB42FE
:100A300018D91F2F11D80A9B01330ED027F00303BA
:100A400012AA134453F8203C05934046042205A9FA
:100A5000043700F0ABFB8046E7E7384600F0EAF9E0
:100A60000590F2E7CDF81480042105A800F0A4F960
:100A700002E70023642104A8049300F093F90028FE
:100A80007FF4B0AE0220FFF703FD00283FF4AAAECA
:100A9000049800F001FA0590E6E70023642104A819
:100AA000049300F07FF900287FF49CAE0220FFF74A
:100AB000EFFC00283FF496AE049800F0EFF9EAE767
:100AC0000220FFF7E5FC00283FF48CAE00F0FEF9B1
:100AD000E1E70220FFF7DCFC00283FF483AE05A924
:100AE000142000F0F9F907460421049004A800F04E
:100AF00063F93946B9E7322000F040F9071EFFF6E6
:100B000071AEBB077FF46EAE384A07EB09039268FB
:100B100093423FF667AE0220FFF7BAFC00283FF48D
:100B200061AE27F003074F44B9453FF4A5AE4846F0
:100B300009F1040900F07EF90421059005A800F0F0
:100B40003BF9F1E74FF47A70FFF7A2FC00283FF47D
:100B500049AE00F0ABF9002844D00A9B01330BD01A
:100B600008220AA9002000F05FFA00283AD02022CB
:100B7000FF210AA800F050FAFFF792FC1C4801F090
:100B8000AFFD13B0BDE8F08F002E3FF42BAE0BF09D
:100B90000B030B2B7FF426AE0023642105A80593DD
:100BA00000F000F9074600287FF41CAE0220FFF792
:100BB0006FFC804600283FF415AEFFF771FC41F250
:100BC000883001F08DFD059800F0BCFA46463C46A1
:100BD00000F06EFAA6E506464EE64FF0000901E683
:100BE000BA467EE637467CE68422002000220020BA
:100BF000A08601002DE9F84F4FF47A7306460D46A2
:100C0000002402FB03F7DFF85080DFF8509098F9DA
:100C100000305FFA84FA5A1C01D0A34212D159F86D
:100C200024002A4631460368D3F820B03B46D84713
:100C3000854207D1074B012083F800A0BDE8F88F5B
:100C40000124E4E7002CFBD04FF4FA7001F048FDDA
:100C50000020F3E7D42300201022002014220020DB
:100C600000232DE9F0471A4605468846012019461B
:100C700000F09CFC0446802002F0C8F907460028DA
:100C800061D0002C5FD03B4E28464FF0800A73693C
:100C900043F0C0637361D6F8143143F0C063C6F803
:100CA000143102F037F805EB080200FB05F34FF4AE
:100CB000D06C50434FF03D0E834233D23269520123
:100CC00043D4D6F8102151013FD4216803F10062CA
:100CD0008A602268D7602268C2F804A02268C2F83D
:100CE00000C0D4F80090D9F8002042F00102C9F801
:100CF0000020D4F80090D9F8002022F01E02C9F894
:100D00000020D4F80090D9F80020D207FBD494F842
:100D10000C90803361680EFA09F20A60CCE700207B
:100D200002F0D6F8204600F081FC384602F0A2F925
:100D3000104B5A6942F0C0625A61D3F8142142F054
:100D4000C062C3F81421BDE8F0870B4B9A6A42F4E5
:100D500000729A629A6A42F400429A6261B6002670
:100D6000012002F0B5F8B045D9D9A819013601F033
:100D7000E9FFF8E70020005200ED00E0002307B58E
:100D8000024601210DF107008DF80730FFF732FF11
:100D900020B19DF8070003B05DF804FB4FF0FF3071
:100DA000F9E700000A46042108B5FFF723FF80F0A9
:100DB0000100C0B2404208BD074B0A4630B4197862
:100DC000064B53F82140014623682046DD69044B59
:100DD000AC4630BC604700BFD42300201422002062
:100DE000A086010070B5104C0025104E01F096FF52
:100DF00020803068238883420CD800252088013861
:100E000001F088FF23880544013BB5F5802F23803E
:100E1000F4D370BD01F07EFF336805440133B5F5AE
:100E2000003F3360E5D3E8E7D6230020902300207D
:100E300002F04EB800F1006000F500300068704725
:100E400000F10060920000F5003001F0C3BF000027
:100E5000054B1A68054B1B889B1A834202D9104424
:100E600001F058BF0020704790230020D6230020B7
:100E700038B50446074D29B128682044BDE83840FC
:100E800001F060BF2868204401F04AFF0028F3D039
:100E900038BD00BF902300200020704700F1FF50B4
:100EA00000F58F10D0F8000870470000064991F84F
:100EB000243033B100230822086A81F82430FFF778
:100EC000BFBF0120704700BF94230020014B18686A
:100ED000704700BF0010005C194B01380322084422
:100EE00070B51D68174BC5F30B042D0C1E88A64268
:100EF0000BD15C680A46013C824213460FD214F9BA
:100F0000016F4EB102F8016BF6E7013A03F10803F5
:100F1000ECD181420B4602D22C2203F8012B04248F
:100F2000094A1688AE4204D1984284BF967803F8E5
:100F3000016B013C02F10402F3D1581A70BD00BFED
:100F40000010005C1C220020184C0008022804D16C
:100F5000054B4FF480129A6170470128FCD1024B77
:100F60004FF48022F7E700BF00100258022803D197
:100F7000044B10229A6170470128FCD1014B0422D6
:100F8000F8E700BF00100258022805D1064A53694D
:100F900083F01003536170470128FCD1024A536962
:100FA00083F00403F6E700BF0010025870B5044652
:100FB0004FF47A764CB1412C254628BF412506FBDB
:100FC00005F0641B01F08CFBF4E770BD002310B545
:100FD000934203D0CC5CC4540133F9E710BD000048
:100FE000013810B510F9013F3BB191F900409C4226
:100FF00003D11AB10131013AF4E71AB191F9002095
:10100000981A10BD1046FCE703460246D01A12F9A2
:10101000011B0029FAD1704702440346934202D0D3
:1010200003F8011BFAE770472DE9F8431F4D1446FA
:101030000746884695F8242052BBDFF870909CB391
:1010400095F824302BB92022FF2148462F62FFF764
:10105000E3FF95F824004146C0F1080205EB80004B
:10106000A24228BF2246D6B29200FFF7AFFF95F802
:101070002430A41B17441E449044E4B2F6B2082E58
:1010800085F82460DBD1FFF711FF0028D7D108E0F5
:101090002B6A03EB82038342CFD0FFF707FF0028C0
:1010A000CBD10020BDE8F8830120FBE7942300208A
:1010B000024B1A78024B1A70704700BFD4230020ED
:1010C0001022002038B51A4C1A4D204600F038FE88
:1010D0002946204600F060FE2D684FF47A70D5F85E
:1010E0009020D2F8043843F00203C2F80438FFF726
:1010F0005DFF1149284600F05DFFD5F890200F4DA7
:10110000D2F80438286823F002030D49A042C2F83F
:1011100004384FF4E1330B6001D000F06FFD6868D4
:10112000A04204D00649BDE8384000F067BD38BD94
:10113000382B0020144E00081C4E000814220020FA
:10114000BC2300200C4B70B50C4D04461E780C4B94
:1011500055F826209A420DD00A4B00211822184635
:10116000FFF75AFF0460014655F82600BDE87040BD
:1011700000F044BD70BD00BFD42300201422002025
:10118000382B0020BC23002008B571B6054B198808
:10119000054B1888FFF764FD02210E20FFF760FD64
:1011A00061B608BDD62300209023002030B50A4444
:1011B000084D91420DD011F8013B5840082340F3EF
:1011C0000004013B2C4013F0FF0384EA5000F6D1E9
:1011D000EFE730BD2083B8ED08B5074B074A196823
:1011E00001F03D01996053680BB190689847BDE8E4
:1011F000084001F0F1BF00BF00000240D8230020EA
:1012000008B5084B1968890901F03D018A019A6007
:10121000054AD3680BB110699847BDE8084001F052
:10122000DBBF00BF00000240D823002008B5084BF8
:101230001968090C01F03D010A049A60054A5369D6
:101240000BB190699847BDE8084001F0C5BF00BFE9
:1012500000000240D823002008B5084B1968890D0A
:1012600001F03D018A059A60054AD3690BB1106A05
:101270009847BDE8084001F0AFBF00BF0000024042
:10128000D823002008B5074B074A596801F03D01F3
:10129000D960536A0BB1906A9847BDE8084001F0E5
:1012A0009BBF00BF00000240D823002008B5084BB8
:1012B0005968890901F03D018A01DA60054AD36A5B
:1012C0000BB1106B9847BDE8084001F085BF00BF27
:1012D00000000240D823002008B5084B5968090CCB
:1012E00001F03D010A04DA60054A536B0BB1906BC3
:1012F0009847BDE8084001F06FBF00BF0000024002
:10130000D823002008B5084B5968890D01F03D012C
:101310008A05DA60054AD36B0BB1106C9847BDE8BB
:10132000084001F059BF00BF00000240D823002050
:1013300008B5074B074A196801F03D019960536CE5
:101340000BB1906C9847BDE8084001F045BF00BF65
:1013500000040240D823002008B5084B1968890909
:1013600001F03D018A019A60054AD36C0BB1106D02
:101370009847BDE8084001F02FBF00BF00040240BD
:10138000D823002008B5084B1968090C01F03D016D
:101390000A049A60054A536D0BB1906D9847BDE8F9
:1013A000084001F019BF00BF00040240D82300200C
:1013B00008B5084B1968890D01F03D018A059A604E
:1013C000054AD36D0BB1106E9847BDE8084001F097
:1013D00003BF00BF00040240D823002008B5074B1C
:1013E000074A596801F03D01D960536E0BB1906E08
:1013F0009847BDE8084001F0EFBE00BF000402407E
:10140000D823002008B5084B5968890901F03D012F
:101410008A01DA60054AD36E0BB1106F9847BDE8B8
:10142000084001F0D9BE00BF00040240D8230020CC
:1014300008B5084B5968090C01F03D010A04DA604F
:10144000054A536F0BB1906F9847BDE8084001F013
:10145000C3BE00BF00040240D823002008B5084BDB
:101460005968890D01F03D018A05DA60054AD36F9C
:1014700013B1D2F880009847BDE8084001F0ACBE37
:1014800000040240D823002000230C4910B51A465E
:101490000B4C0B6054F82300026001EB4300043353
:1014A0004260402BF6D1074A4FF0FF339360D36080
:1014B000C2F80834C2F80C3410BD00BFD823002095
:1014C000284C0008000002400F28F8B510D9102859
:1014D00010D0112811D0122808D10F240720DFF8CE
:1014E000C8E00126DEF80050A04208D9002653E0EB
:1014F0000446F4E70F240020F1E70724FBE706FA8F
:1015000000F73D424AD1264C4FEA001C3D4304EB14
:1015100000160EEBC000CEF80050C0E90123FBB26C
:1015200073B12048D0F8D83043F00103C0F8D83068
:10153000D0F8003143F00103C0F80031D0F8003199
:1015400017F47F4F0ED01748D0F8D83043F002037D
:10155000C0F8D830D0F8003143F00203C0F80031B1
:10156000D0F8003154F80C00036823F01F03036027
:10157000056815F00105FBD104EB0C033D2493F83D
:101580000CC05F6804FA0CF43C60212405604461DF
:1015900012B1987B00F066F93046F8BD0130A3E740
:1015A000284C000800440258D823002010B53024ED
:1015B00084F31188FFF788FF002383F3118810BD9F
:1015C00010B50446807B00F063F901231549627B66
:1015D00003FA02F20B6823EA0203DAB20B6072B973
:1015E000114AD2F8D81021F00101C2F8D810D2F86F
:1015F000001121F00101C2F80011D2F8002113F40A
:101600007F4F0ED1084BD3F8D82022F00202C3F846
:10161000D820D3F8002122F00202C3F80021D3F829
:10162000003110BDD82300200044025808B53023F3
:1016300083F31188FFF7C4FF002383F3118808BDEB
:10164000026843681143016003B118477047000006
:10165000024A136843F0C003136070470010014052
:1016600013B50E4C204600F0BDFA04F1140000231F
:101670004FF400720A49009400F07AF9094B4FF4D4
:101680000072094904F13800009400F0F3F9074AA8
:10169000074BC4E9172302B010BD00BF5C24002033
:1016A000C824002051160008C82600200010014060
:1016B00000E1F505037C30B5244C002918BF0C4629
:1016C000012B11D1224B98420ED1224BD3F8F0209E
:1016D00042F01002C3F8F020D3F8182142F01002B3
:1016E000C3F81821D3F818312268036EC16D03EBDB
:1016F00052038466B3FBF2F36268150442BF23F021
:10170000070503F0070343EA4503CB60A36843F0F2
:1017100040034B60E36843F001038B6042F496732F
:1017200043F001030B604FF0FF330B62510505D509
:1017300012F0102205D0B2F1805F04D080F864303E
:1017400030BD7F23FAE73F23F8E700BF284D0008AC
:101750005C240020004402582DE9F047C66D054680
:101760003768F469210734621AD014F0080118BFF1
:101770004FF48071E20748BF41F02001A3074FF00A
:10178000300348BF41F04001600748BF41F080018D
:1017900083F31188281DFFF753FF002383F311887B
:1017A000E2050AD5302383F311884FF48061281DA8
:1017B000FFF746FF002383F311884FF030094FF005
:1017C000000A14F0200838D13B0616D54FF0300936
:1017D00005F1380A200610D589F31188504600F02B
:1017E0007DF9002836DA0821281DFFF729FF27F0A8
:1017F00080033360002383F31188790614D56206D1
:1018000012D5302383F31188D5E913239A4208D1E6
:101810002B6C33B127F040071021281DFFF710FF74
:101820003760002383F31188E30618D5AA6E136985
:10183000ABB15069BDE8F047184789F31188736A66
:10184000284695F86410194000F0E6F98AF31188EB
:10185000F469B6E7B06288F31188F469BAE7BDE8C5
:10186000F0870000090100F16043012203F56143A4
:10187000C9B283F8001300F01F039A4043099B008C
:1018800003F1604303F56143C3F880211A60704798
:1018900000F01F0301229A40430900F160409B00C1
:1018A00000F5614003F1604303F56143C3F8802014
:1018B000C3F88021002380F800337047F8B515463F
:1018C000826804460B46AA4200D28568A16926694F
:1018D000761AB5420BD218462A46FFF777FBA36962
:1018E0002B44A3612846A3685B1BA360F8BD0CD9F9
:1018F000AF1B18463246FFF769FB3A46E1683044B1
:10190000FFF764FBE3683B44EBE718462A46FFF722
:101910005DFBE368E5E7000083689342F7B50446A2
:10192000154600D28568D4E90460361AB5420BD258
:101930002A46FFF74BFB63692B4463612846A36883
:101940005B1BA36003B0F0BD0DD93246AF1B019104
:10195000FFF73CFB01993A46E0683144FFF736FB5C
:10196000E3683B44E9E72A46FFF730FBE368E4E736
:1019700010B50A440024C361029B8460C160026107
:101980000362C0E90000C0E9051110BD08B5D0E947
:101990000532934201D1826882B982680132826045
:1019A0005A1C426119700021D0E904329A4224BFC6
:1019B000C368436100F0B0FE002008BD4FF0FF3067
:1019C000FBE7000070B5302304460E4683F3118810
:1019D000A568A5B1A368A269013BA360531CA361DC
:1019E00015782269934224BFE368A361E3690BB1D0
:1019F00020469847002383F31188284607E03146A4
:101A0000204600F079FE0028E2DA85F3118870BDE7
:101A10002DE9F74F04460E4617469846D0F81C901D
:101A20004FF0300A8AF311884FF0000B154665B16C
:101A30002A4631462046FFF741FF034660B941463A
:101A4000204600F059FE0028F1D0002383F31188CE
:101A5000781B03B0BDE8F08FB9F1000F03D00190FF
:101A60002046C847019B8BF31188ED1A1E448AF368
:101A70001188DCE7C160C361009B82600362C0E93A
:101A800005111144C0E9000001617047F8B5044632
:101A90000D461646302383F31188A768A7B1A368C3
:101AA000013BA36063695A1C62611D70D4E9043272
:101AB0009A4224BFE3686361E3690BB1204698470B
:101AC000002080F3118807E03146204600F014FE24
:101AD0000028E2DA87F31188F8BD0000D0E9052379
:101AE00010B59A4201D182687AB982680021013228
:101AF00082605A1C82611C7803699A4224BFC368C1
:101B0000836100F009FE204610BD4FF0FF30FBE777
:101B10002DE9F74F04460E4617469846D0F81C901C
:101B20004FF0300A8AF311884FF0000B154665B16B
:101B30002A4631462046FFF7EFFE034660B941468C
:101B4000204600F0D9FD0028F1D0002383F311884E
:101B5000781B03B0BDE8F08FB9F1000F03D00190FE
:101B60002046C847019B8BF31188ED1A1E448AF367
:101B70001188DCE7026843681143016003B118472C
:101B8000704700001430FFF743BF00004FF0FF33F1
:101B90001430FFF73DBF00003830FFF7B9BF000039
:101BA0004FF0FF333830FFF7B3BF00001430FFF7BA
:101BB00009BF00004FF0FF311430FFF703BF0000F2
:101BC0003830FFF763BF00004FF0FF323830FFF7C7
:101BD0005DBF0000012914BF6FF0130000207047A3
:101BE000FFF73EBD044B036000234360C0E90233AE
:101BF00001230374704700BF404D000810B5302327
:101C0000044683F31188FFF755FD02230020237457
:101C100080F3118810BD000038B5C36904460D4635
:101C20001BB904210844FFF7A5FF294604F114005D
:101C3000FFF7ACFE002806DA201D4FF40061BDE876
:101C40003840FFF797BF38BD026843681143016011
:101C500003B118477047000013B5406B00F580547E
:101C6000D4F8A4381A681178042914D1017C022907
:101C700011D11979012312898B4013420BD101A98B
:101C80004C3002F099F9D4F8A4480246019B21791E
:101C9000206800F0DFF902B010BD0000143002F03F
:101CA0001BB900004FF0FF33143002F015B90000EB
:101CB0004C3002F0EDB900004FF0FF334C3002F031
:101CC000E7B90000143002F0E9B800004FF0FF312E
:101CD000143002F0E3B800004C3002F0B9B9000053
:101CE0004FF0FF324C3002F0B3B9000000207047D3
:101CF00010B500F58054D4F8A4381A681178042976
:101D000017D1017C022914D15979012352898B40C2
:101D100013420ED1143002F07BF8024648B1D4F8D9
:101D2000A4484FF4407361792068BDE8104000F08A
:101D30007FB910BD406BFFF7DBBF000070470000AC
:101D40007FB5124B01250426044603600023057469
:101D500000F1840243602946C0E902330C4B029033
:101D6000143001934FF44073009602F02DF8094BA4
:101D700004F69442294604F14C000294CDE9006334
:101D80004FF4407302F0F4F804B070BD684D0008E1
:101D9000351D0008591C00080A68302383F3118898
:101DA0000B790B3342F823004B79133342F82300AD
:101DB0008B7913B10B3342F8230000F58053C3F83D
:101DC000A41802230374002080F3118870470000D8
:101DD00038B5037F044613B190F85430ABB90125F0
:101DE000201D0221FFF730FF04F114006FF0010104
:101DF000257700F09DFC04F14C0084F854506FF0FE
:101E00000101BDE8384000F093BC38BD10B5012198
:101E100004460430FFF718FF0023237784F854307A
:101E200010BD000038B504460025143001F0E4FF71
:101E300004F14C00257702F0B3F8201D84F85450CB
:101E40000121FFF701FF2046BDE83840FFF750BFF2
:101E500090F8803003F06003202B06D190F88120A9
:101E60000023212A03D81F2A06D800207047222ADF
:101E7000FBD1C0E91D3303E0034A426707228267B2
:101E8000C3670120704700BF3422002037B500F53A
:101E90008055D5F8A4381A68117804291AD1017C24
:101EA000022917D11979012312898B40134211D1CC
:101EB00000F14C04204602F033F958B101A9204644
:101EC00002F07AF8D5F8A4480246019B21792068EF
:101ED00000F0C0F803B030BD01F10B03F0B550F8CD
:101EE000236085B004460D46FEB1302383F311888C
:101EF00004EB8507301D0821FFF7A6FEFB6806F1FD
:101F00004C005B691B681BB1019002F063F80198FB
:101F100003A902F051F8024648B1039B2946204626
:101F200000F098F8002383F3118805B0F0BDFB683A
:101F30005A691268002AF5D01B8A013B1340F1D17F
:101F400004F18002EAE70000133138B550F821406F
:101F5000ECB1302383F3118804F58053D3F8A4281F
:101F60001368527903EB8203DB689B695D6845B1B6
:101F700004216018FFF768FE294604F1140001F0FF
:101F800051FF2046FFF7B4FE002383F3118838BDCC
:101F90007047000001F01EBA01234022002110B555
:101FA000044600F8303BFFF737F80023C4E901335B
:101FB00010BD000010B53023044683F3118824229D
:101FC000416000210C30FFF727F8204601F024FA89
:101FD00002230020237080F3118810BD70B500EB40
:101FE0008103054650690E461446DA6018B1102286
:101FF0000021FFF711F8A06918B110220021FFF7A6
:102000000BF831462846BDE8704001F00BBB0000DC
:1020100083682022002103F0011310B50446836079
:102020001030FEF7F9FF2046BDE8104001F086BBF6
:10203000F0B4012500EB810447898D40E4683D43FD
:10204000A469458123600023A2606360F0BC01F0B5
:10205000A3BB0000F0B4012500EB810407898D408B
:10206000E4683D436469058123600023A2606360E6
:10207000F0BC01F019BC000070B502230025044635
:10208000242203702946C0F888500C3040F8045CC4
:10209000FEF7C2FF204684F8705001F057FA6368DB
:1020A0001B6823B129462046BDE87040184770BD23
:1020B0000378052B10B504460AD080F88C30052330
:1020C000037043681B680BB1042198470023A36089
:1020D00010BD00000178052906D190F88C204368D6
:1020E00002701B6803B118477047000070B590F884
:1020F0007030044613B1002380F8703004F1800280
:10210000204601F03FFB63689B68B3B994F88030C8
:1021100013F0600535D00021204601F031FE00218A
:10212000204601F021FE63681B6813B1062120469A
:102130009847062384F8703070BD204698470028E1
:10214000E4D0B4F88630A26F9A4288BFA36794F9AE
:102150008030A56F002B4FF0300380F20381002DFB
:1021600000F0F280092284F8702083F311880021A6
:102170002046D4E91D23FFF76DFF002383F3118868
:10218000DAE794F8812003F07F0343EA022340F268
:102190000232934200F0C58021D8B3F5807F48D049
:1021A0000DD8012B3FD0022B00F09380002BB2D131
:1021B00004F1880262670222A267E367C1E7B3F510
:1021C000817F00F09B80B3F5407FA4D194F88230EA
:1021D000012BA0D1B4F8883043F0020332E0B3F50C
:1021E000006F4DD017D8B3F5A06F31D0A3F5C06301
:1021F000012B90D86368204694F882205E6894F89A
:102200008310B4F88430B047002884D043686367F3
:102210000368A3671AE0B3F5106F36D040F60242A8
:1022200093427FF478AF5C4B63670223A36700237C
:10223000C3E794F88230012B7FF46DAFB4F8883097
:1022400023F00203A4F88830C4E91D55E56778E758
:10225000B4F88030B3F5A06F0ED194F882302046E8
:1022600084F88A3001F0D0F963681B6813B101214A
:1022700020469847032323700023C4E91D339CE7BD
:1022800004F18B0363670123C3E72378042B10D188
:10229000302383F311882046FFF7BAFE85F31188B7
:1022A0000321636884F88B5021701B680BB12046B2
:1022B000984794F88230002BDED084F88B300423CA
:1022C000237063681B68002BD6D0022120469847F4
:1022D000D2E794F8843020461D0603F00F010AD59A
:1022E00001F042FA012804D002287FF414AF2B4BEE
:1022F0009AE72B4B98E701F029FAF3E794F882303C
:10230000002B7FF408AF94F8843013F00F01B3D0A2
:102310001A06204602D501F04BFDADE701F03CFD69
:10232000AAE794F88230002B7FF4F5AE94F884305D
:1023300013F00F01A0D01B06204602D501F020FDAE
:102340009AE701F011FD97E7142284F8702083F3D7
:1023500011882B462A4629462046FFF769FE85F359
:102360001188E9E65DB1152284F8702083F31188A5
:1023700000212046D4E91D23FFF75AFEFDE60B227B
:1023800084F8702083F311882B462A46294620467C
:10239000FFF760FEE3E700BF984D0008904D00088E
:1023A000944D000838B590F870300446002B3ED0AC
:1023B000063BDAB20F2A34D80F2B32D8DFE803F00D
:1023C0003731310822323131313131313131373722
:1023D000856FB0F886309D4214D2C3681B8AB5FB66
:1023E000F3F203FB12556DB9302383F311882B46AA
:1023F0002A462946FFF72EFE85F311880A2384F822
:1024000070300EE0142384F87030302383F3118889
:10241000002320461A461946FFF70AFE002383F3DD
:10242000118838BDC36F03B198470023E7E7002147
:10243000204601F0A5FC0021204601F095FC6368D0
:102440001B6813B10621204698470623D7E70000F2
:1024500010B590F870300446142B29D017D8062BED
:1024600005D001D81BB110BD093B022BFBD80021C0
:10247000204601F085FC0021204601F075FC6368D0
:102480001B6813B1062120469847062319E0152B37
:10249000E9D10B2380F87030302383F311880023B7
:1024A0001A461946FFF7D6FD002383F31188DAE7B1
:1024B000C3689B695B68002BD5D1C36F03B1984794
:1024C000002384F87030CEE7002382680375036927
:1024D0001B6899689142FBD25A68036042601060A1
:1024E0005860704700238268037503691B68996808
:1024F0009142FBD85A680360426010605860704790
:1025000008B50846302383F311880A7D0023052A85
:1025100006D8DFE802F00B050503120E826913608E
:102520004FF0FF338361FFF7CFFF002383F3118860
:1025300008BD8269936801339360D0E9003213606B
:102540005A60EDE7FFF7C0BF054BD96808751868FA
:10255000026853601A600122D8600275FDF752BF0D
:10256000C82800200C4B30B5DD684B1C87B00446F2
:102570000FD02B46094A684600F06EF92046FFF757
:10258000E3FF009B13B1684600F070F9A86907B03B
:1025900030BDFFF7D9FFF9E7C82800200125000862
:1025A00038B50C4D04468161EB6881689A689142A8
:1025B00003D8BDE83840FFF787BF1846FFF792FF02
:1025C00001230146EC6020462375BDE83840FDF745
:1025D00019BF00BFC8280020044B1A68DB68906848
:1025E0009B68984294BF002001207047C8280020B3
:1025F000084B10B51C68D868226853601A60012225
:10260000DC602275FFF76EFF01462046BDE81040F2
:10261000FDF7F8BEC828002038B50123084C002576
:102620002370656001F0B8FD01F0DEFD0549064844
:1026300001F0B2FE0223237085F3118838BD00BF7C
:10264000302B0020A04D0008C828002000F044B91D
:10265000034A516853685B1A9842FBD8704700BF21
:10266000001000E08B600223086108468B827047EF
:102670008368A3F1840243F8142C026943F8442CC4
:10268000426943F8402C094A43F8242CC268A3F15C
:10269000200043F8182C022203F80C2C002203F827
:1026A0000B2C034A43F8102C704700BF1D04000890
:1026B000C828002008B5FFF7DBFFBDE80840FFF79A
:1026C00041BF0000024BDB6898610F20FFF73CBF61
:1026D000C8280020302383F31188FFF7F3BF0000E0
:1026E00008B50146302383F311880820FFF73AFF2D
:1026F000002383F3118808BD064BDB6839B14268BB
:1027000018605A60136043600420FFF72BBF4FF03E
:10271000FF307047C82800200368984206D01A6826
:102720000260506018469961FFF70CBF70470000C7
:1027300038B504460D462068844200D138BD036890
:1027400023605C608561FFF7FDFEF4E7036810B568
:102750009C68A2420CD85C688A600B604C60216067
:10276000596099688A1A9A604FF0FF33836010BDF0
:10277000121B1B68ECE700000A2938BF0A2170B55C
:1027800004460D460A26601901F000FD01F0E8FC40
:10279000041BA54203D8751C04462E46F3E70A2EF7
:1027A00004D90120BDE8704001F036BE70BD0000C4
:1027B000F8B5144B0D460A2A4FF00A07D96103F108
:1027C0001001826038BF0A22416019691446016015
:1027D00048601861A81801F0C9FC01F0C1FC431B56
:1027E0000646A34206D37C1C28192746354601F02D
:1027F000CDFCF2E70A2F04D90120BDE8F84001F032
:102800000BBEF8BDC8280020F8B506460D4601F0FD
:10281000A7FC0F4A134653F8107F9F4206D12A4661
:1028200001463046BDE8F840FFF7C2BFD169BB683A
:10283000441A2C1928BF2C46A34202D92946FFF777
:102840009BFF224631460348BDE8F840FFF77EBFB4
:10285000C8280020D8280020C0E90323002310B492
:102860005DF8044B4361FFF7CFBF000010B5194C72
:10287000236998420DD08168D0E9003213605A6014
:102880009A680A449A60002303604FF0FF33A36103
:1028900010BD0268234643F8102F536000220260E7
:1028A00022699A4203D1BDE8104001F069BC9368E7
:1028B00081680B44936001F053FC2269E1699268DE
:1028C000441AA242E4D91144BDE81040091AFFF7A6
:1028D00053BF00BFC82800202DE9F047DFF8BC80B7
:1028E00008F110072C4ED8F8105001F039FCD8F838
:1028F0001C40AA68031B9A423ED814444FF00009BA
:10290000D5E90032C8F81C4013605A60C5F8009041
:10291000D8F81030B34201D101F032FC89F31188AC
:10292000D5E9033128469847302383F311886B6932
:10293000002BD8D001F014FC6A69A0EB0409824690
:102940004A450DD2022001F067FD0022D8F8103070
:10295000B34208D151462846BDE8F047FFF728BFEB
:10296000121A2244F2E712EB09092946384638BF09
:102970004A46FFF7EBFEB5E7D8F81030B34208D06F
:102980001444C8F81C00211AA960BDE8F047FFF7FD
:10299000F3BEBDE8F08700BFD8280020C82800207B
:1029A00000207047FEE70000704700004FF0FF3046
:1029B0007047000002290CD0032904D001290748E0
:1029C00018BF00207047032A05D8054800EBC20055
:1029D0007047044870470020704700BF784E0008D9
:1029E000442200202C4E000870B59AB005460846D7
:1029F000144601A900F0C2F801A8FEF705FB431C2C
:102A00000022C6B25B001046C5E9003423700323E0
:102A1000023404F8013C01ABD1B202348E4201D839
:102A20001AB070BD13F8011B013204F8010C04F850
:102A3000021CF1E708B5302383F311880348FFF740
:102A400025FA002383F3118808BD00BF382B00202E
:102A500090F8803003F01F02012A07D190F88120FE
:102A60000B2A03D10023C0E91D3315E003F06003F6
:102A7000202B08D1B0F884302BB990F88120212A7E
:102A800003D81F2A04D8FFF7E3B9222AEBD0FAE7CC
:102A9000034A426707228267C3670120704700BF6D
:102AA0003B22002007B5052917D8DFE801F01916E9
:102AB00003191920302383F31188104A0121019052
:102AC000FFF78CFA019802210D4AFFF787FA0D48AB
:102AD000FFF7A8F9002383F3118803B05DF804FB26
:102AE000302383F311880748FFF772F9F2E73023A8
:102AF00083F311880348FFF789F9EBE7CC4D000811
:102B0000F04D0008382B002038B50C4D0C4C2A46EF
:102B10000C4904F10800FFF767FF05F1CA0204F150
:102B200010000949FFF760FF05F5CA7204F11800AB
:102B30000649BDE83840FFF757BF00BF10440020EA
:102B400044220020AC4D0008B64D0008C14D0008DD
:102B500070B5044608460D46FEF756FAC6B2204642
:102B6000013403780BB9184670BD32462946FEF78A
:102B700037FA0028F3D10120F6E700002DE9F84FDD
:102B800005460C46FEF740FA2C49C6B22846FFF728
:102B9000DFFF08B10536F6B229492846FFF7D8FF0E
:102BA00008B11036F6B2632E0DD8DFF89080DFF84A
:102BB0009090244FDFF894A0DFF894B02E7846B9B7
:102BC0002670BDE8F88F29462046BDE8F84F02F090
:102BD00005B8252E2ED1072241462846FEF700FAD9
:102BE00070B9DBF8003007350C3444F80C3CDBF8E6
:102BF000043044F8083CDBF8083044F8043CDDE7D6
:102C0000082249462846FEF7EBF998B9A21C0E4B5C
:102C1000197802320909C95D02F8041C13F8011B76
:102C200001F00F015345C95D02F8031CF0D11834BF
:102C30000835C3E7013504F8016BBFE7984E00087B
:102C4000C14D0008AD4E000800E8F11F0CE8F11F6F
:102C5000A04E0008BFF34F8F044B1A695107FCD1F7
:102C6000D3F810215207F8D1704700BF002000525E
:102C700008B50D4B1B78ABB9FFF7ECFF0B4BDA68CF
:102C8000D10704D50A4A5A6002F188325A60D3F853
:102C90000C21D20706D5064AC3F8042102F1883276
:102CA000C3F8042108BD00BF6E460020002000527A
:102CB0002301674508B5114B1B78F3B9104B1A690E
:102CC000510703D5DA6842F04002DA60D3F81021E8
:102CD000520705D5D3F80C2142F04002C3F80C216D
:102CE000FFF7B8FF064BDA6842F00102DA60D3F86A
:102CF0000C2142F00102C3F80C2108BD6E460020F1
:102D0000002000520F289ABF00F580604004002088
:102D1000704700004FF400307047000010207047EB
:102D20000F2808B50BD8FFF7EDFF00F50033026858
:102D3000013204D104308342F9D1012008BD0020C2
:102D4000FCE700000F2838B505463FD8FFF782FFA3
:102D50001F4CFFF78DFF4FF0FF3307286361C4F866
:102D600014311DD82361FFF775FF030243F02403DC
:102D7000E360E36843F08003E36023695A07FCD40F
:102D80002846FFF767FFFFF7BDFF4FF4003100F063
:102D9000C3F92846FFF78EFFBDE83840FFF7C0BFF4
:102DA000C4F81031FFF756FFA0F108031B0243F0EF
:102DB0002403C4F80C31D4F80C3143F08003C4F878
:102DC0000C31D4F810315B07FBD4D9E7002038BDB3
:102DD000002000522DE9F84F04460D46104644EA03
:102DE0000203DE0602D00020BDE8F88F20F01F00AD
:102DF000DFF8D4B0DFF8D4A0FFF73AFF05EB000806
:102E0000454503D10120FFF755FFEDE72022294674
:102E1000204601F0D3FE10B920342035F0E72346D8
:102E200004F120021F68791CDDD104339342F9D1EB
:102E300004F178432048214EB3F5801F204B38BF62
:102E4000184603F1F80332BFD946D1461E46FFF7B4
:102E500001FF0760A4EB050C336805F11C0143F08A
:102E6000020333602B1FD9F8007017F00507FAD161
:102E700053F8042F8B424CF80320F4D1BFF34F8F4B
:102E8000FFF7E8FE4FF0FF330360336823F00203DF
:102E90003360BFF34F8F0B4BC3F85C42BFF34F8FD0
:102EA000BFF36F8F20222946204601F087FE0028BD
:102EB000B2D03846A7E700BF142100520C200052C0
:102EC0001420005200ED00E01020005210210052AA
:102ED00010B5084C237828B11BB9FFF7C9FE0123B0
:102EE000237010BD002BFCD02070BDE81040FFF710
:102EF000E1BE00BF6E4600202DE9F04F0D4685B0C3
:102F0000814658B111F00D0614BF2022082211F09D
:102F10000803019304D0431E03426AD0002435E025
:102F2000002E37D009F11F0121F01F094FF00108D1
:102F3000324F05F00403DFF8D0A005EA080BBBF11F
:102F4000000F32D07869C0072FD408F101080C3780
:102F5000B8F1060FF3D19EB9294D4946A81901923F
:102F600001F064F9044600283AD11836019A782E07
:102F7000F3D1494601F05AF90446002830D1019AAC
:102F80004946204801F052F9044668BB204605B086
:102F9000BDE8F08F0029C9D101462846029201F010
:102FA00045F90446E0B9029AC0E713B178694107D0
:102FB000CBD5AC0702D578698007C6D5019911B188
:102FC00078690107C1D51820494600FB08A0CDE962
:102FD000022301F02BF90446DDE902230028B4D0D6
:102FE0004A460021204601E04A460021FEF714F837
:102FF000CCE70246002E95D198E700BFC04E0008EE
:10300000A046002070460020884600200121FFF7DE
:1030100073BF0000F8B5144D01241827134E40F279
:10302000FF3200210120FDF7F7FF07FB04600134A8
:103030002A6955F80C1F01F0E5F8062CF5D1372563
:103040004FF4C0542046FFF7E1FF014628B1224665
:103050000748BDE8F84001F0D5B8C4EBC404013D11
:103060004FEAD404EED1F8BDC04E000888460020D7
:103070007046002008B101F04BB970470244074B7D
:10308000D2B210B5904200D110BD441C00B253F82A
:10309000200041F8040BE0B2F4E700BF50400058B4
:1030A0000E4B30B51C6F240405D41C6F1C671C6FBD
:1030B00044F400441C670A4C02442368D2B243F42F
:1030C00080732360074B904200D130BD441C51F8FF
:1030D000045B00B243F82050E0B2F4E70044025829
:1030E000004802585040005807B5012201A90020AD
:1030F000FFF7C4FF019803B05DF804FB13B5044665
:10310000FFF7F2FFA04205D0012201A9002001949F
:10311000FFF7C6FF02B010BD0144BFF34F8F064B4F
:10312000884204D3BFF34F8FBFF36F8F7047C3F84C
:103130005C022030F4E700BF00ED00E0034B1A68AA
:103140001AB9034AD2F8D0241A60704718470020F1
:103150000040025808B5FFF7F1FF024B1868C0F3B2
:10316000806008BD18470020EFF3098305496833E4
:103170004A6B22F001024A6383F30988002383F338
:103180001188704700EF00E0302080F3118862B6AC
:103190000D4B0E4AD96821F4E0610904090C0A4379
:1031A0000B49DA60D3F8FC2042F08072C3F8FC20AF
:1031B000084AC2F8B01F116841F0010111602022D5
:1031C000DA7783F82200704700ED00E00003FA058B
:1031D00055CEACC5001000E0302310B583F3118844
:1031E0000E4B5B6813F4006314D0F1EE103AEFF36A
:1031F00009844FF08073683CE361094BDB6B236605
:1032000084F30988FFF7E8F910B1064BA36110BDFC
:10321000054BFBE783F31188F9E700BF00ED00E001
:1032200000EF00E02F0400083204000870B5BFF37F
:103230004F8FBFF36F8F1A4A0021C2F85012BFF3AD
:103240004F8FBFF36F8F536943F400335361BFF364
:103250004F8FBFF36F8FC2F88410BFF34F8FD2F838
:10326000803043F6E074C3F3C900C3F34E335B010F
:1032700003EA0406014646EA81750139C2F8605244
:10328000F9D2203B13F1200FF2D1BFF34F8F5369D6
:1032900043F480335361BFF34F8FBFF36F8F70BD23
:1032A00000ED00E0FEE70000214B2248224A70B505
:1032B000904237D3214BC11EDA1C121A22F00302AE
:1032C0008B4238BF00220021FDF7A6FE1C4A0023D6
:1032D000C2F88430BFF34F8FD2F8803043F6E074E9
:1032E000C3F3C900C3F34E335B0103EA040601468E
:1032F00046EA81750139C2F86C52F9D2203B13F1CC
:10330000200FF2D1BFF34F8FBFF36F8FBFF34F8FFB
:10331000BFF36F8F0023C2F85032BFF34F8FBFF35C
:103320006F8F70BD53F8041B40F8041BC0E700BF4B
:10333000EC5000080C4900200C4900200C490020EA
:1033400000ED00E0074BD3F8D81021EA0001C3F8E4
:10335000D810D3F8002122EA0002C3F80021D3F8E4
:10336000003170470044025870B5D0E92443002270
:103370004FF0FF359E6804EB42135101D3F800096A
:10338000002805DAD3F8000940F08040C3F80009AE
:10339000D3F8000B002805DAD3F8000B40F080408A
:1033A000C3F8000B013263189642C3F80859C3F8FA
:1033B000085BE0D24FF00113C4F81C3870BD000068
:1033C000890141F02001016103699B06FCD41220B0
:1033D000FFF73EB910B50A4C2046FEF7DDFD094B5C
:1033E000C4F89030084BC4F89430084C2046FEF7DF
:1033F000D3FD074BC4F89030064BC4F8943010BD91
:103400001C470020000008402C4F0008B84700204F
:1034100000000440384F000870B503780546012BC2
:103420005CD1434BD0F89040984258D1414B0E218B
:103430006520D3F8D82042F00062C3F8D820D3F832
:10344000002142F00062C3F80021D3F80021D3F834
:10345000802042F00062C3F88020D3F8802022F060
:103460000062C3F88020D3F88030FEF7FBF9324BBE
:10347000E360324BC4F800380023D5F89060C4F8FC
:10348000003EC02323604FF40413A3633369002B71
:10349000FCDA01230C203361FFF7DAF83369DB072C
:1034A000FCD41220FFF7D4F83369002BFCDA002695
:1034B0002846A660FFF758FF6B68C4F81068DB6801
:1034C000C4F81468C4F81C6883BB1D4BA3614FF09B
:1034D000FF336361A36843F00103A36070BD194B20
:1034E0009842C9D1134B4FF08060D3F8D82042F0F6
:1034F0000072C3F8D820D3F8002142F00072C3F85C
:103500000021D3F80021D3F8802042F00072C3F8E4
:103510008020D3F8802022F00072C3F88020D3F8F6
:103520008030FFF70FFF0E214D209EE7064BCDE7C1
:103530001C470020004402584014004003002002B1
:10354000003C30C0B8470020083C30C0F8B5D0F887
:103550009040054600214FF000662046FFF730FFFF
:10356000D5F8941000234FF001128F684FF0FF3010
:10357000C4F83438C4F81C2804EB431201339F42CA
:10358000C2F80069C2F8006BC2F80809C2F8080B5B
:10359000F2D20B68D5F89020C5F8983063621023FA
:1035A0001361166916F01006FBD11220FFF750F8D0
:1035B000D4F8003823F4FE63C4F80038A36943F458
:1035C000402343F01003A3610923C4F81038C4F862
:1035D00014380B4BEB604FF0C043C4F8103B094B61
:1035E000C4F8003BC4F81069C4F80039D5F8983025
:1035F00003F1100243F48013C5F89820A362F8BDCC
:10360000084F000840800010D0F8902090F88A10F1
:10361000D2F8003823F4FE6343EA0113C2F80038FD
:10362000704700002DE9F84300EB8103D0F890507B
:103630000C468046DA680FFA81F94801166806F0F0
:103640000306731E022B05EB41134FF0000194BFDC
:10365000B604384EC3F8101B4FF0010104F11003FB
:1036600098BF06F1805601FA03F3916998BF06F5F9
:10367000004600293AD0578A04F1580137434901DE
:103680006F50D5F81C180B430021C5F81C382B18B7
:103690000127C3F81019A7405369611E9BB3138A11
:1036A000928B9B08012A88BF5343D8F8982098181A
:1036B00042EA034301F140022146C8F89800284637
:1036C00005EB82025360FFF77BFE08EB8900C368BD
:1036D0001B8A43EA845348341E4364012E51D5F8B3
:1036E0001C381F43C5F81C78BDE8F88305EB491763
:1036F000D7F8001B21F40041C7F8001BD5F81C18AF
:1037000021EA0303C0E704F13F030B4A28462146A0
:1037100005EB83035A60FFF753FE05EB4910D0F821
:10372000003923F40043C0F80039D5F81C3823EAE7
:103730000707D7E70080001000040002D0F89420AB
:103740001268C0F89820FFF70FBE00005831D0F87B
:10375000903049015B5813F4004004D013F4001F6B
:103760000CBF0220012070474831D0F89030490149
:103770005B5813F4004004D013F4001F0CBF022068
:103780000120704700EB8101CB68196A0B68136058
:103790004B6853607047000000EB810330B5DD6873
:1037A000AA691368D36019B9402B84BF4023136002
:1037B0006B8A1468D0F890201C4402EB4110013C45
:1037C00009B2B4FBF3F46343033323F0030343EA86
:1037D000C44343F0C043C0F8103B2B6803F003031D
:1037E000012B0ED1D2F8083802EB411013F4807F80
:1037F000D0F8003B14BF43F0805343F00053C0F8AF
:10380000003B02EB4112D2F8003B43F00443C2F804
:10381000003B30BD2DE9F041D0F8906005460C46E4
:1038200006EB4113D3F8087B3A07C3F8087B08D5A9
:10383000D6F814381B0704D500EB8103DB685B68FE
:103840009847FA071FD5D6F81438DB071BD505EBC8
:103850008403D968CCB98B69488A5A68B2FBF0F600
:1038600000FB16228AB91868DA6890420DD2121A43
:10387000C3E90024302383F3118821462846FFF74B
:103880008BFF84F31188BDE8F081012303FA04F271
:103890006B8923EA02036B81CB68002BF3D02146AE
:1038A0002846BDE8F041184700EB81034A0170B596
:1038B000DD68D0F890306C692668E66056BB1A4423
:1038C0004FF40020C2F810092A6802F00302012A0E
:1038D0000AB20ED1D3F8080803EB421410F4807F2B
:1038E000D4F8000914BF40F0805040F00050C4F8F4
:1038F000000903EB4212D2F8000940F00440C2F87C
:1039000000090122D3F8340802FA01F10143C3F897
:10391000341870BD19B9402E84BF40202060206843
:103920001A442E8A8419013CB4FBF6F440EAC440E0
:1039300040F00050C6E700002DE9F843D0F8906051
:1039400005460C464F0106EB4113D3F8088918F0E1
:10395000010FC3F808891CD0D6F81038DB0718D53A
:1039600000EB8103D3F80CC0DCF81430D3F800E08E
:10397000DA68964530D2A2EB0E024FF000091A60C9
:10398000C3F80490302383F31188FFF78DFF89F388
:10399000118818F0800F1DD0D6F834380126A640C3
:1039A000334217D005EB84030134D5F89050D3F897
:1039B0000CC0E4B22F44DCF8142005EB0434D2F838
:1039C00000E05168714514D3D5F8343823EA06066F
:1039D000C5F83468BDE8F883012303FA01F20389CE
:1039E00023EA02030381DCF80830002BD1D098478A
:1039F000CFE7AEEB0103BCF81000834228BF0346BB
:103A0000D7F8180980B2B3EB800FE3D89068A0F123
:103A1000040959F8048FC4F80080A0EB0908984401
:103A2000B8F1040FF5D818440B4490605360C8E710
:103A30002DE9F84FD0F8905004466E69AB691E40EE
:103A400016F480586E6103D0BDE8F84FFEF714BB42
:103A5000002E12DAD5F8003E9B0705D0D5F8003EBF
:103A600023F00303C5F8003ED5F80438204623F0C0
:103A70000103C5F80438FEF72DFB370505D52046B0
:103A8000FFF772FC2046FEF713FBB0040CD5D5F807
:103A9000083813F0060FEB6823F470530CBF43F49F
:103AA000105343F4A053EB6031071BD56368DB6808
:103AB0001BB9AB6923F00803AB612378052B0CD14C
:103AC000D5F8003E9A0705D0D5F8003E23F0030351
:103AD000C5F8003E2046FEF7FDFA6368DB680BB1CF
:103AE00020469847F30200F1BA80B70226D5D4F8F1
:103AF000909000274FF0010A09EB4712D2F8003BE3
:103B000003F44023B3F5802F11D1D2F8003B002BF2
:103B10000DDA62890AFA07F322EA0303638104EBF0
:103B20008703DB68DB6813B13946204698470137C5
:103B3000D4F89430FFB29B689F42DDD9F00619D5C6
:103B4000D4F89000026AC2F30A1702F00F0302F4DD
:103B5000F012B2F5802F00F0CA80B2F5402F09D1E3
:103B600004EB8303002200F58050DB681B6A974258
:103B700040F0B0803003D5F8185835D5E90303D5A7
:103B800000212046FFF746FEAA0303D50121204667
:103B9000FFF740FE6B0303D502212046FFF73AFEF4
:103BA0002F0303D503212046FFF734FEE80203D597
:103BB00004212046FFF72EFEA90203D50521204649
:103BC000FFF728FE6A0203D506212046FFF722FEF2
:103BD0002B0203D507212046FFF71CFEEF0103D57A
:103BE00008212046FFF716FE700340F1A780E90781
:103BF00003D500212046FFF79FFEAA0703D5012128
:103C00002046FFF799FE6B0703D502212046FFF7F8
:103C100093FE2F0703D503212046FFF78DFEEE0606
:103C200003D504212046FFF787FEA80603D505210A
:103C30002046FFF781FE690603D506212046FFF7DF
:103C40007BFE2A0603D507212046FFF775FEEB050C
:103C500074D520460821BDE8F84FFFF76DBED4F8B3
:103C600090904FF0000B4FF0010AD4F894305FFAB7
:103C70008BF79B689F423FF638AF09EB4713D3F8A9
:103C8000002902F44022B2F5802F20D1D3F8002978
:103C9000002A1CDAD3F8002942F09042C3F8002928
:103CA000D3F80029002AFBDB3946D4F89000FFF74F
:103CB00087FB22890AFA07F322EA0303238104EB34
:103CC0008703DB689B6813B13946204698470BF1A0
:103CD000010BCAE7910701D1D0F80080072A02F151
:103CE00001029CBF03F8018B4FEA18283FE704EB61
:103CF000830300F58050DA68D2F818C0DCF8082099
:103D0000DCE9001CA1EB0C0C00218F4208D1DB6820
:103D10009B699A683A449A605A683A445A6029E71B
:103D200011F0030F01D1D0F800808C4501F10101A1
:103D300084BF02F8018B4FEA1828E6E7BDE8F88F48
:103D400008B50348FFF774FEBDE80840FFF744BA22
:103D50001C47002008B50348FFF76AFEBDE808408D
:103D6000FFF73ABAB8470020D0F8903003EB411182
:103D7000D1F8003B43F40013C1F8003B704700004A
:103D8000D0F8903003EB4111D1F8003943F400131F
:103D9000C1F8003970470000D0F8903003EB4111B2
:103DA000D1F8003B23F40013C1F8003B704700003A
:103DB000D0F8903003EB4111D1F8003923F400130F
:103DC000C1F800397047000030B50433039C01721C
:103DD000002104FB0325C160C0E90653049B036373
:103DE000059BC0E90000C0E90422C0E90842C0E91F
:103DF0000A11436330BD00000022416AC260C0E97D
:103E00000411C0E90A226FF00101FEF791BC000025
:103E1000D0E90432934201D1C2680AB9181D704733
:103E200000207047036919600021C2680132C26036
:103E3000C269134482699342036124BF436A0361E8
:103E4000FEF76ABC38B504460D46E3683BB16269CB
:103E50000020131D1268A3621344E36207E0237A73
:103E600033B929462046FEF747FC0028EDDA38BD75
:103E70006FF00100FBE70000C368C269013BC3604B
:103E80004369134482699342436124BF436A436197
:103E900000238362036B03B11847704770B530236A
:103EA000044683F31188866A3EB9FFF7CBFF0546C7
:103EB00018B186F31188284670BDA36AE26A13F828
:103EC000015B9342A36202D32046FFF7D5FF002394
:103ED00083F31188EFE700002DE9F84F04460E4602
:103EE000174698464FF0300989F311880025AA46F5
:103EF000D4F828B0BBF1000F09D141462046FFF7A6
:103F0000A1FF20B18BF311882846BDE8F88FD4E9D2
:103F10000A12A7EB050B521A934528BF9346BBF133
:103F2000400F1BD9334601F1400251F8040B914276
:103F300043F8040BF9D1A36A403640354033A362FD
:103F4000D4E90A239A4202D32046FFF795FF8AF369
:103F50001188BD42D8D289F31188C9E730465A4644
:103F6000FDF734F8A36A5E445D445B44A362E7E76F
:103F700010B5029C0433017203FB0421C460C0E944
:103F800006130023C0E90A33039B0363049BC0E9C3
:103F90000000C0E90422C0E90842436310BD0000EC
:103FA000026A6FF00101C260426AC0E90422002285
:103FB000C0E90A22FEF7BCBBD0E904239A4201D132
:103FC000C26822B9184650F8043B0B6070470023C2
:103FD0001846FAE7C3680021C2690133C360436928
:103FE000134482699342436124BF436A4361FEF7ED
:103FF00093BB000038B504460D46E3683BB1236926
:1040000000201A1DA262E2691344E36207E0237AEA
:1040100033B929462046FEF76FFB0028EDDA38BD9C
:104020006FF00100FBE7000003691960C268013A04
:10403000C260C269134482699342036124BF436A28
:10404000036100238362036B03B1184770470000CC
:1040500070B530230D460446114683F31188866AF5
:104060002EB9FFF7C7FF10B186F3118870BDA36AA0
:104070001D70A36AE26A01339342A36204D3E1692B
:1040800020460439FFF7D0FF002080F31188EDE7C8
:104090002DE9F84F04460D46904699464FF0300AF8
:1040A0008AF311880026B346A76A4FB949462046CD
:1040B000FFF7A0FF20B187F311883046BDE8F88FE5
:1040C000D4E90A073A1AA8EB0607974228BF174611
:1040D000402F1BD905F1400355F8042B9D4240F8B1
:1040E000042BF9D1A36A40364033A362D4E90A23F2
:1040F0009A4204D3E16920460439FFF795FF8BF318
:1041000011884645D9D28AF31188CDE729463A4627
:10411000FCF75CFFA36A3D443E443B44A362E5E7F1
:10412000D0E904239A4217D1C3689BB1836A8BB14B
:10413000043B9B1A0ED01360C368013BC360C36984
:104140001A4483699A42026124BF436A03610023CF
:1041500083620123184670470023FBE700F060BA32
:10416000014B586A704700BF000C0040034B00220F
:1041700058631A610222DA60704700BF000C0040E9
:10418000014B0022DA607047000C0040014B58637D
:10419000704700BF000C0040024B034A1A60034AFC
:1041A0005A6070476C48002010490020000002202F
:1041B000074B494210B55C68201A08401968821AFA
:1041C0008A4203D3A24201D85A6010BD0020FCE706
:1041D0006C48002008B5302383F31188FFF7E8FF0F
:1041E000002383F3118808BD04480121044B0360B8
:1041F0000023C0E901330C3000F016B974480020E8
:10420000D5410008CB1D083A23F00703591A521A6A
:10421000012110B4D2080024C0E9004384600C30AE
:104220001C605A605DF8044B00F0FEB82DE9F84FB1
:10423000364ECD1D0F46002818BF0646082A4FEA05
:10424000D50538BF082206F10C08341D91464046BA
:1042500000F006F909F10701C9F1000E22462468B1
:104260006CB9404600F006F93368CBB308224946E2
:10427000E8009847044698B340E9026730E004EB51
:10428000010CD4F804A00CEA0E0C0AF10100ACF108
:10429000080304EBC0009842E0D9A0EB0C0CB5EB8E
:1042A000EC0F4FEAEC0BD9D89C421CD204F1080267
:1042B000AB45A3EB02024FEAE202626009D9691C36
:1042C000ED43206803EBC1025D44556043F83100C3
:1042D00022601C465F60404644F8086B00F0CAF854
:1042E0002046BDE8F88FAA45216802D11160234617
:1042F000EFE7013504EBC50344F8351003F108017D
:10430000401AC01058601360F1E700BF74480020E5
:10431000F8B550F8043C044650F8085CA0F10806D3
:1043200007332F1D0C35DB0840F8043C284600F00D
:1043300097F83B469F421A6801D0B34228D20AB18F
:10434000964225D244F8082C54F8042C1E60013201
:1043500054F8081C06EBC200814206D148680244AA
:1043600044F8042C0A6844F8082C5868411C03EBF4
:10437000C1018E4207D154F8042C013202445A6024
:1043800054F8082C1A602846BDE8F84000F072B8CE
:104390001346CFE7FEE7000070B51B4B002504462F
:1043A00086B058600E4685620163FEF7EDFE04F1AB
:1043B0001003A560E562C4E904334FF0FF33C4E99C
:1043C0000044C4E90635FFF7CBFE2B46024604F154
:1043D00034012046C4E9082380230C4A2565FEF7F2
:1043E00041F901230A4AE060009203756846726849
:1043F0000192B268CDE90223064BCDE90435FEF700
:1044000059F906B070BD00BF302B0020444F0008A2
:10441000494F000895430008024AD36A1843D06206
:10442000704700BFC8280020C0E9000081607047C5
:104430008368013B002B10B583600CDA074BDC6806
:104440004368A061206063601C6044600520FEF743
:104450007BF8A06910BD0020FCE700BFC828002041
:1044600008B5302383F31188FFF7E2FF002383F3BD
:10447000118808BD08B5302383F3118883680133A0
:10448000002B836007DC036800211A68026050601B
:104490001846FEF785F8002383F3118808BD000055
:1044A0004B6843608B688360CB68C3600B69436172
:1044B0004B6903628B6943620B68036070470000BD
:1044C00008B53C4B40F2FF713B48D3F888200A43C3
:1044D000C3F88820D3F8882022F4FF6222F0070274
:1044E000C3F88820D3F88820D3F8E0200A43C3F823
:1044F000E020D3F808210A43C3F808212F4AD3F853
:1045000008311146FFF7CCFF00F5806002F11C0175
:10451000FFF7C6FF00F5806002F13801FFF7C0FF2A
:1045200000F5806002F15401FFF7BAFF00F58060EA
:1045300002F17001FFF7B4FF00F5806002F18C0119
:10454000FFF7AEFF00F5806002F1A801FFF7A8FFBA
:1045500000F5806002F1C401FFF7A2FF00F5806062
:1045600002F1E001FFF79CFF00F5806002F1FC0121
:10457000FFF796FF02F58C7100F58060FFF790FF62
:1045800000F01AF90E4BD3F8902242F00102C3F862
:104590009022D3F8942242F00102C3F8942205221B
:1045A000C3F898204FF06052C3F89C20054AC3F826
:1045B000A02008BD0044025800000258504F0008D7
:1045C00000ED00E01F00080308B500F0D7FAFEF781
:1045D00023F8104BD3F8DC2042F04002C3F8DC2073
:1045E000D3F8042122F04002C3F80421D3F80431A7
:1045F000094B1A6842F008021A601A6842F0040275
:104600001A60FEF79BFDFEF705FDBDE80840FEF7CA
:104610007BBA00BF004402580018024870470000EF
:10462000114BD3F8E82042F00802C3F8E820D3F891
:10463000102142F00802C3F810210C4AD3F81031BF
:10464000D36B43F00803D363C722094B9A624FF040
:10465000FF32DA6200229A615A63DA605A600122FC
:104660005A611A60704700BF004402580010005C95
:10467000000C0040094A08B51169D3680B40D9B253
:104680009B076FEA0101116107D5302383F311887D
:10469000FDF7DCFF002383F3118808BD000C004008
:1046A000064BD3F8DC200243C3F8DC20D3F8042106
:1046B0001043C3F80401D3F8043170470044025892
:1046C00008B53C4B4FF0FF31D3F8802062F0004238
:1046D000C3F88020D3F8802002F00042C3F8802085
:1046E000D3F88020D3F88420C3F88410D3F8842032
:1046F0000022C3F88420D3F88400D86F40F0FF4034
:1047000040F4FF0040F4DF4040F07F00D867D86FEE
:1047100020F0FF4020F4FF0020F4DF4020F07F0075
:10472000D867D86FD3F888006FEA40506FEA5050CE
:10473000C3F88800D3F88800C0F30A00C3F88800E3
:10474000D3F88800D3F89000C3F89010D3F8900005
:10475000C3F89020D3F89000D3F89400C3F89410D5
:10476000D3F89400C3F89420D3F89400D3F89800B9
:10477000C3F89810D3F89800C3F89820D3F898009D
:10478000D3F88C00C3F88C10D3F88C00C3F88C20BD
:10479000D3F88C00D3F89C00C3F89C10D3F89C107D
:1047A000C3F89C20D3F89C30FCF76EFEBDE80840AF
:1047B00000F0B8B90044025808B50122534BC3F8C1
:1047C0000821534BD3F8F42042F00202C3F8F4203E
:1047D000D3F81C2142F00202C3F81C210222D3F8B4
:1047E0001C314C4BDA605A689104FCD54A4A1A6075
:1047F00001229A60494ADA6000221A614FF440426D
:104800009A61444B9A699204FCD51A6842F480720A
:104810001A603F4B1A6F12F4407F04D04FF480327D
:104820001A6700221A671A6842F001021A60384BB0
:104830001A685007FCD500221A611A6912F0380272
:10484000FBD1012119604FF0804159605A67344A09
:10485000DA62344A1A611A6842F480321A602C4BC8
:104860001A689103FCD51A6842F480521A601A68DB
:104870009204FCD52C4A2D499A6200225A6319638E
:1048800001F57C01DA6301F2E71199635A64284A61
:104890001A64284ADA621A6842F0A8521A601C4B5D
:1048A0001A6802F02852B2F1285FF9D148229A61C1
:1048B0004FF48862DA6140221A621F4ADA641F4AA2
:1048C0001A651F4A5A651F4A9A6532231E4A1360A9
:1048D000136803F00F03022BFAD10D4A136943F05A
:1048E00003031361136903F03803182BFAD14FF057
:1048F0000050FFF7D5FE4FF08040FFF7D1FE4FF09C
:104900000040BDE80840FFF7CBBE00BF008000516B
:10491000004402580048025800C000F002000001A4
:104920000000FF01008890081210200063020901B6
:10493000470E0508DD0BBF0120000020000001101C
:104940000910E00000010110002000524FF0B042B9
:1049500008B5D2F8883003F00103C2F8883023B1DB
:10496000044A13680BB150689847BDE80840FEF749
:1049700033BC00BF8C4800204FF0B04208B5D2F8DD
:10498000883003F00203C2F8883023B1044A9368E8
:104990000BB1D0689847BDE80840FEF71DBC00BFCA
:1049A0008C4800204FF0B04208B5D2F8883003F0B0
:1049B0000403C2F8883023B1044A13690BB150696B
:1049C0009847BDE80840FEF707BC00BF8C480020B0
:1049D0004FF0B04208B5D2F8883003F00803C2F8AF
:1049E000883023B1044A93690BB1D0699847BDE878
:1049F0000840FEF7F1BB00BF8C4800204FF0B042EA
:104A000008B5D2F8883003F01003C2F8883023B11B
:104A1000044A136A0BB1506A9847BDE80840FEF794
:104A2000DBBB00BF8C4800204FF0B04310B5D3F87B
:104A3000884004F47872C3F88820A30604D5124A8B
:104A4000936A0BB1D06A9847600604D50E4A136B7F
:104A50000BB1506B9847210604D50B4A936B0BB1F1
:104A6000D06B9847E20504D5074A136C0BB1506C24
:104A70009847A30504D5044A936C0BB1D06C9847B2
:104A8000BDE81040FEF7A8BB8C4800204FF0B043B3
:104A900010B5D3F8884004F47C42C3F8882062053E
:104AA00004D5164A136D0BB1506D9847230504D5F4
:104AB000124A936D0BB1D06D9847E00404D50F4AAC
:104AC000136E0BB1506E9847A10404D50B4A936E38
:104AD0000BB1D06E9847620404D5084A136F0BB12E
:104AE000506F9847230404D5044A936F0BB1D06FDD
:104AF0009847BDE81040FEF76FBB00BF8C48002010
:104B000008B50348FCF728FEBDE80840FEF764BB83
:104B10005C24002008B5FFF7ADFDBDE80840FEF7B6
:104B20005BBB0000062108B50846FCF79BFE06218A
:104B30000720FCF797FE06210820FCF793FE0621CC
:104B40000920FCF78FFE06210A20FCF78BFE0621C8
:104B50001720FCF787FE06212820FCF783FE092199
:104B60007A20FCF77FFE07213220FCF77BFE0C2128
:104B70002520BDE80840FCF775BE000008B5FFF72A
:104B80009FFD00F00DF8FDF72BF8FDF703FAFDF798
:104B9000D5F8FFF743FDBDE80840FFF7DFBA000096
:104BA0000023054A19460133102BC2E9001102F116
:104BB0000802F8D1704700BF8C48002010B50139B9
:104BC0000244904201D1002005E0037811F8014F22
:104BD000A34201D0181B10BD0130F2E7034611F8C3
:104BE000012B03F8012B002AF9D1704753544D33A0
:104BF0003248373F3F3F0053544D333248373378C4
:104C00002F3732780053544D3332483734332F37EF
:104C100035332F373530000001105A00031059008A
:104C200001205800032056001000024008000240F6
:104C30000008024000000B0028000240080002406B
:104C40000408024006010C00400002400800024037
:104C50000808024010020D005800024008000240FF
:104C60000C08024016030E00700002400C000240C7
:104C70001008024000040F00880002400C000240AF
:104C80001408024006051000A00002400C0002407B
:104C90001808024010061100B80002400C00024043
:104CA0001C08024016072F001004024008040240AE
:104CB000200802400008380028040240080402408E
:104CC000240802400609390040040240080402405A
:104CD00028080240100A3A00580402400804024022
:104CE0002C080240160B3B00700402400C040240EA
:104CF00030080240000C3C00880402400C040240D2
:104D000034080240060D4400A00402400C04024096
:104D100038080240100E4500B80402400C0402405E
:104D20003C080240160F46000096000000000000FC
:104D30000000000000000000000000000000000073
:104D400000000000A11B00088D1B0008C91B000803
:104D5000B51B0008C11B0008AD1B0008991B00080B
:104D6000851B0008D51B000800000000B91C0008C6
:104D7000A51C0008E11C0008CD1C0008D91C000877
:104D8000C51C0008B11C00089D1C0008ED1C000893
:104D9000000000000100000000000000633000007F
:104DA0009C4D000820290020302B002041726475A2
:104DB00050696C6F740025424F415244252D424C7E
:104DC000002553455249414C2500000002000000D7
:104DD00000000000D91E0008491F000840004000E4
:104DE000E0430020F043002002000000000000002B
:104DF0000300000000000000911F000800000000F8
:104E0000100000000044002000000000010000002D
:104E1000000000001C47002001010200A52A000834
:104E2000B5290008512A0008352A0008430000006F
:104E3000344E000809024300020100C03209040098
:104E400000010202010005240010010524010001F7
:104E5000042402020524060001070582030800FF5E
:104E600009040100020A00000007050102400000D9
:104E7000070581024000000012000000804E00087B
:104E80001201100102000040091241570002010204
:104E9000030100000403090425424F415244250048
:104EA0004D69636F41697237343376320030313285
:104EB00033343536373839414243444546000000E3
:104EC000000000200000020002000000000000308E
:104ED000000004000800000000000024000008009A
:104EE000040000000004000000FC000002000000BC
:104EF00000000430008000000800000000000038BE
:104F0000000001000100000000000000ED2000088A
:104F1000A523000851240008400040005448002008
:104F20005448002001000000644800208000000078
:104F30004001000008000000000100000010000017
:104F4000080000006D61696E0069646C6500000016
:104F50000000A86A00000000AAAAAAAA000014641F
:104F6000FFFF00000000000070A70A000000000121
:104F700000000000AAAAAAAA00000001FFFF00008A
:104F80000000000000000000000000000000000021
:104F9000AAAAAAAA00000000FFFF0000000000006B
:104FA000000000000005000000000000AAAAAAAA54
:104FB00000050000FFFF00000000000000000000EE
:104FC0001001000000000000AAAAAAAA0000000028
:104FD000EBFF0000000000000000000000000000E7
:104FE00000000000AAAAAAAA00000000FFFF00001B
:104FF00000000000000000000000000000000000B1
:10500000AAAAAAAA00000000FFFF000000000000FA
:10501000000000000000000000000000AAAAAAAAE8
:1050200000000000FFFF0000000000000000000082
:105030000000000000000000AAAAAAAA00000000C8
:10504000FFFF000000000000000000000000000062
:1050500000000000AAAAAAAA00000000FFFF0000AA
:105060000000000000000000000000000000000040
:10507000AAAAAAAA00000000FFFF0000000000008A
:1050800000000000000000009B0400000000000081
:1050900000001A0000000000FF000000382B002074
:1050A0005C24002000000000EC4B0008830400009A
:1050B000F74B000850040000054C00080096000063
:1050C0000000080096000000000800000400000036
:1050D000944E0008000000000000000000000000E6
:1050E000000000000000000000000000FFFFFFFFC4
:1050F000FFFFFFFFFFFFFFFFFFFFFFFFFFFFFFFFC0
:10510000FFFFFFFFFFFFFFFFFFFFFFFFFFFFFFFFAF
:10511000FFFFFFFFFFFFFFFFFFFFFFFFFFFFFFFF9F
:10512000FFFFFFFFFFFFFFFFFFFFFFFFFFFFFFFF8F
:020000040801F1
:020000040802F0
:1000000000060030510D0208418B08089D8A08083F
:10001000098B08089D8A0808D58A0808530D02082C
:10002000530D0208530D0208530D020879F90A080E
:10003000530D0208530D0208530D0208530D020818
:10004000530D0208530D0208530D0208530D020808
:10005000530D0208530D020809090B0835090B0856
:1000600061090B088D090B08B9090B089DA30A0843
:10007000C5A30A08F1A30A081DA40A0849A40A088E
:1000800071A40A089DA40A08C19F0A08530D02081A
:10009000530D0208530D0208530D0208E5090B0821
:1000A000530D0208710B0B08530D0208850B0B084A
:1000B000530D0208890B0B089D0B0B082DAC0A0889
:1000C0005DAC0A088DAC0A08BDAC0A08D5B50A08B3
:1000D000EDB50A08D10A0B08E50A0B08F90A0B0866
:1000E000490A0B08530D0208530D0208B10B0B0807
:1000F000530D0208530D0208530D0208C9A40A0843
:10010000530D0208BD0A0B08530D020805B60A0874
:100110000D0B0B08210B0B08530D0208530D0208A1
:10012000F5A40A081DA50A0849A50A0875A50A0824
:10013000A1A50A08530D0208530D0208530D020829
:10014000530D0208530D0208530D0208530D020807
:10015000C9A50A08F5A50A0821A60A08350B0B0847
:10016000530D0208530D0208530D0208530D0208E7
:10017000530D020865050B08530D0208530D0208C4
:10018000530D0208530D0208490B0B085D0B0B08B9
:10019000530D0208530D0208530D0208530D0208B7
:1001A000530D0208530D0208530D0208530D0208A7
:1001B000530D0208530D0208530D0208530D020897
:1001C000530D0208530D0208530D0208530D020887
:1001D000530D020851050B08530D0208530D020878
:1001E000530D0208530D0208530D0208530D020867
:1001F000530D0208530D0208530D0208530D020857
:10020000530D0208530D0208530D0208530D020846
:10021000530D0208530D0208530D0208530D020836
:10022000530D0208530D0208530D0208530D020826
:10023000530D0208530D0208530D0208E19F0A08EE
:10024000530D020869A10A0891A10A08BDA10A0874
:10025000E9A10A0815A20A0841A20A086DA20A0823
:1002600099A20A08530D0208530D0208530D020803
:10027000530D0208530D0208530D0208530D0208D6
:10028000530D0208530D0208530D0208530D0208C6
:10029000530D0208530D0208530D0208530D0208B6
:1002A000530D0208530D0208530D0208530D0208A6
:1002B000530D0208530D0208530D0208530D020896
:1002C000530D0208530D0208530D0208530D020886
:1002D000530D0208530D0208530D0208530D020876
:1002E00065250208C13502083D940208090B04087F
:1002F0009919060859380608959E060859A6060851
:1003000099A90608C91407088531070839BB0708E9
:1003100095D00708EDDD07082D7C0808A5810808A1
:10032000C5660908F58609087DD9090825010A0866
:1003300019180A086D490A08314F0A080000000020
:1003400081F0004102E000BF83F0004330B54FEA86
:1003500041044FEA430594EA050F08BF90EA020FF3
:100360001FBF54EA000C55EA020C7FEA645C7FEA86
:10037000655C00F0E2804FEA5454D4EB5555B8BFA9
:100380006D420CDD2C4480EA020281EA030382EA1A
:10039000000083EA010180EA020281EA0303362DAC
:1003A00088BF30BD11F0004F4FEA01314FF4801C7F
:1003B0004CEA113102D0404261EB410113F0004F91
:1003C0004FEA03334CEA133302D0524263EB430348
:1003D00094EA050F00F0A780A4F10104D5F1200EE6
:1003E0000DDB02FA0EFC22FA05F2801841F1000141
:1003F00003FA0EF2801843FA05F359410EE0A5F115
:1004000020050EF1200E012A03FA0EFC28BF4CF045
:10041000020C43FA05F3C01851EBE37101F00045FB
:1004200007D54FF0000EDCF1000C7EEB00006EEB08
:100430000101B1F5801F1BD3B1F5001F0CD3490892
:100440005FEA30004FEA3C0C04F101044FEA4452E9
:1004500012F5800F80F09A80BCF1004F08BF5FEA70
:10046000500C50F1000041EB045141EA050130BD50
:100470005FEA4C0C404141EB0101013C28BFB1F562
:10048000801FE9D291F0000F04BF01460020B1FAAD
:1004900081F308BF2033A3F10B03B3F120020CDA80
:1004A0000C3208DD02F1140CC2F10C0201FA0CF05E
:1004B00021FA02F10CE002F11402D8BFC2F1200CC3
:1004C00001FA02F120FA0CFCDCBF41EA0C01904079
:1004D000E41AA2BF01EB0451294330BD6FEA0404C2
:1004E0001F3C1CDA0C340EDC04F11404C4F12002AD
:1004F00020FA04F001FA02F340EA030021FA04F3BF
:1005000045EA030130BDC4F10C04C4F1200220FA15
:1005100002F001FA04F340EA0300294630BD21FA53
:1005200004F0294630BD94F0000F83F4801306BF19
:1005300081F480110134013D4EE77FEA645C18BF0D
:100540007FEA655C29D094EA050F08BF90EA020FA4
:1005500005D054EA000C04BF1946104630BD91EA9C
:10056000030F1EBF0021002030BD5FEA545C05D19F
:100570004000494128BF41F0004130BD14F58004DE
:100580003CBF01F5801130BD01F0004545F0FE4152
:1005900041F470014FF0000030BD7FEA645C1ABF87
:1005A000194610467FEA655C1CBF0B46024650EABE
:1005B000013406BF52EA033591EA030F41F40021EA
:1005C00030BD00BF90F0000F04BF0021704730B570
:1005D0004FF4806404F132044FF000054FF0000145
:1005E00050E700BF90F0000F04BF0021704730B506
:1005F0004FF4806404F1320410F0004548BF4042DB
:100600004FF000013EE700BF42004FEAE2014FEA2F
:1006100031014FEA02701FBF12F07F4393F07F4F0A
:1006200081F06051704732F07F4208BF704793F00D
:100630007F4F04BF41F40021704730B54FF4607420
:1006400001F0004521F000411CE700BF50EA010223
:1006500008BF704730B54FF000050AE050EA0102CC
:1006600008BF704730B511F0004502D5404261EB3C
:1006700041014FF4806404F132045FEA915C3FF47D
:10068000D8AE4FF003025FEADC0C18BF03325FEA1A
:10069000DC0C18BF033202EBDC02C2F1200300FACB
:1006A00003FC20FA02F001FA03FE40EA0E0021FAF0
:1006B00002F11444BDE600BF80F0004002E000BF3C
:1006C00081F0004142001FBF5FEA410392EA030F3D
:1006D0007FEA226C7FEA236C6AD04FEA1262D2EB87
:1006E0001363C1BFD218414048404140B8BF5B428C
:1006F000192B88BF704710F0004F40F4000020F025
:100700007F4018BF404211F0004F41F4000121F03A
:100710007F4118BF494292EA030F3FD0A2F1010284
:1007200041FA03FC10EB0C00C3F1200301FA03F1C2
:1007300000F0004302D5494260EB4000B0F5000FE5
:1007400013D3B0F1807F06D340084FEA310102F1A4
:100750000102FE2A51D2B1F1004F40EBC25008BF56
:1007600020F0010040EA03007047490040EB000020
:10077000013A28BFB0F5000FEDD2B0FA80FCACF121
:10078000080CB2EB0C0200FA0CF0AABF00EBC2504E
:1007900052421843BCBFD0401843704792F0000F3C
:1007A00081F4000106BF80F400000132013BB5E78F
:1007B0004FEA41037FEA226C18BF7FEA236C21D005
:1007C00092EA030F04D092F0000F08BF084670476A
:1007D00090EA010F1CBF0020704712F07F4F04D138
:1007E000400028BF40F00040704712F100723CBF4B
:1007F00000F50000704700F0004343F0FE4040F475
:10080000000070477FEA226216BF08467FEA236332
:100810000146420206BF5FEA412390EA010F40F41D
:10082000800070474FF0000304E000BF10F0004369
:1008300048BF40425FEA000C08BF704743F0964350
:1008400001464FF000001CE050EA010208BF70476B
:100850004FF000030AE000BF50EA010208BF7047F2
:1008600011F0004302D5404261EB41015FEA010C07
:1008700002BF84460146002043F0B64308BFA3F1FF
:100880008053A3F50003BCFA8CF2083AA3EBC253E1
:1008900010DB01FA02FC634400FA02FCC2F1200200
:1008A000BCF1004F20FA02F243EB020008BF20F037
:1008B0000100704702F1200201FA02FCC2F120029D
:1008C00050EA4C0021FA02F243EB020008BF20EA92
:1008D000DC7070477BB972B90029BEBF00204FF0B1
:1008E000004106E008BF00281CBF6FF000414FF038
:1008F000FF3000F02BBAADF1080C6DE904CE0029F1
:1009000009DB002B1ADB00F0B9F8DDF804E0DDE9C3
:10091000022304B07047404261EB4101002B1BDB16
:1009200000F0ACF8DDF804E0DDE9022304B0404259
:1009300061EB4101524263EB43037047524263EB68
:10094000430300F09BF8DDF804E0DDE9022304B086
:10095000404261EB41017047524263EB430300F0B8
:100960008DF8DDF804E0DDE9022304B0524263EBC8
:100970004303704753B94AB9002908BF00281CBF78
:100980004FF0FF314FF0FF3000F0E0B9ADF1080C4F
:100990006DE904CE00F072F8DDF804E0DDE9022331
:1009A00004B07047430803F05533C01A830803F0BE
:1009B000333300F03330184400EB101000F00F30E8
:1009C00000EB002000EB0040000E704708B5024627
:1009D0000B4643EC172BB5EEC07BF1EE10FA03D4B7
:1009E000BDE8084000F02AB8B1EE477B51EC170B88
:1009F00000F024F8404261EB410108BD9FED0B6B14
:100A000007EE900A9FED0B5BB7EEE77A27EE066BD9
:100A1000BCEEC66BB8EE464BA4EE457BFCEEC77B46
:100A200016EE101A17EE900A704700BF0000000083
:100A30000000F03D000000000000F0419FED0B6B56
:100A400041EC170B9FED0B5B27EE066BBCEEC66B04
:100A5000B8EE464BA4EE457BFCEEC77B16EE101AB3
:100A600017EE900A704700BFAFF30080000000004F
:100A70000000F03D000000000000F0412DE9F047CB
:100A8000089D04468E46002B4DD18A42944669D972
:100A9000B2FA82F252B101FA02F3C2F1200120FA55
:100AA00001F10CFA02FC41EA030E94404FEA1C48A3
:100AB000210CBEFBF8F61FFA8CF708FB16E341EA9F
:100AC000034306FB07F199420AD91CEB030306F125
:100AD000FF3080F01F81994240F21C81023E634446
:100AE0005B1AA4B2B3FBF8F008FB103344EA0344EA
:100AF00000FB07F7A7420AD91CEB040400F1FF33FF
:100B000080F00A81A74240F207816444023840EA3B
:100B10000640E41B00261DB1D4400023C5E9004374
:100B20003146BDE8F0878B4209D9002D00F0EF80F7
:100B30000026C5E9000130463146BDE8F087B3FA2A
:100B400083F6002E4AD18B4202D3824200F2F98012
:100B5000841A61EB030301209E46002DE0D0C5E915
:100B6000004EDDE702B9FFDEB2FA82F2002A40F061
:100B70009280A1EB0C014FEA1C471FFA8CFE012664
:100B8000200CB1FBF7F307FB131140EA01410EFB08
:100B900003F0884208D91CEB010103F1FF3802D2AF
:100BA000884200F2CB804346091AA4B2B1FBF7F0A9
:100BB00007FB101144EA01440EFB00FEA64508D9CC
:100BC0001CEB040400F1FF3102D2A64500F2BB8009
:100BD0000846A4EB0E0440EA03409CE7C6F1200758
:100BE000B34022FA07FC4CEA030C20FA07F401FA9E
:100BF00006F31C43F9404FEA1C4900FA06F3B1FB27
:100C0000F9F8200C1FFA8CFE09FB181140EA01418B
:100C100008FB0EF0884202FA06F20BD91CEB010128
:100C200008F1FF3A80F08880884240F28580A8F180
:100C300002086144091AA4B2B1FBF9F009FB1011D2
:100C400044EA014100FB0EFE8E4508D91CEB010170
:100C500000F1FF346CD28E456AD90238614440EA13
:100C60000840A0FB0294A1EB0E01A142C846A64693
:100C700056D353D05DB1B3EB080261EB0E0101FA1C
:100C800007F722FA06F3F1401F43C5E90071002679
:100C90003146BDE8F087C2F12003D8400CFA02FCCF
:100CA00021FA03F3914001434FEA1C471FFA8CFEDF
:100CB000B3FBF7F007FB10360B0C43EA064300FBCF
:100CC0000EF69E4204FA02F408D91CEB030300F16D
:100CD000FF382FD29E422DD9023863449B1B89B224
:100CE000B3FBF7F607FB163341EA034106FB0EF3AD
:100CF0008B4208D91CEB010106F1FF3816D28B425A
:100D000014D9023E6144C91A46EA004638E72E4625
:100D1000284605E70646E3E61846F8E64B45A9D21D
:100D2000B9EB020864EB0C0E0138A3E74646EAE78C
:100D3000204694E74046D1E7D0467BE7023B61443A
:100D400032E7304609E76444023842E7704700BFA3
:100D500002E000F000F8FEE772B6374880F308883A
:100D6000364880F3098836483649086040F200006A
:100D7000CCF200004EF63471CEF200010860BFF3F1
:100D80004F8FBFF36F8F40F20000C0F2F0004EF6BD
:100D90008851CEF200010860BFF34F8FBFF36F8F11
:100DA0004FF00000E1EE100A4EF63C71CEF2000169
:100DB0000860062080F31488BFF36F8F8EF03EFE2C
:100DC0008DF06AFD4FF055301F491B4A91423CBFE0
:100DD00041F8040BFAE71D49184A91423CBF41F81B
:100DE000040BFAE71A491B4A1B4B9A423EBF51F8C3
:100DF000040B42F8040BF8E700201849184A914206
:100E00003CBF41F8040BFAE78EF056FE8DF0C8FDAA
:100E1000144C154DAC4203DA54F8041B8847F9E72B
:100E200001F090FB114C124DAC4203DA54F8041B54
:100E30008847F9E78EF03EBE000600300022003001
:100E40000000020808ED00E000000030000600305D
:100E500028950D0800220030B0250030B025003064
:100E6000C8CB0130E00202083C0302083C03020840
:100E70003C0302082DE9F04F2DED108AC1F80CD08B
:100E8000D0F80CD0BDEC108ABDE8F08F002383F3BE
:100E900011882846A04700208DF06EFAFEE78DF0FD
:100EA000DDF800DFFEE7000070B54FF0FF0C4CF4FA
:100EB000E06C1CEA11541DBF1CEA135594EA0C0F98
:100EC00095EA0C0F00F0DEF82C4481EA030621EAD3
:100ED0004C5123EA4C5350EA013518BF52EA03350E
:100EE00041F4801143F4801338D0A0FB02CE4FF0C0
:100EF0000005E1FB02E506F00042E0FB03E54FF0F0
:100F00000006E1FB03569CF0000F18BF4EF0010EE7
:100F1000A4F1FF04B6F5007F64F5407404D25FEAE3
:100F20004E0E6D4146EB060642EAC62141EA555196
:100F30004FEAC52040EA5E504FEACE2EB4F1FD0CD8
:100F400088BFBCF5E06F1ED8BEF1004F08BF5FEA56
:100F5000500E50F1000041EB045170BD06F0004608
:100F600046EA010140EA020081EA0301B4EB5C04B5
:100F7000C2BFD4EB0C0541EA045170BD41F48011AD
:100F80004FF0000E013C00F3AB8014F1360FDEBFD2
:100F9000002001F0004170BDC4F10004203C35DAAE
:100FA0000C341BDC04F11404C4F1200500FA05F331
:100FB00020FA04F001FA05F240EA020001F00042D2
:100FC00021F0004110EBD37021FA04F642EB060148
:100FD0005EEA430E08BF20EAD37070BDC4F10C0472
:100FE000C4F1200500FA04F320FA05F001FA04F236
:100FF00040EA020001F0004110EBD37041F1000122
:101000005EEA430E08BF20EAD37070BDC4F120052C
:1010100000FA05F24EEA020E20FA04F301FA05F294
:1010200043EA020321FA04F001F0004121FA04F23C
:1010300020EA020000EBD3705EEA430E08BF20EA0C
:10104000D37070BD94F0000F0FD101F00046400046
:1010500041EB010111F4801F08BF013CF7D041EAC8
:10106000060195F0000F18BF704703F000465200CC
:1010700043EB030313F4801F08BF013DF7D043EA9D
:101080000603704794EA0C0F0CEA135518BF95EA53
:101090000C0F0CD050EA410618BF52EA4306D1D1DA
:1010A00081EA030101F000414FF0000070BD50EAF9
:1010B000410606BF1046194652EA430619D094EA83
:1010C0000C0F02D150EA013613D195EA0C0F05D16D
:1010D00052EA03361CBF104619460AD181EA0301C1
:1010E00001F0004141F0FE4141F470014FF0000079
:1010F00070BD41F0FE4141F4780170BD4FEA4102FC
:1011000012F5001215D211D56FF47873B3EB625259
:1011100012D94FEAC12343F0004343EA505311F080
:10112000004F23FA02F018BF404270474FF0000012
:10113000704750EA013005D111F0004008BF6FF050
:10114000004070474FF00000704700BF4FEA410277
:10115000B2F1E04324BFB3F5001CDCF1FE5C0DD915
:1011600001F0004C4FEAC0024CEA5070B2F1004F5F
:1011700040EB830008BF20F00100704711F0804F62
:1011800021D113F13872BCBF01F00040704741F427
:1011900080114FEA5252C2F11802C2F1200C10FA2B
:1011A0000CF320FA02F018BF40F001004FEAC1230F
:1011B0004FEAD32303FA0CFC40EA0C0023FA02F3B3
:1011C0004FEA4303CCE77FEA625307D150EA013389
:1011D0001EBF4FF0FE4040F44000704701F0004059
:1011E00040F0FE4040F40000704700BF01F0FF01F6
:1011F000102A2BDB10F0070F08D010F8013B013A42
:101200008B422DD010F0070F42B3F6D1F0B441EA73
:10121000012141EA014122F007047FF00007002389
:10122000F0E80256083C85EA010586EA010685FADF
:1012300047F5A3FA87F586FA47F6A5FA87F68EB939
:10124000EED1F0BC01F0FF0102F0070232B110F85C
:10125000013B013A83EA010313B1F8D10020704742
:1012600001387047002D06BF35460338073815F0A2
:10127000010F07D1013015F4807F02BF013015F452
:10128000C03F0130F0BC0138704700BF10F8012B9F
:1012900011F8013B012A28BF9A42F7D0D01A7047B3
:1012A000034613F8012B002AFBD1181A01387047A6
:1012B0000020704770470000704700007047000032
:1012C00000207047002070470020704701207047C1
:1012D00000207047704700000020704700207047D2
:1012E00070470000704700000020704700207047E2
:1012F00070B5154ED6F8C00D03681B6898470428D2
:101300001ADC01281DDC002814BF012441240F4BE6
:101310001D68E86A0368DB69984701280AD0D6F897
:10132000C02D0B4B9A4205D0EB6A93F89C300BB161
:1013300044F08004204670BD0A2814BF01241924FB
:10134000E5E71924E3E700BFB8550030B4250030C5
:1013500080630030044B03F6C852D3F8C00D9042AE
:1013600014BF042002207047B8550030014B93F899
:10137000A80A7047B84500307047000038B5C578F6
:101380000B4604461C221C2D4FF00001184628BFB6
:101390001C2593F025FD04F10C012A46BDE83840D8
:1013A00093F0D4BC38B5C5780B4604461022102DF6
:1013B0004FF00001184628BF102593F011FD04F1ED
:1013C0000C012A46BDE8384093F0C0BC08B54BF08C
:1013D00073FA30B9034A92F8543E43F0040382F89A
:1013E000543E08BDB855003038B5F7EE000A91ED0F
:1013F000000A0D4619F0D6FB20B10B4801F050FF52
:10140000002038BDD5ED007A9FED087AF0EEE77A3E
:10141000F4EEC77AF1EE10FA03D5034801F054FF59
:10142000EEE70320EDE700BFB825003000000034F0
:1014300010B5044608F010F8204610BD13B58B8B8C
:101440000C46B72B07D0B3F5967F21D002B0BDE88C
:1014500010404FF093BB1E221149124801F05EFF6D
:10146000D4ED017A94ED007AFCEEE77A0C48BCEEFC
:10147000C77A17EE903A8DED017A9AB29DF8041072
:1014800001F0DAFB002814BF0020042002B010BDD8
:1014900004480222044901F041FF0020F6E700BFA2
:1014A000A8630030B82500307C630030244BDFEDAA
:1014B000256A03F6486200B592ED007A03F64C62A5
:1014C0008BB0007CD2ED007AA3F5805292F9CA2A43
:1014D000002A03F63C62116803F6346207FE277A9D
:1014E00003F63863D2ED007A04913E21FDEEE77AEF
:1014F0008DED057A17EE902AD3ED007A0023F4EEF5
:10150000E67A12B203930693F1EE10FA0793ADF860
:101510002020ADF822204FF0B70258BFF0EE667AD7
:10152000FCEEE77A17EE903AADF824301A23CDE9B5
:10153000003203AA48F072FB0BB05DF804FB00BF59
:10154000B855003000FF7F4770B5164C8AB094F84C
:101550005A2E22B90AB0BDE8704049F017BE057C8A
:1015600067F020FBD4F8B86DD4F8BC1DD4F8B43DB6
:10157000A4F50054CDE90513B4F810270023212168
:10158000ADF82430ADF826206822CDE907331C23BE
:10159000CDE90306CDE90032284603AA48F03EFB18
:1015A0000AB070BDB8550030F0B5464C8DB0054658
:1015B000B4F8EC3ADE0743D504F69C3304F6BC32AB
:1015C00004F6983ED3F800C004F53B6312681F6828
:1015D00004F6A433DEF800E01E6804F6A833CDF864
:1015E000252003AA186804F6AC33CDF80CE019687E
:1015F00004F6B833079062201B6808910221CDF8E9
:10160000293021238DF82410C221CDF810C0069670
:101610000597CDE900301923287C48F0FFFA287C93
:1016200048F092FA0646287C49F096F900F1210329
:101630009E4205D2287C0DB0BDE8F04047F0FCBCCE
:10164000B4F8EC3A99073BD504F5496304F54B62CD
:10165000D3F800C004F6A44312681F6804F6984348
:10166000CDF8252062221E6804F69C43CDF810C0F8
:10167000186804F54A630597196804F6AC4304F644
:101680008C4407901B6808910321CDF82930212351
:101690002468287C8DF82410C22103940696CDE995
:1016A0000032192303AA48F0B9FA287C48F04CFA12
:1016B0000446287C49F050F900F121039C42B9D33B
:1016C0000DB0F0BDB845003005207047024BD3F88F
:1016D000C00D03681B681847B855003030B5CD7889
:1016E0008BB00C462722272D4FF00001684628BFFB
:1016F000272593F075FB04F10C0168462A4693F008
:1017000025FB1D4B03F55D62D3F8C01D914230D11E
:10171000DDED057A9FED197AF0EEE77AF4EEC77AFF
:10172000F1EE10FA25D59DF8262002F0410141295D
:101730001FD111061DD402F01801182919D003F683
:10174000D451019882F00402086003F6D85102983F
:10175000C2F38002086003F6DC51039883F8E42D9D
:10176000086003F55E61049803F6E853079A086081
:101770001A600BB030BD00BFB85500300000003417
:1017800030B5194D85B00C4695F8593E4BBBCA781B
:1017900001A80C318DF80C30092A28BF0922CDE9A7
:1017A000013393F0D3FA9DF808305A1F012A18D953
:1017B00003F0F703122B14D0A5F58053B3F9AA2A2E
:1017C00012B9E279A3F8AA2A227AE179074800F04F
:1017D000B5F9227AE179054800F0E8F9012385F8A6
:1017E000593E05B030BD00BFB8550030605B0030D9
:1017F0001B4BF0B5B3F9AA3A89B005460E4614461C
:101800003BB1D779BB4204D009B0BDE8F0404DF000
:10181000A7BBA27A637A43EA0223E27A43EA02434D
:101820001D2B13D0212B08D01BB921462846FFF7CA
:10183000A7FF224631462846E6E701A92046FFF7E2
:101840009DFD01A9074802F01FF8F2E701A9204613
:10185000FFF7A8FD01A9034802F074F8E9E700BF0B
:10186000B8450030B825003013B5CA7800230446C7
:101870000C31072A6846009328BF0722CDF80330B1
:1018800093F064FABDF900304BB901231C212046C6
:1018900084F80F3302B0BDE810404FF027B902B012
:1018A00010BD000030B5CD7889B00C461E221E2D2B
:1018B0004FF00001684628BF1E2593F091FA04F10D
:1018C0000C0168462A4693F041FA6946024802F044
:1018D00089F809B030BD00BFB825003000B589B027
:1018E000084601A9FFF74AFD01A9034801F0CCFF12
:1018F00009B05DF804FB00BFB82500301FB50846ED
:101900006946FFF74FFD6946024802F01BF805B033
:101910005DF804FBB82500302DE9F041CC7894B097
:1019200088462622262C4FF00001074602AD28BF2C
:1019300026240AA893F054FA08F10C0122460AA8BA
:1019400093F004FA284607F06FFA9DF84A3006AC87
:10195000022B03D0032B44D0002B66D1DFED357A68
:101960000023DDED106A9FED346A66EEA76A9DEDF7
:101970000F7ADDED0E7A27EE067A67EE867AFDEEB7
:10198000E66A0093BDEEC77A2046FDEEE77A16EED2
:10199000903A17EE102A17EE901A07F065FA94E8BD
:1019A0000F0085E80F0097F80F3363BB012698F806
:1019B00008302F2198F807208DF8193000238DF872
:1019C000182099228DF81B300423387C8DF81A607A
:1019D000CDE900320323224648F020F914B0BDE8D7
:1019E000F081DFED147A0123DDED106A9FED126ABC
:1019F00066EEA76A9DED0F7ADDED0E7A27EE067A88
:101A000067EE867ABBE7BDF8446086B93246294660
:101A10000A4801F01DFC0028C8D0094A06213846B2
:101A20004AF0E0FB87F80F63C1E70226BFE7002614
:101A3000BDE700BF0000C8428096184BB8250030B3
:101A4000788F0B0838B58A7A05464B7A0C4643EAFC
:101A50000223CA7A43EA0243272B0CD81C2B10D945
:101A60001D3B0A2B0DD8DFE803F01E0C0C0C1B0CE1
:101A70000C0C0C121500452B0FD0522B01D1FFF787
:101A80002DFE21462846BDE838404EF0C5B9FFF787
:101A9000EBFEF6E7FFF740FFF3E7FFF703FFF0E7A2
:101AA000FFF71CFFEDE7FFF729FFEAE7002070478B
:101AB000C820704701207047002070470020704701
:101AC0000120704790F8D8308B4286BF00EB810030
:101AD000D0F8DC000020704790F8D8308B4286BFE9
:101AE00000EB8100D0F8DC0000207047014B93F838
:101AF000A60A7047B8450030C36A43F4E053C36296
:101B0000036B43F4E0530363436B43F4E0534363D9
:101B10007047000013B54FF44470CDE9002107F081
:101B200093FC044628B1DDE900214EF097FB024BFF
:101B30002360204602B010BD18910B082DE9F04F2C
:101B4000064685B00F4690460025DFF85C904FF4BE
:101B5000837AECB296F8D830A34222D9204647F0D7
:101B6000F3FF8346204648F0F7FE031D9B4514D340
:101B700099F9CB3A942242212046ADF80830062349
:101B80008DF80A708DF80B80ADF80CA0CDE900320D
:101B900002AA48F043F80135DBE7204647F04CFA4B
:101BA000F9E705B0BDE8F08FB84500302DE9F04FFA
:101BB000064685B00F4690460025DFF85C9040F25F
:101BC000011AECB296F8D830A34222D9204647F049
:101BD000BBFF8346204648F0BFFE031D9B4514D340
:101BE00099F9CB3A942242212046ADF808300623D9
:101BF0008DF80A708DF80B80ADF80CA0CDE900329D
:101C000002AA48F00BF80135DBE7204647F014FA4A
:101C1000F9E705B0BDE8F08FB84500307047000027
:101C20001FB500F54053002100F5A85003F63C62B3
:101C300003F6346301911030126801A91B68029207
:101C4000039302F03DF803F035FC03F0E3F905B02F
:101C50005DF804FB70B586B006461322002101A88A
:101C600010EE105A10EE904A93F0BAF8A3238DF8B4
:101C7000043095238DF8053066F09CFFCDF8070001
:101C800006F59550CDF80B10132201A91030CDF8B0
:101C90000F50CDF8134042F023FE06B070BD000097
:101CA0002DE9F0418AB004468846174600212322D8
:101CB00001A8109D1E4693F093F8A3238DF80430DD
:101CC00095238DF8053001238DF8063066F072FFFC
:101CD0002B682322CDF8070004F59550CDF81B3072
:101CE0006B681030CDF80B1001A9CDF81F30AB6830
:101CF000CDF80F80CDF81370CDF81760CDF82330F4
:101D000042F0EEFD0AB0BDE8F08100009720704778
:101D100000F5405310B50446D3F8C00D03681B68A6
:101D200098471A22C1B204F59550103042F098FF3E
:101D300004F59070BDE810400FF092BF37B500F584
:101D40002A51044601220125243141F049FA04F5C3
:101D5000225100230F4A3831DA2000953EF07EFCF4
:101D600004F5955100230C4A1031FD2000953EF0FA
:101D700075FC0A4B1A68D20705D404F5A154084A29
:101D80001D60183414600121054803B0BDE83040DF
:101D90003EF0B6BC7C400D08106F0C08B02500303A
:101DA0000022003000207047002070470069C0F317
:101DB000401070470F299DBF302303FB01005030B6
:101DC00000207047002070470120704770470000D6
:101DD00000207047002070470020704700207047A7
:101DE0000020704700207047002070470020704797
:101DF00000207047002070477047000003680022F1
:101E00001B6818471020704700207047704700007B
:101E10000320704701207047704700000120704781
:101E2000002070477047000000F52B503430704799
:101E30000048704748B50B0800F5405008B5D0F889
:101E4000C00D03681B689847C0B208BD034808600E
:101E50000F2111704FF0FF321A607047A4CD0B08AC
:101E600000207047002070477047000016F028BC23
:101E700042F09CBE4FF0B6B94DF0D2B905F0C2BDEC
:101E800006F0A0BD00F006BF00F000BF00F01EBFCE
:101E900001F096BC00F0ECBE00F0F2BE00F05CBFBA
:101EA000234B244A70B5036000F540530446D3F831
:101EB000AC07C3F8A82508B107F0D2FA1E4B23607F
:101EC00004F5005393F8EC2642B9D3F8E8562DB147
:101ED000284615F0CBFA284607F0BEFA04F5A050C4
:101EE00004F6B47504F654761C3063F049FE04F52C
:101EF0009F5051F0F9FAB54204D0183D284614F02D
:101F000029FFF8E70D4B04F52D60C4F8703945F052
:101F100045FF04F6A42045F041FF04F6042045F0F7
:101F20003DFF04F6D81045F039FF204670BD00BFD4
:101F3000D8CE0B08408B0C08B8670C08E41C0C08C2
:101F40004F4B70B5044640F8043B52F0DBFB0025D4
:101F500004F1100004F5805606F05AFE04F1680002
:101F600040F09EF904F590700FF032FA04F5A0608D
:101F700005F0BCFB04F2246007F074FA04F5176066
:101F800016F0DCF904F5736052F044FB30463FF084
:101F9000B1FE04F59550103042F0D6FB04F59E508A
:101FA000043057F049FF04F59F5051F085FA04F5CD
:101FB000A0501C3063F0D0FD04F5A150183040F063
:101FC00079FC04F5A4500C3053F07AFD04F5A553C8
:101FD0002C4A04F5A650103386F8B05413603BF039
:101FE000A7FE04F5A8502946103001F05FFF04F564
:101FF000DB5018305DF0BCFE04F515503C3060F04D
:10200000EFFD04F51A50143062F000FF04F51B5088
:10201000383063F035FB04F51D50103001F0A6FD9B
:1020200004F5225038305EF0BBFB04F5245016490D
:1020300010303EF00FFF04F52450283058F0A0F97E
:1020400004F52750243064F095F804F5005304F5A6
:10205000295083F83C5A14300C4D64F0ABF904F568
:102060002950383045F0F2FC2B6813B1084866F06F
:102070006BFD204607493EF0EDFE20462C6070BD0A
:10208000B8670C086471003084380D0804680030AB
:1020900004CB0B08C0660C089FED225AF7EE004AED
:1020A0009FED214A9FED212AF0EE453ADFED201AFF
:1020B000B0EE453A9FED1F1AF0EE452A9FED1E0A3D
:1020C000F0EE450A10B586B0044654308DED054A51
:1020D0008DED042ACDED031A8DED021A8DED015A16
:1020E0008DED000A5DF050FB9DED015AF7EE004AC0
:1020F0009DED054A04F5A470F0EE453A9DED042AE5
:10210000B0EE453ADDED031AF0EE452A9DED021AD8
:10211000F0EE450A9DED000A5DF036FB204606B064
:1021200010BD00BF00000000CDCCCC3D00007A45C2
:102130000AD7A33CCDCC4C3DCDCC4C3EF0B500F500
:102140000055234B87B00446B5F8A62A1A7051F003
:1021500013F850F083FD204601F078FC04F580531D
:1021600093F88C2712F0010210D102A8019206F018
:102170005BFE04F5A85002A9103002F061FF28B1FF
:10218000236802A9019A2046DB6C9847114E3368F8
:10219000DB6A93F89C7037B195F83E3A1BB966F04C
:1021A00001FDC5F8400A336885F83E7ADB6A93F88A
:1021B0009C20094B5A7140F0E5FA40F037F804F5DD
:1021C0002F502C3007B0BDE8F0405DF02DBB00BFB4
:1021D000E8220030B42500302D670030FFF7AEBF95
:1021E00010B50821044601F0E1F918B118F074F8AF
:1021F00015F0A6FF0121204601F0D8F910B12046C4
:10220000FFF70EFD0421204601F0D0F920B104F5BE
:102210009550103041F058FE1021204601F0C6F9CB
:1022200030B104F59550BDE81040103041F0E6BEE5
:1022300010BD0000FFF7D4BF102926D8DFE801F059
:10224000090D11191525252525251D2525252525AA
:10225000210000F577500C30704700F5775034308E
:10226000704700F577502C30704700F577501030EC
:10227000704700F577503030704700F577500430E4
:10228000704700F577500830704700207047000015
:1022900008B55EF089FB044B1B68DB6A93F89C1061
:1022A000BDE808405EF05CBBB4250030FFF7F0BF2E
:1022B0002DE9FF410446FFF743FE884B43F2340605
:1022C00004F52A5004F5005523602430844FFFF7AD
:1022D000E3FE002304F53350C5F8E03C24304FF012
:1022E00099F9804BC5F8E43C42F6345560194FF03B
:1022F00021FB67513035B542F8D1601904F55657C6
:1023000050F004FE04F5565004F5405504F55756B8
:102310000C30283745F084FF04F55650203604F57C
:102320005A58183045F07CFF002307F11400A5F837
:10233000A4356D4BC5F8A83565F0D2FB3046143690
:102340004AF0EAFE4645F9D11E2340F2CC60C5F8BA
:10235000B0370023A5F8B43707F07CF8C5F8AC0710
:1023600004F55E50383065F0BBFB04F55F503C303F
:1023700065F0B6FB5D4B1A6802B91F605C4B002626
:1023800004F560504021C5F8A8350027594B183096
:10239000029404F57758039304AB009608F13808CB
:1023A00013E90C0005F048FF04F57650303006F0D4
:1023B0003BFD04F577534FF07E5208F104000833DB
:1023C000C5F8C03D4C4BC5F8C43D4C4BC5F8C83DA5
:1023D0004B4BC5F8CC3D4B4BC5F8D03D05F6D4531F
:1023E0001A60DF609F605F60474BC5F8EC3D474B6C
:1023F000C5F8F03D464BC5F8F43D06F015FD08F173
:10240000140006F011FD05F6246304F579524148E5
:102410001F604FF0140C5F6018329F604FF6FF771B
:102420003D4B186033469EB201330CFB0601097C1C
:102430000029F8D1394B3A491E800B6813B139484D
:1024400066F082FB85F8593E04F5795001230A6055
:102450001C3004F57A5685F85A3E64F059F8324B30
:1024600004F57B50C5F8B04EC5F85C3E2F4B1830D4
:10247000C5F8B84EC5F8B43E2D4BC5F8C04EC5F8EA
:10248000BC3E2C4BC5F8C43E06F0CEFC04F57B5098
:10249000343006F0C9FC04F57C50103006F0C4FC62
:1024A000254B06F1AC00A5F8287FC5F8243F14366B
:1024B00006F0BAFC04F580434FF0FF3230461F4966
:1024C000C3F8DC201E4B1E603EF0C4FC2046A5F87D
:1024D000D07EA5F8EC7E04B0BDE8F081D8CE0B0824
:1024E0003CCB0B08E8CA0B08408B0C08D86B0030BB
:1024F000F4910B089D1E02084CCF0B0890CB0B08E3
:1025000094CF0B0880CF0B08A8CF0B08A4CB0B08E7
:10251000B8CB0B0800C50B08C8670030C667003091
:102520008467003018CB0B0850CB0B08611E0208E3
:10253000651E0208691E02080000FFFF2C270C0818
:102540000067003038B5054B0A4601461C68236811
:1025500020461D68024BA847002038BDB425003036
:10256000B825003010B565F019FE064C064B186012
:102570002046FFF79DFE2046044A0549BDE810406D
:102580008EF068BEB8250030B42500308C120130C2
:10259000A11E020838B52DED028B0D46F0EE608AC3
:1025A000B0EE408A144602F085FF90ED937AD0EDAC
:1025B000957A67EE877A90ED927A67EEA87AE7EEE1
:1025C000087AC5ED007AD0ED920AD0ED937A90EDBD
:1025D000957A67EEA07A67EEA80AE7EE480ABDECA6
:1025E000028BC4ED000A38BD30B52DED068B83B0EB
:1025F000F0EE409AB0EE60AA0D46044602F05AFF93
:10260000D0ED7F7AD0F80002B8EEE79A18F0CEFB52
:1026100007EE900AF8EEE78A79EEC9AA3AEE688AE0
:10262000FDEEEAAAB0EE480A18F0A2FBBDEEC00A21
:102630005DB110EE103ADFED1D0A002BCCBF38EE75
:10264000608A38EE208ABDEEC80AF8EEC00A01AAF8
:102650006946B8EEEA0A2046FFF79CFF144B009942
:1026600003F56462DFED137A116003F644620199A9
:1026700069EEA79A29EE279A1160A3F58D622AEEDA
:1026800027AAC2ED009AA3F2644268EEA78A82EDFF
:10269000009AA3F55D72A3F55C7382ED00AAC3ED09
:1026A000008A03B0BDEC068B30BD00BF00A00C4714
:1026B000B85500300AD7233C38B52DED028B0D46B6
:1026C000B0EE408AF0EE608A144602F0F3FED0EDE0
:1026D000937A9FED147AF0EEE77AF4EEC77AF1EE92
:1026E00010FA1DD4D0ED957A90ED927A67EEE87AE3
:1026F000E8EE077AC5ED007A90ED937AD0ED957A01
:1027000090ED926A0120C7EE876AC6EE077A67EEFF
:10271000A80AE6EE880AC4ED000ABDEC028B38BDBB
:102720000020FAE70000003430B55D4C05465D48F6
:102730002DED068BB4F9E43A85B0DFED5B8AF6EE59
:10274000009A5B4208EE103A45F06EFDB4F9E43AA7
:10275000B8EEC88A90ED00AA524828EE288A98EE72
:1027600029AA08EE103A45F05FFDB4F9E83AB8EE50
:10277000C88A90ED009A4D4828EE288A98EE299A4A
:1027800008EE103A45F050FDB4F9EA3AB8EEC88ABE
:10279000D0ED009A0AEE903A444845F045FDF0EE3F
:1027A0004A0AF8EEEAAA6A46D8EE289A90ED008A1C
:1027B00002A928469AEEA88A8DED00AA8DED019A0D
:1027C000B0EE690ACDED029A8DED038AFFF774FF32
:1027D000F0EE490A01AAB0EE480A03A92846FFF71D
:1027E0006BFF02F067FED0F8000218F0DFFA04F584
:1027F000F15304F6DC2408EE100A93ED050AD4ED3B
:10280000007A30EE270A20EE280A18F0B1FAB8EE66
:10281000C88A30EE480A18F0ABFAB5EEC00ADFED10
:10282000247A9DED007AF1EE10FAABBF70EE676A84
:10283000F0EE406AF0EE407A70EE277AB4EEE67A77
:10284000F1EE10FA2ADD9DED016AB4EEE76AF1EED1
:1028500010FA23D5B5EEC00AF1EE10FA08DD77EED6
:10286000665A37EEC65AF4EEC55AF1EE10FA13D492
:10287000B5EEC00AF1EE10FA10D537EE667A77EEB3
:10288000C67AB4EEE77AF1EE10FACCBF0120002050
:1028900005B0BDEC068B30BD0120F9E70020F7E75D
:1028A000B8450030445B00300000C842505B003047
:1028B00000A00C4770B5364C054604F63462A4F20D
:1028C0002453A4F580562DED028BD3ED007A84B00D
:1028D00092ED000ADFED2F8A30EE270A20EE280A5B
:1028E00018F046FAB6F9EA3A04F63C62B0EE408ACD
:1028F00001EE103AB6F9E83A92ED000A0C2000EE2B
:10290000903AA4F5A463B8EEC11AD3ED007AF8EEBC
:10291000E00A30EE270A18F085FA20EE280A284649
:102920008DED010AFFF700FFF0EE480A01469DED2C
:10293000010A2846FFF758FEF0EE480A03AA02A94A
:102940009DED010A2846FFF725FEB6F9E63A002B71
:102950000FDD07EE903A04F63862F8EEE77A92ED72
:10296000007AB4EEE77AF1EE10FA02DA94F8F83D64
:102970004BB99DED020A084800F014FB9DED030AD7
:10298000054800F0F3FB04B0BDEC028B70BD00BF46
:10299000B85500300000C842B825003038B54C4C5E
:1029A000054694F8543E13F0010046D1A4F5805238
:1029B0009FED487A04F63461F7EE006AB2F9B82A5E
:1029C00013F0100F91ED000A07EE902AC3F30012E6
:1029D000F8EEE77A67EE877ABFEE007A06FE877A2E
:1029E000A7EE270ADFED3C7AB5EEC00A81ED000ABA
:1029F000F1EE10FA0AD51AB160F3041384F8543ECC
:102A0000B4EEE70AF1EE10FA06DC0BE0B4EEE70AEA
:102A1000F1EE10FA06DD2AB994F8543E43F01003A3
:102A200084F8543E2C209FED2C1ADFED2C0A18F070
:102A3000F9F904F6346383ED000A94F8543E9A07DA
:102A4000C3F3400032D426499FED227AB1F9BA2A65
:102A500007EE902AB1F9E82AB1F9EA1AF8EEE77A16
:102A600000EE902A01EE101A04F63C621907F8EE07
:102A7000E00A67EE877A92ED007AB8EEC11A1AD5AD
:102A800077EE677AF4EEE07AC2ED007AF1EE10FAB2
:102A900003D560F3C30384F8543E04F63C643C2041
:102AA00094ED000A18F0BEF984ED000A2846BDE84E
:102AB0003840FFF7FFBE77EE877AF4EEC17AC2EDB9
:102AC000007AF1EE10FAE8DD43F00803E3E700BF17
:102AD000B85500300AD7A33C0000B4430000000002
:102AE000B84500300A20704701207047094B024664
:102AF00093F8F81D09B1FFF7DDBE93F8591E29B907
:102B0000A3F5805393F8F03ADB0702D51046FFF7A0
:102B100045BF7047B855003004207047012070470A
:102B200030B504462DED028B8BB09FED298A66F0FF
:102B300039F8054607AB06AA05A9201D19F066FF5E
:102B4000244A41F288311368EB1A8B4216D915607A
:102B50004DF042F99DED067A06211F4A27EE087ACC
:102B6000B7EEC77A8DED027B9DED077A27EE087AE6
:102B7000B7EEC77A8DED007B46F03EF8DDED067AC4
:102B80002046DDED070A00219FED140A60EE880A59
:102B900027EE888A60EE800A28EE000AFFF724FDFF
:102BA00009AA08A9DDED070A9DED060A2046FFF7F0
:102BB000F1FC9DED080A0A4800F0F4F99DED090AC0
:102BC000074800F0D3FA0BB0BDEC028B30BD00BF5C
:102BD000E02E65429866003058CF0B080000C842CE
:102BE000B82500300020704701207047024B014695
:102BF0001868026812681047E06B003008B50020C2
:102C0000FFF7F4FFC188472050F00CF947204FF040
:102C1000A5FF0120FFF7EAFFC188482050F002F924
:102C20004820BDE808404FF099BF000002207047DF
:102C300001207047FFF7B2BE08B50B461146013BB5
:102C4000DBB2012B11D85BB9472050F0EBF84720DD
:102C50004FF084FF50F0BCF94FF052FE012008BD48
:102C6000482050F0DFF84820F2E70020F7E70000A6
:102C700008B54EF02BFEBDE808404EF007BD000041
:102C800000F5A8500021103002F09ABB00F2246039
:102C900007F090B810B5044607F07CF990F925309C
:102CA0008BB190F8443373B194F94C365BB1064B59
:102CB0001B68DB6A93F89C302BB904F22460BDE8F2
:102CC000104006F083BE10BDB425003070B5044638
:102CD00000F590700FF0E0FF1D4994F8143404EBF8
:102CE0000312D2F8C4010A68824210D0B02294F8CC
:102CF000585402FB034292F8F12145B9022A06D941
:102D0000144E08603278012A02D9013A327070BD3F
:102D1000FDD104F54055D5F8B82D2AB9D5F8BC2D0C
:102D200012B905233370F2E7B02205F55B6502FBAB
:102D3000034303F5FE730FCB85E80F0004F57651CE
:102D4000236800222046DB6C303198470023E9E7F6
:102D50009C6600300C2200307047000037B50446F6
:102D600050F00AFA4FF07AFF472104F50055002091
:102D700050F0A6F84821012050F0A2F8B5F8E41A66
:102D8000472001EB810101EB8101490089B24FF03D
:102D9000CFFEB5F9E83AB5F9EA1A48200E4DC91A3E
:102DA00001EB810101EB8101490089B24FF0C0FEC6
:102DB00050F00EF94FF0A4FD04F5565001A901950D
:102DC0000C3045F08FFA04F5565001A901951830E2
:102DD00045F088FA03B030BDCDCCCC3D00F50053B2
:102DE00070B50446642548202DED028BB3F8E82A1F
:102DF00084B0B3F8EA3A12FB05F613FB05F54FF081
:102E000087FE04F52B5004F57953B0EE408A00217B
:102E10003830DFED240A93ED000A01905CF002FFE8
:102E200007EE906A38EE000A0198F8EEE77AB4EE01
:102E3000E70AF1EE10FA27D98DED020A07EE905A53
:102E40009DED027AF8EEE77AF4EEC77AF1EE10FA29
:102E500003D8CDED027A5CF0A5FD48209DED020A75
:102E60004FF042FE04F5565004F54054183094F8E3
:102E7000A53583B10C4B03AA02A9039345F036FA9A
:102E800004B0BDEC028B70BD0190CDED027A5CF018
:102E900089FD0198D2E702A945F0C8F9012384F819
:102EA000A535EDE70AD7A33C0AD7A33C00F5795333
:102EB00000F5005093ED007A00F52D6200F6D8235E
:102EC000D2ED007AF0EEC76A93ED006A67EE867A7B
:102ED000F4EEE76AF1EE10FA04D59FED180A4820E7
:102EE0004FF002BEB5EEC07ADFED157A20EE270A6C
:102EF000F1EE10FA10DDB0F8E83A642213FB02F3A9
:102F000007EE903AF8EEE77AF4EEC07AF1EE10FAB6
:102F100002D59FED0C0AE2E7B0F8EA3A642213FB0F
:102F200002F307EE903AF8EEE77AF4EEC07AF1EEAB
:102F300010FA02DD9FED040AD1E77047000000009F
:102F40000000C84200A00CC600A00C4610B5044604
:102F500000F5795300F52B50002104F50054DFED06
:102F6000100A93ED000A38305CF05CFEB4F9EA0A0E
:102F7000B4F9E83A3221C21A1B1A80204A434B4363
:102F800001EE102A00EE903AB8EEC11AF8EEE00A0F
:102F900017F048FF4820BDE810404FF0A5BD00BF26
:102FA0000AD7A33C00F5005393F9C83A012B03D08C
:102FB000022B03D0FFF712BFFFF778BFFFF7C6BFA2
:102FC00000F500530021DFED350AF0B500F52F566E
:102FD00000F5405704462C362DED028BB3F8E45A29
:102FE000322383B0304615FB03F507F6446393EDB7
:102FF000000A5CF017FE9FED2A1ADFED2A0ABF20B7
:1030000017F010FFB0EE408A47204FF081FDC0203E
:1030100030EE080A9FED221ADFED220A17F002FFB8
:103020006B4207EE903AF8EEE77AB4EEE70AF1EE7B
:1030300010FA26D98DED000A07EE905A9DED007A20
:10304000F8EEE77AF4EEC77AF1EE10FA04D83046DB
:10305000CDED007A5CF0A6FC47209DED000A4FF014
:1030600043FD04F5565097F8A4350C307BB10E4B58
:1030700001AA6946019345F039F903B0BDEC028B12
:10308000F0BD3046CDED007A5CF08CFCD4E76946AB
:1030900045F0CCF8012387F8A435EEE70AD7A33C26
:1030A00000A08C4600A08CC60AD7A33C00F579533B
:1030B00000F500509FED127AD3ED017A00F6CC2393
:1030C00000F6D42067EE877A93ED007A90ED006ADF
:1030D000F0EEE76A27EE067AF4EEC76AF1EE10FA30
:1030E00004D59FED080A47204FF0FEBCF5EEC07AEC
:1030F000F1EE10FACCBF9FED040A9FED040AF2E74F
:103100000AD7233C0000000000A08C4600A08CC61B
:1031100010B5044600F5795300F52F50002104F551
:103120000054DFED110A93ED010A2C305CF07AFDBA
:10313000B4F9E43A4FF6CE713222F120B1EE400AF2
:1031400013FB02F213FB01F301EE102A00EE903A9A
:10315000B8EEC11AF8EEE00A17F064FE4720BDE8A9
:1031600010404FF0C1BC00BF0AD7A33C00F500538C
:1031700093F9C93A012B03D0022B03D0FFF720BFEC
:10318000FFF794BFFFF7C4BFFEF7C2BD00F50050C4
:1031900070B590F9F10A88B00C46D8B105210E48F7
:1031A00050F0A6F8092106460B4850F0A1F801217D
:1031B000039004AD084850F09BF800210346039AA1
:1031C00000912846314605F04FFE95E80F0084E84F
:1031D0000F00012008B070BDA066003037B5002296
:1031E0000C4605460F48114650F09AF862680121D6
:1031F0000C4850F0ADF8A26805210A4850F0A8F834
:10320000E2680921074850F0A3F805F52B50012486
:103210000DF1070131308DF807403EF065FC204686
:1032200003B030BDA066003037B503680446019195
:10323000DD6C0FF06FFDB02390F8F412019A03FBE0
:10324000010120462B46DC3103B0BDE83040184771
:103250007FB5044668460D4605F0E6FD04F5A85620
:1032600069461036304601F02FFF48B929462046FE
:10327000FFF7B4FF064650B90026304604B070BDD3
:103280002946304601F0CAFD0028EFD1F4E704F5E5
:10329000765495E80F00303484E80F00EDE7000025
:1032A000084B01211B6810B50446D86A03681B68E7
:1032B000984704F5955001211030BDE8104041F0C9
:1032C000F3BA00BFB4250030084B00211B6810B5CD
:1032D0000446D86A03681B68984704F59550002196
:1032E0001030BDE8104041F0DFBA00BFB425003017
:1032F00010B5044665F056FC002104F50054C4F8EE
:10330000E00C47204FF0ACFD002148204FF0A8FD15
:103310004FF05EFEBDE810404FF0F2BA70B50446C3
:103320001646084604F5005304F5405583F83C2A38
:10333000D5F8C03D8B422AD0C5F8C01D0B685B682C
:10334000984728B32046FFF7ABFFD5F8C00D05F628
:10335000346503681B6898473246C1B204F595503E
:10336000103041F07DFC04F5565004F580540021E6
:1033700028304DF0DBFB04F5E2639FED077AD3EDD7
:10338000007AF8EEE77A67EE877AC5ED007A70BDCD
:103390002046FFF799FFD8E70AD7233CF7B5044644
:1033A00000F5A6503AF04AFE012204F56050634B46
:1033B00004F5565604F5A06718309A71DA7104F0D6
:1033C000E7FF08232836384604F5A855C4F8143515
:1033D00004F04EFE304649F0E9FE30464DF002FF63
:1033E000103506F0D7FD2023436306F0D3FD07F028
:1033F0003FFF022304F59070C4F8A4310EF07CF86E
:10340000284600F0CBFE04F58053002204F5176037
:1034100083F81928B4F9A4301BB9B4F8A230A4F881
:10342000A430B4F8A41017F019F8284600F0B0FF43
:103430003846012104F5005504F0F4FB404B04F537
:10344000955004F5405700933E4B1030019302AB6A
:1034500013E9060041F01CFA4EF038FA99222921AE
:103460004FF08EF94EF032FA4EF0D8F92046FFF7C1
:1034700075FC05F6BC23DFED347A93ED007AF0EEAF
:10348000C76AF4EEE76AF1EE10FA4FD804F52B5351
:10349000DFED2E6AD3ED007AB0EEE76AB4EEE66AAD
:1034A000F1EE10FA42D8DFED2A6A27EE267A67EEAF
:1034B000A67ABDEEC77AFDEEE77A17EE103AC7F8A6
:1034C000B83D17EE903AC7F8BC3DD7F8B83D43B9C0
:1034D000D7F8BC3D2BB904F5765120463031FFF7C3
:1034E00055FE1C4B4FF47A711B68986A03685B6841
:1034F000984795F9EE1A2046FEF79EFE014610B950
:1035000004F577510C3105F6C4251F222046FFF73C
:1035100005FFD5ED007AF5EEC07AF1EE10FA0BDD7D
:10352000204603B0BDE8F040FFF7E2BE0A4A05219D
:10353000304645F061FBC8E703B0F0BD2D670030B1
:10354000B8250030893102080000B442000034433D
:103550008096184BB4250030B4CF0B0808B50A2963
:1035600022D8DFE801F00D1911151D21212121219B
:10357000060000F577510431FFF7D0FE012008BDA9
:1035800000F577510C31F7E700F577512C31F3E76F
:1035900000F577513031EFE700F577513431EBE743
:1035A00000F577511031E7E70020E8E700F5955086
:1035B000103041F0B1BF000000207047002070477C
:1035C000032101484FF0F8BDA066003070B50546F4
:1035D00005F540542DED028B65F0DCFAD4F81C3E65
:1035E000DFED247AC31A08EE103AB8EE488A28EEC6
:1035F000278AF1EE047AB4EEE78AF1EE10FA37D5B5
:1036000004F6FC5304F60C660FCB86E80F0004F6B4
:10361000286305F5785093ED001A04F624630C3006
:1036200093ED000A28EE011A28EE000AB7EEC11A3F
:10363000B7EEC00A05F0FCFE04F62C63DFED0E7A4F
:1036400093ED007AD4F8103E27EE277A07EE903AF1
:10365000F8EEE77AE7EE087AFDEEE77A17EE903AB1
:10366000C4F8103E012384F8F83DBDEC028B70BD18
:103670000023F8E7BD3786350000C84230B585B075
:1036800004466D46284605F0CFFB04F5A8502946B0
:10369000103001F0D5FC50B104F54054002304F57E
:1036A0005B6484F8AA3095E80F0084E80F0005B049
:1036B00030BD0000F8B500F5405405462DED028BF5
:1036C00094F8F83D002B69D000F57753D4F8C02D5D
:1036D00000F5765600F578572C3330360C379A4281
:1036E00019D094F8543EDA0715D43946304605F01F
:1036F00055FDB6EE007B04F634639FED2C6BA0EE17
:10370000067BBDEEC77BDFED2B7AB8EEC77A27EEDE
:10371000277A83ED007A3046394605F015FEB7EE7C
:10372000C00B04F6386305F50055DFED236A04F697
:103730004C6683ED000A95F9CA3A012B05BFD4F80F
:10374000103ED4F8B42DD4F8303E9B1A07EE903AD0
:10375000F8EEE77A87EEA67A86ED007AD4F8C00D07
:1037600003681B689847022818D094F8543E9B07BA
:1037700014D404F638639FED118AD3ED000A95F94D
:10378000CA3A04F63C6563B904F6486494ED000A4D
:103790008EF03EFD20EE080A85ED000ABDEC028B9E
:1037A000F8BD96ED000AF3E7AFF3008000000000DB
:1037B0009461B6400AD7233C0000C842E02E65421F
:1037C00073B50446FFF702FF04F500552046FFF7E6
:1037D00055FF204605F6C426FFF76CFFD6ED007AAC
:1037E000F5EEC07AF1EE10FA09DC244B1E68F06A9F
:1037F0000368DB699847012816D102B070BD65F0F7
:10380000D1F9D5F8E03C96ED007AC01ADFED1C6ADC
:1038100007EE900A27EE267AF8EE677AF4EEC77A7A
:10382000F1EE10FAE1D5E8E7F36A93F89C10E9B9F4
:1038300095F9EF3A012B10D19FED120A47204FF076
:1038400053F99FED100A48204FF04EF94FF0C0FB9E
:1038500002B0BDE870404FF053B8472001914FF0DF
:10386000E1FA019948204FF0DDFAEFE704F5405402
:10387000D4F8C00D03689B689847E7E7B42500308B
:1038800000007A440000000037B54B68054613B9C4
:103890008A68002A51D005F540540A20DFED287AC5
:1038A000C4F8043E8B68C4F8083ECA6892FBF0F284
:1038B000C4F8002E0B6993FBF0F3C4F8303EB1F965
:1038C0001630B1F9142007EE103AB1F91830B8EEFD
:1038D000C77A87EE276A07EE103A04F62463B8EE3B
:1038E000C77AC7EE276A07EE102AB8EEC77AC7EE86
:1038F000275AC3ED005A04F6286383ED006A04F6E4
:103900002C63C3ED006A65F045F9C4F81C0E65F040
:1039100049F90221C4F8200E2846FFF747FE60B19E
:1039200005F57853284624330093D4F8003ED4F8A4
:10393000082ED4F8041EFEF7B3F903B030BD00BF63
:103940000000C84210B50446DFED247A00F5A060FF
:10395000242294F811352DED028B91ED018A02FBA2
:10396000030328EE278A93ED090AF0EE480A03F0D4
:1039700035FEB4EE400AF0EE400AF1EE10FA24D61D
:10398000F0EEC07A9FED167AF4EE477AF1EE10FA77
:103990001BDC04F5405303F5656103F64862D1ED85
:1039A000007A77EE807AC2ED007A93F8540E4007E1
:1039B0000BD5F1EE407AC1ED007A0021116093F849
:1039C000542E6FF3820283F8542EB0EE480A20463C
:1039D000BDEC028BBDE81040FEF73CB90000C842C8
:1039E000FFFF7F7FB1F9002000F5405007EE902ADD
:1039F00000F63463F8EEE77A10B5C3ED007A00F60E
:103A00003C63B1F9022047F6FF7407EE902A0022CA
:103A1000F8EEE77AC3ED007A00F638631A60B1F980
:103A2000002090F8543E121B18BF012262F30003DD
:103A300080F8543EB1F9023090F8542E1B1B18BF89
:103A4000012363F3410280F8542E10BD10B500F538
:103A50004054D4F8200E50B165F0A4F8D4F8203EBC
:103A6000C01A41F2873398428CBF00200120014BDD
:103A7000187110BD2D67003000F5405370B500F58A
:103A80000054164603F6346203F63C63DA200D4612
:103A90002DED028BD2ED008AB7EE008AB4F9EA2A46
:103AA000D3ED007A01EE102AB4F9E82A00EE902A4C
:103AB00004F52E62B8EEC11A92ED000AF8EEE00AA3
:103AC00030EE270A17F0AEF9B4F9E82AB4F9EA3A69
:103AD00007EE902A9B1AF8EEE77A30EE670A07EEB7
:103AE000903A04F6DC23F8EEE77A30EE000A80EE36
:103AF000277A37EE487A86ED007A93ED000A38EEA1
:103B0000800A17F0F5F8B4F9E43A30EE000A012023
:103B100007EE103AB8EEC77AC0EE077A77EEC87AA9
:103B2000BDEC028BC5ED007A70BD0000704700004F
:103B30000020704770470000002070470020704749
:103B400000207047002070479FED010A704700BFBA
:103B5000000000009FED010A704700BF0000000058
:103B600070470000002070477047000010B5044601
:103B7000143000F019F804F12C0000F015F804F1ED
:103B8000740065F01BF804F1F80065F017F84FF0C9
:103B9000FF332046C4F8583110BD0000014B1868AF
:103BA000704700BFA466003070470000F0B52DEDEF
:103BB000048B91B004466D46284605F035F994F81B
:103BC000BC33002B72D004F57A73D4EDEC8A94EDFB
:103BD000ED8A94EDEE9A0FCB85E80F0094F8F83358
:103BE000002B63D094F8D033002B5FD02D2200211E
:103BF00004A8D4F8C073D4F8C463D4F8C853D4F874
:103C0000CC4391F0EDF8A3238DF8103095238DF877
:103C1000113046238DF8123064F0CCFF9FED250A59
:103C20009FED257A68EE807ACDF81710CDF8130055
:103C300067EE877AFDEEE77A17EE903A68EE007A43
:103C400029EE000AADF81B3067EE877A20EE070AEE
:103C5000FDEEE77A17EE903AADF81D3017F072F8E6
:103C6000DDED017ABCEEC00A9FED147AF8EEE77A3A
:103C7000CDF82D7010EE103ACDF83160CDF83550FA
:103C800067EE877AADF81F30CDF8394017EE903ADD
:103C9000CDF82130029BCDF82530039BCDF829309B
:103CA00041F016FE2D2204A940F01AFE11B0BDEC21
:103CB000048BF0BDE02E65420000C8420AD7233CC9
:103CC00030B52DED028B8BB0044624220D4601A8A1
:103CD000002191F085F8A3239FED228A8DF804300E
:103CE00095238DF8053048238DF8063064F062FF87
:103CF000D4ED817A2B6867EE887A95ED020ACDF8CB
:103D00000F30CDF80B1017EE903AD4ED827ACDF843
:103D1000070067EE887ACDF813306B68CDF817305E
:103D200017EE903ACDF81B3016F0E2FF10EE103A85
:103D300094ED830A20EE080ACDF81F3016F0D8FF64
:103D400010EE103ACDF8233094F80C338DF827306C
:103D500041F0BEFD242201A940F0C2FD0BB0BDEC34
:103D6000028B30BDE02E654230B587B014460D465B
:103D700018220021684691F033F8A3238DF8003013
:103D800095238DF8013049238DF8023064F012FF3D
:103D9000A368CDF807100393E368CDF803000493FC
:103DA00063688DF80B50059341F092FD1822694627
:103DB00040F096FD07B030BD10B58EB0044602A8A5
:103DC00005F032F802A9204601F03AF9002845D062
:103DD00001F070FB694600F0CBFF1F22002106A80E
:103DE00090F0FEFFA3238DF8183095238DF819303D
:103DF0004A238DF81A3064F0DDFEDDED037A9FED85
:103E00001B7AF8EEE77A049BCDF81B002046CDF82C
:103E1000233067EE877A059BCDF81F1001A9CDF8F6
:103E2000273017EE903ADDED007AF1EE677ACDF8A3
:103E30002B3017EE903ACDF82F3000F00FFC78B110
:103E4000DDED017AF1EE677A17EE903ACDF8333076
:103E500041F03EFD1F2206A940F042FD0EB010BD0C
:103E600041F036FDDFED027AEEE700BF0AD7233CD2
:103E70005241C07F0023036043608360C3600361DD
:103E800043618361C361036270470000B02290F810
:103E9000F43202FB030390F8382393F8D13012B1C7
:103EA000012B28BF01231846704700002DE9F04F71
:103EB00004464FF0000A8BB00D461DF0B1FF04F52B
:103EC000067084F814A24FF07E5763F009FE4FF499
:103ED0007A7384F8685204F51B70A4F862320025E6
:103EE000C4F8487204F52B79C4F84C7204F53476A2
:103EF000C4F8507204F5487B04F096FF032348464B
:103F0000C4F89452C4F8803204F26448C4F8985259
:103F1000C4F89C52C4F8A052C4F8A452C4F8A852E1
:103F2000FFF7A8FF3046FFF7A5FF5846C4F8145323
:103F3000C4F81853C4F81C53FFF79CFFC4F844534B
:103F4000C4F8485304F57570C4F84C53C4F8505382
:103F5000C4F85453C4F85853C4F85C53C4F86053BD
:103F6000C4F86453C4F86853C4F86C53C4F870536D
:103F7000C4F88C53C4F89053C4F89453C4F8A853AD
:103F8000C4F8A453C4F8A053C4F8B053C4F8B4534D
:103F9000C4F8B853C4F8CC53C4F8C853C4F8C453D5
:103FA000C4F89C73C4F8C07304F03EFF04F57A7043
:103FB00004F03AFF04F58063C4F8FC5304F5836011
:103FC0001D6004F581631D605D609D6004F02CFF41
:103FD00004F22C43404604F23C421D605D609D604B
:103FE0006B4BC4F83C3404F50D73C4F8403404F54D
:103FF0000E73C4F8443404F50F73C4F8483404F560
:104000001073C4F84C3404F24523C4F8503404F55A
:104010001173C4F8543404F58B631D605D609D60BA
:10402000FFF728FF04F59160FFF724FF04F597637D
:1040300004F2BC501D605D609D6004F2C4431D60CD
:104040005D609D6004F59A631D605D609D6004F293
:10405000DC431D605D609D6004F2EC431D605D60AB
:104060009D6004F2FC431D605D609D6004F5A163EA
:104070001D605D609D6004F22C53C2F8E070C2F8D0
:10408000E4701D605D609D6004F5A7631D605D6068
:104090009D6004F244531D605D609D6004F5AC6357
:1040A0001F605D6004F284531D605D609D6004F5D7
:1040B000B2631D605D609D6004F5B5631D605D6069
:1040C0009D6004F0B1FE04F2CC53242251461D60E1
:1040D00040465D6004F2D4531D605D6004F2DC5321
:1040E0001D605D6090F07CFE04F2FC50C8F820700A
:1040F000C8F81070C8F80070FFF7BCFE04F5C46380
:1041000004F5CA601D605D609D6004F22C631D6053
:104110005D609D6004F5C7631D605D609D6004F295
:1041200044631D605D609D60354604F07DFE194B63
:10413000204619491C603CF08DFE51462422584609
:104140006E4690F04DFE04F5257204F52873C4F810
:104150004073C4F83073C4F8207307CA83E80700BB
:10416000484694EDAA1AD4EDA90A94EDA80A17F0CE
:1041700071FA4946684617F095F90FCE0FC50FCE74
:104180000FC5204633682B600BB0BDE8F08F00BF31
:10419000F4D10B08A8660030A4D00B0810B5044673
:1041A00088B001F011FA94F93232012B02D127487C
:1041B00004F01EFE022B0AD1032304A904F111000E
:1041C00084F8323201238DF810303DF04FFC94F822
:1041D000323204F23C4084F8903201F0ABF994F9A9
:1041E0003132642B30D1652304A904F231208DF8DB
:1041F00010303DF079FC04A920463BF0D3FF18B302
:1042000004238DF818300023CDE9013303930F23E5
:104210000593694604A83CF043F9059B28B108AA18
:10422000009902EB830242F8581C0133112B0593CD
:10423000EFD962F051F99DED031ADDED020A652117
:104240009DED010A62F006F908B010BD04D00B081C
:1042500070B500F5257600F528758CB0044631461A
:10426000284619F03FFBE0B996E8070085E807000B
:1042700004F52B7194EDAA1AD4EDA90A02AD94EDC0
:10428000A80A0846019117F0E5F9019902A817F06C
:1042900009F904F534740FCD0FC40FCD0FC42B688A
:1042A00023600CB070BD000013B5044600F5067124
:1042B00040F2411201A812F099FE04F23C4001F0D4
:1042C0001FFB20461DF092FF01A812F0B1FE02B0C4
:1042D00010BD0000F8B50B6801F10C0607460C464E
:1042E000C0F8043200F548754B68C0F808328B6896
:1042F000C0F80C320FCE0FC50FCE0FC504F130023F
:1043000033682B6007F5457307CA83E8070004F19B
:104310003C0207F5517307CA83E8070004F148021D
:1043200007F55473543407CA83E8070007F5577339
:1043300094E8070083E80700384601F059FA384648
:10434000BDE8F84001F03CBA13B5044600F23C4029
:10435000019002F053FF04F5BE610198009102F054
:1043600059FA0099204602B0BDE81040FFF7B2BFED
:104370004A78064BC2F340121A754A78C2F380128B
:104380005A750A78C2F300129A7570472D6700308B
:1043900013B5044600F5067140F2F52201A812F0AB
:1043A00025FE002104F23C4001F01EFD94F860322D
:1043B00023B120461EF006F984F8600201A812F02D
:1043C00037FE02B010BD000038B590F80C3305463A
:1043D0000C462BB1032B0BD095F86832DB070CD4BD
:1043E00005F5CA630FCB84E80F0095F8600603E07B
:1043F0001DF052FF0028EFD038BD0020FCE7000080
:1044000000F23C4090ED380A7047000000F23C405A
:1044100090ED390A7047000010B490F80C230C4658
:104420002AB1032A0AD000205DF8044B704700F53A
:10443000B56007C884E807000120F5E75DF8044B84
:104440001DF012BF90F88403431E58425841704734
:1044500038B590F80C330D468BB900F23C4001F0B2
:10446000C1FA044610B90024204638BD01F00EFA06
:10447000D5ED007A27EE800A85ED000AF4E7D0ED4D
:10448000E07AC1ED007A90F87C43002CEBD090EDFF
:10449000DE7ADFED076AB4EEE67AF7EE006AF1EE57
:1044A00010FA27FE267A67EE877AC1ED007ADBE7FD
:1044B0000000003490F80C33032B01D11DF054BEE2
:1044C0000020704790F80C23032A01D11DF0B0BFE3
:1044D00000F23C4001F0EABE30B590F80C3385B0F4
:1044E00004460D468BB1032B18D004F5257019F046
:1044F00033FA284601A98DED010ACDED020A8DEDB2
:10450000031A18F023FB012006E000F23C4001F002
:1045100013FA0028E9D1002005B030BD90F86032D0
:10452000002BF8D01DF06CFFDFE700007FB590F89E
:104530000C2332B1032A4FF0000309D003930493F4
:104540000CE000F23C4007B05DF804EB01F0D0BA9B
:1045500003A90393049305931DF0FCFD9DED030A4D
:10456000DDED040A07B05DF804FB000007B590F824
:104570000C3333B100F57F7003B05DF804EB19F034
:10458000DDB800F23C4001F0B3FA68468DED000A58
:10459000CDED010A19F0D2F803B05DF804FB00007C
:1045A0001DF0D8BE90F80C03003818BF01207047EA
:1045B00008B590F80C23032A05D000F23C40BDE872
:1045C000084001F07DBA1DF0C5FD012008BD0000C6
:1045D00010B590F80C230C461AB1032A07D000201E
:1045E00010BD00F23C40BDE8104001F00DBA1DF0D6
:1045F000C7FD012084ED000AF2E7000090F80C33BB
:10460000032B01D11DF0DCBE0020704730B590F8BF
:104610000C3385B005460C4623B1032B09D000208E
:1046200005B030BD00F23C4005B0BDE8304002F0BE
:1046300021B9002302A9029303931DF073FD002802
:10464000EDD001A928461DF079FD0028E7D0029B96
:104650002360039B6360019BA360E1E790F80C2358
:104660001AB1032A05D00020704700F23C4002F046
:1046700027B91DF063BD000090F932323BB990F8C4
:10468000683213F0010F14BF03200020704703208D
:1046900070470000F7B50446FFF7EEFF0546002817
:1046A00062D0032839D194F860326BB394F8683241
:1046B000D8072BD501A920461EF0BEF8BDF804305E
:1046C000002B18BF002594F8146206F0FD06012E99
:1046D0004AD10023032D019307D101A920461EF0E2
:1046E000B7F820461DF0B0FE064604F23C4002F04A
:1046F00073F908B994F809039DF80430D90703D574
:104700005A0701D59F0632D400252DE020461DF022
:10471000E3FC002808BF0025D5E70025D3E713F008
:10472000020F2EE094F9443223B99DF80430DB09DE
:104730002FD0E9E7002EF8D00EF0ECFAFFF7A6FB39
:10474000022807D99DF805309806DDD59DF804307C
:10475000D906D9D5FB6A93F89C30002BE5D118E037
:10476000DA0601D41B0718D5284603B0F0BD00288F
:10477000FAD094F80923B4F96436002ACFD013F0A4
:10478000010FF1D1154B1F68FB6A93F89C30002B89
:10479000C8D19DF804309C07E2D405F0FBFB05F07E
:1047A000F7FA0028B0D10EF0B5FAFFF76FFB022838
:1047B000AAD90EF0AFFAB02290F8F432F0EE007AF7
:1047C00002FB030090ED3B7AB4EEE77AF1EE10FACB
:1047D0009AD59DF80530DB09C6D195E7B4250030A0
:1047E0002DE9F04790F8603292B00446002B00F0BB
:1047F000938020461EF030F92046FFF74BFF032838
:104800007AD104F54878002720464FF00C0A41463B
:104810000097019702971DF0E9FD694620461DF0BB
:10482000DBFD009B2046C4F80432019BC4F808322B
:10483000029BC4F80C3200F0DBFF204600F0C0FF02
:1048400015F04AFD054620461DF05EFC002803AA2F
:104850004FF0FF31AEBFC6B295F8EB9495F8EC641B
:104860002046A8BFB1460397049705971DF096FC14
:1048700003A804F5577719F06FF80AFB09500AFBF3
:10488000065504F5517184EDD10A00F55C70C4ED54
:10489000D20A05F5007584EDD31A06AE19F06CF84E
:1048A0003A4684EDC50A4FF0FF31C4EDC60A2046F2
:1048B00084EDC71A1DF086FC95E8070086E807001E
:1048C0003946304619F0BEF804F52B72414609A866
:1048D00016F07AFD314609A816F0F8FC09A9204621
:1048E00084EDD40AC4EDD50A84EDD61A1DF0B0FFCC
:1048F00009A92046FFF73CFD94F86636002B3AD113
:1049000009A804F091FA09A920461DF0D1FC90B342
:10491000012384F866362EE0D0F864321BB964F0C7
:1049200041F9C4F86402154B1B68D86A03685B68D8
:10493000984788B164F036F9D4F86432C01AB4F8F4
:104940006232984204D920461DF03CFE84F8600291
:1049500094F860327BB14CE764F024F9D4F8643207
:10496000C01A41F287339842E4D840F0B1FF40F0DA
:10497000EFFD0028DED112B0BDE8F087B42500308D
:1049800090F80C3323B1032B4FF0000007D0704791
:1049900090F93222032A04D10A700120704708706E
:1049A000FBE718467047000073B50D460DF107018F
:1049B0000446FFF7E5FF064628B19DF807302BB106
:1049C000032B09D00026304602B070BD04F5CA633F
:1049D0000FCB85E80F00F6E7294620461DF05CFC6A
:1049E00094F86062EFE700007FB50E460DF1030119
:1049F0000446FFF7C5FF054618B90025284604B050
:104A000070BD9DF8033083B1032B16D004F52570DB
:104A100018F0A2FF01A930468DED010ACDED020A82
:104A20008DED031A18F092F8E8E7314604F23C40A5
:104A300000F082FF0028E9D1DFE794F86032002B14
:104A4000DBD0314620461DF0DBFCDFE737B50D46F5
:104A50000DF107010446FFF793FF28B19DF80730D9
:104A600023B1032B0FD0002003B030BD04F5BE638B
:104A70001B682B6004F2F45304F5BF641B686B6081
:104A80002368AB60F0E7204629461DF0A5FC94F8AA
:104A90006002E9E710B50446FFF7EEFD18B1032800
:104AA00007D0002010BD04F23C40BDE8104000F0EB
:104AB0006DBF94F86032002BF3D020461DF00CFB44
:104AC0000028EED094F8143203F0FD03012BE9D155
:104AD00094F80C03C31E58425841E3E710B504464E
:104AE000FFF7CAFD80B1032810D194F8600250B1DD
:104AF00064F058F8D4F86432C01A44F6206398423F
:104B000094BF0020012010BD0120FCE70020FAE73F
:104B100008B50246FFF7B0FD032804D110461DF08A
:104B200097FE012008BD0020FCE7000030B585B0ED
:104B300004460191FFF732F80199054610B90020AB
:104B400005B030BD0191FEF7F9FF01990028F6D0BC
:104B50002846FEF7F7FF0028F1D0B4F8643659076D
:104B6000EED494F80933002BEAD00B4A1268D26ACB
:104B700092F89C506DB103A92046FFF7C9FF30B1F0
:104B80009DF80E309A07DBD5C3F38000D8E728469E
:104B9000D6E71846D4E700BFB42500302DE9F04130
:104BA00090F80C338CB000270646032B0C461546B4
:104BB00000970197029719D11DF0A6FA6A46804620
:104BC0004FF0FF3130461DF0FDFAB8F1FF3FA7600E
:104BD000676027600DD115F07FFB2B46224690F8C9
:104BE000EC1414F093FA0CB0BDE8F0814FF0FF38EC
:104BF000EBE715F071FB2B4622465FFA88F114F0C3
:104C000085FA95ED000A684618F0E2FE03A92046F1
:104C10008DED051A8DED030ACDED040A18F012FF93
:104C200006F52B7206F5487103A816F0CDFB214658
:104C300003A816F04BFBDFED077A84ED021A84ED32
:104C4000000AC4ED010A95ED007AA7EE271A84ED5B
:104C5000021AC8E70AE81C4137B5054600F5067197
:104C600040F6033201A812F0C1F92846FFF704FD0F
:104C7000044640B103280AD0002401A812F0D8F954
:104C8000204603B030BD28461DF0CAFAF5E7284695
:104C90001DF0C6FA0446F0E708B50246FFF7ECFC43
:104CA00010B1032806D008BD02F23C40BDE8084020
:104CB00000F036BE1046BDE808401DF0D5BD00002E
:104CC0000B46114610B42BB1032B09D000205DF820
:104CD000044B704700F23C405DF8044B00F036BED8
:104CE0005DF8044B1DF0E4BA13B504460A46FFF71D
:104CF000C3FC014620460192FFF7E2FF70B9084B62
:104D0000019A1B68DB6A93F89C0038B194F80C1385
:104D1000204602B0BDE81040FFF7D2BF02B010BD80
:104D2000B425003037B504460D4640F2B25200F5C6
:104D3000067101A812F05AF9294620461DF0D6FA4C
:104D400094F80C330546032B10D148B104F5836168
:104D50002046FFF7C9FF84F82804204600F076FDBE
:104D600001A812F065F9284603B030BD0025F7E729
:104D700070B590F87C3286B004460D46DB070CD443
:104D800003F0A6F82422437C02FB0300D0ED0B7A4B
:104D9000F1EE677AC5ED007A3BE002A804F044F832
:104DA00001A92046FFF75AFCE8B90DF0B3FF94F9CA
:104DB00044320646022BE3D1FFF768F80228DFD918
:104DC000B02396F8F4029FED147A03FB0066D4F842
:104DD0007032D6F8E0209B1A07EE903AF8EEE77AA8
:104DE00067EE877AD6E702A92046FFF77DFF002805
:104DF000DBD0D4F87022039BDFED076A9B1A9DED90
:104E0000017A07EE903AF8EEE77AA7EEE67A85EDBA
:104E1000007A06B070BD00BF0AD7233CF0B587B05A
:104E20000C46064600F5067140F6863201A812F0DF
:104E3000DDF8A36853B9E36843B9636833B9002761
:104E400001A812F0F5F8384607B0F0BD204604F08E
:104E5000F9F80028F3D002AD94E80F0085E80F00C0
:104E60000021284604F0AAF807460028E7D096F863
:104E70007C32DB0704D440F02BFD192140F0BEFA50
:104E800006F51B7C95E80F008CE80F0096F87C3245
:104E9000304643F0010386F87C3200F0D7FC4AF03C
:104EA0009BFF46214BF042FE4AF096FF45214BF016
:104EB0003DFE054BA2681B68DB6A1A61E2685A6115
:104EC00062689A61BCE700BFB425003038B5144B66
:104ED00004461B68DD6A2B6828465B689847F0B17A
:104EE0002B690BB96A69D2B1C4F8743200226B69BC
:104EF00004F51B70C4F87832A96903F09BFF94F89D
:104F00007C3223F0030343F0030384F87C324AF03D
:104F100063FF044A0621BDE8384043F06DBE38BD4A
:104F2000B42500302CD00B0810B588B0044605938A
:104F3000FFF7A2FB0328059B4FF000000AD1069063
:104F4000079006A802900B9801900A9800902046BE
:104F50001DF060FA08B010BD38B50446FEF71EFE1D
:104F60000546D0B194F80C33032B03D095F8564185
:104F7000204638BD20461DF083F9FF280446F5D0B1
:104F800001462846FEF7DEFD0028EFD021462846E0
:104F9000FEF7D4FD0028E9D0EAE70446E8E7000080
:104FA00008B590F80C33032B05D015F095F990F95E
:104FB000EB04C0B208BD1DF0A7F8431CF9D1F4E71B
:104FC00008B590F80C3383B1032B03D1BDE808403A
:104FD0001DF092B83EF00CFE40F6ED424FF4801109
:104FE0003EF0BEFD4FF0FF3008BD1846FCE7000064
:104FF00090F80C33032B01D11DF07ABE70470000EE
:1050000090F80C33032B01D11CF0C0BF7047000097
:105010001DF04AB810B504461FF0ECFF2046FEF71D
:10502000C5FD2046BDE81040FEF7C6BE90F80C3323
:105030000BB1032B01D11DF0D9BE00207047000039
:1050400000F5757330B504460D460FCB85E80F00AB
:1050500094F8E40330BD00007FB5054668460E466F
:1050600003F0E2FE95F87C32DB0703D400242046EF
:1050700004B070BD69462846FFF7E2FF04460028E9
:10508000F4D0694605F51B7004F0C8F886ED000AF7
:10509000C6ED010AEBE70000D0F880330B6090F812
:1050A0007C037047D0F888330B6090F88503704715
:1050B00000F5677330B504460D460FCB85E80F0049
:1050C00094F8AC0330BD000000F5836330B50446AE
:1050D0000D460FCB85E80F0094F8280430BD000082
:1050E00000F22C42034610B50C4607CA84E80700BC
:1050F00093F8380410BD00002DE9F04305460E4634
:1051000017462DED028B8BB0FFF726FF0146804638
:105110002846FFF70BFD0446002846D0FEF73EFD6B
:105120004146FEF711FD86ED000A95F93032002B5D
:1051300038DD0DF0EFFDFEF7A9FE012832D90DF0A4
:10514000E9FDB02290F8F432B7EE008AD5EDDE7AB0
:10515000DFED598A02FB030095F93032F4EEE87A6C
:10516000D0ED3B0A07EE103A96ED000A40F2B63059
:10517000F1EE10FAB8EEC77A67FE887A20EE270AB9
:1051800037EE201A70EEC70A15F04CFED5EDDE7A28
:10519000F4EEE87AF1EE10FA67FE887A80EE277A6C
:1051A00086ED007A01233B7003E095F8083333B9AC
:1051B000387020460BB0BDEC028BBDE8F0834FF099
:1051C000000995F80C33CDF80490CDF80890CDF88F
:1051D0000C9043B1032B10D0CDF81090CDF8149063
:1051E000CDF818907CB902233246414605F23C4086
:1051F0003B7001F0B5FB0446DBE701A928461DF032
:1052000033F80446E8E795F80C33002BEBD004A9FB
:105210002846FFF765FF04460028E4D001A904A84A
:1052200018F0C0FB07A8CDED080A8DED091A8DED29
:10523000070A18F0C9FF04A8B0EE408A18F0C4FFAE
:1052400095F93032002B2EDD07EE903A4FF47F7047
:10525000F8EEE77A70EE670A37EE801AB0EE480A89
:10526000F5EEC00AF1EE10FA48BFDFED140AF4EED5
:10527000410AF1EE10FA30FE811A15F0D3FDB0EEBE
:10528000408AD5EDDE7A03239FED0B7AF4EEC77AE0
:10529000B7EE007AF1EE10FA67FE877A88EE277A89
:1052A00086ED007A7FE7B5EEC08AF1EE10FA48BFCE
:1052B0009FED028AE5E700BF000000340000000017
:1052C00010B50446FFF76CFE84F80D032046FFF787
:1052D00067FE84F80E032046FFF762FE84F80F0392
:1052E0002046FFF76DFE04F55A7184F8100320463E
:1052F000FFF792F884F8740300F0C8FA04F56172BD
:1053000084EDDE0A04F560712046FFF7F5FE04F532
:10531000627184F87C032046FFF79AF804F5637104
:1053200084F885032046FFF7C5F804F5677184F813
:1053300098032046FFF7D0F804F56C7184F8AC03AD
:105340002046FFF783FB04F5707184F8BC03204608
:10535000FFF74AFB04F5757184F8D0032046FFF788
:1053600033F804F57A7184F8E4032046FFF71CFB58
:1053700084F8F8032046FFF7D9F804F58063204647
:1053800084EDFF0AC3ED000AFFF7F0F804F20443CE
:1053900004F2144204F5816183ED000A2046FFF710
:1053A000FDFB04F583612046FFF79EFC04F22C41CF
:1053B00084F828042046FFF7FBF884F8380410BD71
:1053C00037B50D46044600F0FFF81DB914F084FF10
:1053D00013F06EFD4FF4BE7204F5067101A811F0D2
:1053E00005FE94F869322BB92046FFF76FFD0123C3
:1053F00084F86932224B1D68A86A03689B69984744
:105400002046FEF725FF2046FEF79EFF204600F0CF
:105410004FFA2046FFF7E4F9286B30B10368D4ED6A
:10542000D20ADB6894EDD10A9847D4F8100208B18B
:1054300064F026FB204600F07DF82046FFF72AF9AD
:1054400094F8903284F80C0383420ED084F89002D2
:1054500098B10C4D0C4B032808BF1D464AF0BCFC0C
:105460002B460A4A062143F0C7FB2046FFF728FFD8
:1054700001A811F0DDFD03B030BD054DEEE700BF22
:10548000B4250030A7A20B0823D00B0844D00B088A
:1054900028D00B08D0EDDE7AB7EE000A9FED047A33
:1054A000F4EEC77AF1EE10FA27FE800A704700BFCB
:1054B00000000034014B1868704700BFA866003038
:1054C0004FF0FF3070470000012070477047000028
:1054D00000207047002070477047000070470000B0
:1054E0000020704700207047002070470020704760
:1054F000002070470020704700207047012070474F
:105500000368D3F894301847002070470020704794
:10551000002070470020704700207047002070472F
:10552000002070470020704700207047002070471F
:10553000704700007047000008B514F0CDFE90F8E9
:10554000EC0408BD08B514F0C7FE90F8EB0408BDE4
:1055500030B59FED1B1A0C46DFED1A0A05462D20CB
:105560002DED028B87B091ED000A8DED011ACDED86
:10557000000A15F057FC9DED011AF0EE408ADDEDB2
:10558000000A2E2094ED010A15F04CFC9DED011A45
:10559000B0EE408ADDED000A2F2094ED020A15F0EE
:1055A00041FC03A905F52570CDED038A8DED048A34
:1055B0008DED050A3CF07CFB07B0BDEC028B30BDE5
:1055C000C2B8323EC2B832BE10B5044663F0EAFA41
:1055D000D4F8F4321BB1C21AB2F57A7F12D30A4A58
:1055E0001268D26A92F89C2002B15BB9C4F8F40246
:1055F00094F8314214F070FE80F8E24404F0CAFCE2
:1056000080F8294010BD00BFB42500302DE9F043DB
:105610002DED028B87B091ED007AD1ED037A0C4627
:105620008DED047AB0EEC77A15461E46DDF84C9033
:10563000B5EEC07ACDED057ADDE91087F1EE10FA0E
:1056400006DCF0EEE77AF5EEC07AF1EE10FA02DD54
:1056500004A818F0CDF8B7EE001A6B20FFEE000A90
:105660009DED050A15F0DEFBB7EE001AFFEE000A0D
:105670006C2089ED000AB7EE008A9DED040A15F052
:10568000D1FB04A888ED000A18F03CF8002852D09D
:105690000023C9F8003088ED008AD4ED067A67EE61
:1056A000A77AF4EEC87AF1EE10FA4ADB00233360F1
:1056B00085ED008AB7EE001A7C20DFED3E0A96EDFC
:1056C000000A15F0AFFBB7EE001A86ED000AFFEEF8
:1056D000000A7D2095ED000A15F0A4FB85ED000A77
:1056E000D4ED067A129BF1EE677ADFED336AC3EDF3
:1056F000007A96ED007AF0EEC77AF4EEE67AF1EEF3
:1057000010FA2BD503AB02AA01A9204616F002F825
:105710009DED018AB0EE480A8BF0A2FD85ED000AEE
:10572000B0EE480A8CF078FB87ED000A07B0BDECBC
:10573000028BBDE8F08304A817F0D0FF0028A7D1A2
:10574000ABE738EE670A15F09BFA86ED000A94ED98
:10575000087AC7EE007AC5ED007AABE794ED076AE8
:10576000C6EE077AC7ED007A96ED007AB0EEC77AFA
:10577000B4EEE67AF1EE10FAC4D495ED007ADFEDDE
:105780000F6AB0EEC76AB4EE666AF1EE10FAB9DCE1
:10579000B4EE477AF1EE10FAB4D6B0EEE77AB4EE92
:1057A000667AF1EE10FAADDCF4EE677AF1EE10FAFB
:1057B000BCD7A7E70000000000000034FFFF7F7F98
:1057C0001FB500F5177300F5127200F548710393C9
:1057D00000F51673029300F51573019300F5147329
:1057E000009300F51373FFF711FF05B05DF804FB9C
:1057F0009FED146A90ED817ADFED136A27EE067A49
:10580000D0ED837A67EE867A27EE267A67EEA67A5F
:10581000BDEEC77AFDEEE77A80ED7E7A90ED827A72
:1058200017EE903A27EE067A002B27EE267ABCBFB9
:1058300003F50C43A033BDEEC77AC0F8003280ED0B
:105840007F7A7047E02E65420000C8421FB50E4BBC
:1058500004461B68B3B1684603F0E6FA6946204681
:10586000FFF732FC20B16A4600212046FEF77CFAA1
:1058700094F87C32DB0705D504F51B720121204624
:10588000FEF772FA04B010BD8C69003008B502F062
:105890001FFBBDE8084001F0B5BE000010B504468E
:1058A00080F8F81263F07EF9C4F8FC0210BD000025
:1058B00010B590F8F832044653B163F073F9D4F898
:1058C000FC32C01AB0F57A7F84BF002384F8F83226
:1058D00094F8003353B163F065F9D4F80433C01A77
:1058E000B0F57A7F84BF002384F8003310BD000038
:1058F00000F5B6700B4607C883E807000120704723
:105900000023C0F89C30C0F89830C0F89430C0F83C
:10591000A830C0F8A430C0F8A030C0F8AC30704750
:1059200070470000024B0B604FF07C5313607047D0
:10593000000048427047000008B50B4600F12801FE
:10594000184616F093FE012008BD000000F5C07057
:1059500010B50C460FC884E80F00204603F054FA37
:1059600030B1FFF7A7FD00F51B700FC884E80F00EA
:10597000204603F049FA80F00100C0B210BD0000DB
:1059800010B5044603F068FD204610BD10B5D0F8F0
:10599000783104465BB163F005F9D4F87831C01A68
:1059A00041F28833984294BF0020012010BD0120AD
:1059B000FCE7000013B5009303680192D3F8903020
:1059C00098470446DDE9002128B90448044B0068E3
:1059D000C06A11F0E5FC204602B010BDB4250030CD
:1059E00064D10B0813B504460191FEF7D7F8019A6C
:1059F000236801461B6D08B190F85611204602B08D
:105A0000BDE810401847000030B5002385B00D46B2
:105A1000019301A9029303930368DB6D9847044641
:105A200020B1039B2B60204605B030BD02F050FA38
:105A3000417C01F01DFF04460028F4D002F048FA32
:105A400001F07CFEB1EE400A85ED000AEBE70000B4
:105A500090ED007ADFED0F7AB0EEC77AB4EEE77A18
:105A6000F1EE10FA14D590ED017AB0EEC77AB4EEEB
:105A7000E77AF1EE10FA0BD590ED027AB0EEC77A24
:105A8000B4EEE77AF1EE10FA4CBF01200020704727
:105A9000002070470000003410B5FEF77FF8044680
:105AA00058B190F85611FEF749F830B194F85611F4
:105AB0002046BDE81040FEF745B8002010BD0000AC
:105AC00038B50D460DF026F90446FEF7DFF9022839
:105AD00085BF94F8F402B023002003FB004081BF8F
:105AE00000F5827007C885E80700012038BD000076
:105AF0002DE9F043002504462DED028B8FB003689D
:105B000002A9DB6C039504950595069502959847C7
:105B1000064638B1FFF7BAFEDDED027A27EE800ABD
:105B20008DED020A0DF0F6F8FEF7B0F90746002EEB
:105B300050D0DDED027A0BA9D4ED6A6A204694EDCF
:105B40006B7A236827EE877A0B9567EEA67A0C9519
:105B50000D9509AD8DED097ACDED0A7A9B6C9847CC
:105B60000BA9284617F034FD012F8DED030ACDED6A
:105B7000040A40F2B3800DF0CDF8B02590F8F4326D
:105B8000DFED5A7A05FB030090ED3C8A28EE278A68
:105B9000B0EE480A8BF064FBF0EE408AB0EE480AA3
:105BA0008CF03AF98DED0C0ACDED0B8A0DF0B2F8C0
:105BB00090F8F43205FB030009AD90ED3B0A0BA809
:105BC00017F026FD05A88DED050ACDED060A96BB5A
:105BD00003C885E00128CED89DED020AB5EEC00AC3
:105BE000F1EE10FA7FDD07AED4F8AC21D4F8A8317D
:105BF00030460792089317F029FD23680BA90B95EF
:105C000020460C950D959B6C9847DDED077A9DED30
:105C10000B7A09AB77EE877A9DED0C7ACDED077A9A
:105C2000DDED087A77EE877ACDED087A96E8030005
:105C300083E8030049E02369B7EE008A04F5C879D8
:105C400004F5D07693ED000A03AF04F5CC7838EE76
:105C5000408A17F0DDFC8DED090A4846CDED0A0AB1
:105C6000B0EE480A17F0D4FC0BA92846CDED0C0A7B
:105C70008DED0B0A17F0ACFC3146C4ED650A3846D1
:105C800084ED640A17F0B4FC8DED090AB0EE480A01
:105C90004046CDED0A0A17F0BBFC0BA928468DED56
:105CA0000B0ACDED0C0A17F093FC84ED660AC4EDE7
:105CB000670A97E8030086E803004946404617F064
:105CC00087FC8DED090ACDED0A0A9DED090ADDED8F
:105CD0000A0A0FB0BDEC028BBDE8F083DDE90301D9
:105CE00085E80300F1E709950A95EEE735FA8E3C61
:105CF00010B590F84613044603F05AFD7C23C0B259
:105D000003FB0044D4F8A40010BD0000044B026F54
:105D10001B68DB6A5A60426F9A60826FDA60704774
:105D2000B4250030F0B58FB0044614F0D5FA002346
:105D300002AA90F8EB1402930546039304F194072A
:105D4000049301AB13F084F9D8B39DED010AB5EECD
:105D5000C00AF1EE10FA34DD04F1B00602A817F023
:105D600047FE394684ED2C0A3046C4ED2D0A84EDF9
:105D70002E1A17F04DFE04F17C01304617F0FCFDA1
:105D800004F1880105A88DED050ACDED060A8DED1B
:105D9000071A17F0F1FD08A88DED080A9DED010A1C
:105DA000CDED090A8DED0A1A17F012FE0BA904F1C8
:105DB00028008DED0B0ACDED0C0A8DED0D1A15F0B6
:105DC000CBFC95F8EB040C23394603FB005000F59F
:105DD0005C7017F0D1FD84ED2C0AC4ED2D0A84ED22
:105DE0002E1A0FB0F0BD0000804B2DE9F0470025C2
:105DF0001F6804460E462DED028BC0F89C508AB0F9
:105E0000C0F8985004F12809C0F89450C0F88450A4
:105E1000C0F88050C567C0F89050C0F88C50C0F8EA
:105E20008850C0F8B850C0F8B450C0F8B050F86A04
:105E300003685B68984700284CD062F0B3FE42F2DA
:105E40000F73984246D8FB6A484693ED010A84EDE9
:105E50001C0AD3ED020AC4ED1D0A93ED031A84ED6A
:105E60001E1A15F0F7FB49F0B7FFDFED617A94EDEC
:105E70001E6A062194ED1C7A26EE276A5D4A27EEFB
:105E8000277AB7EEC66A8DED046B94ED1D6A26EE97
:105E9000276AB7EEC77AB7EEC66A8DED007B8DED47
:105EA000026B42F0A9FE94ED1E8AB0EE480A8BF018
:105EB000D7F984ED6B0AB0EE480A8BF0ADFF84EDA4
:105EC0006A0A62F06FFEC4F87C010AB0BDEC028B76
:105ED000BDE8F087A6B194ED1C0AB4EE400AF1EEDD
:105EE00010FA0DD6D4ED1D0AF4EE600AF1EE10FAA8
:105EF00006D694ED1E1AB4EE411AF1EE10FA54D7FC
:105F000014F0EAF94FF00C0A90F8EC34B2EE028A81
:105F1000F2EE068A07460AFB030307AE4FF01508A8
:105F200003F5007393E8070086E80700304618F091
:105F30004BF9B4EEC80AF1EE10FA3AD508F1FF3881
:105F400018F0FF083ED1304618F03EF9F1EE047A21
:105F5000B4EEE70AF1EE10FA45DD9DED090ADDED3C
:105F6000087A20EE000A9DED078AA7EEA70AB7EE91
:105F7000C00A8CF0BBF8F7EEC00BB0EE480A8CF00C
:105F800047F9DDED090A84ED1D0A9DED080AF1EEE1
:105F9000600AB1EE400A8CF03BF984ED1C0A9FEDDB
:105FA000161AD4ED1D0A94ED1C0A484615F052FB52
:105FB00079E7304618F008F9B4EEE80AF1EE10FA85
:105FC000BCDCC0E7384612F091FE384612F070FF94
:105FD00097F8EC340AFB037303F5007393E80700AA
:105FE00086E80700A2E725676567D8E7B425003093
:105FF000E02E654270D10B08000000000021FFF781
:10600000F3BE000037B5044608461546019118F066
:10601000DBF8B7EE007AB4F8DC300198C7EE007A0E
:1060200094ED367A0133A4F8DC3037EE277A84ED2C
:10603000367AB0EE007AF4EEC77AF1EE10FA06D5B1
:10604000B6EE007AF4EEC77AF1EE10FA0DDC9FEDB1
:106050000E7AF4EEC77AF1EE10FA13D59FED0B7AB3
:10606000F4EEC77AF1EE10FA0CDDB0EE670A17F025
:10607000AFFC0120C5ED010A85ED000A85ED021A8D
:1060800003B030BD0020FBE700247449BD378635DE
:1060900070B500F1280600F1340504462946304663
:1060A0002DED028BB6EE008A8AB017F00DFD284662
:1060B00020EE088AB0EE480A17F08AFC07A930469D
:1060C000CDED080A8DED091A8DED070A17F06AFC6F
:1060D0008DED010AB0EE480A3046CDED020A8DED95
:1060E000031A17F075FC07A928468DED070ACDEDB8
:1060F000080A8DED091A17F055FC04A901A88DEDC9
:10610000040ACDED050A8DED061A17F0F1FC3246B2
:1061100001A920468DED070ACDED080A8DED091A7B
:10612000FFF770FF58B962F03DFD0121C4F8780116
:106130002046FFF759FE0AB0BDEC028B70BD2A461F
:1061400004A92046FFF75EFF0028ECD004F14002CE
:1061500007A92046FFF756FF0028E4D0EBE7000030
:1061600030B50D4604462DED028B284683B091F8DC
:10617000461303F01DFBC1B27C2000FB015104F16A
:106180002800943115F0FEF868468DED000ACDED3B
:10619000010A17F0D3FADFED1C7AB4EEE70AF1EE4C
:1061A00010FA05D59FED190A03B0BDEC028B30BD86
:1061B000684617F01DFB684617F0A4FA0028F1D1D5
:1061C00094ED488A284603F067FCF0EE400AB0EEF2
:1061D000480A14F0E7FC80B9284603F05DFCB0EEF5
:1061E000408A84ED480A8BF03BF884ED490AB0EE12
:1061F000480A8BF011FE84ED4A0A04F59271684654
:1062000017F04EFAD0E700BF000000340000000095
:10621000B7EEC00A9FED0C6BB4EEC60BF1EE10FAB0
:106220000BD49FED0B7BB4EEC70BF1EE10FA07DC3D
:1062300080EE067BB7EEC70B7047B7EE000A7047DB
:10624000B2EE040A704700BF0000005ADEECEB3FDC
:10625000000040F80A7421401C3008B517F06EFAAF
:10626000F1EE007AB4EEE70AF1EE10FA97BFF1EE24
:10627000027A9FED050A37EEC00ADFED047A98BF77
:1062800020EE270A08BD00BFCDCCCC3DCDCC4C3E86
:1062900008B5836993F9000038B10CF03BFDFDF7B8
:1062A000F5FD012894BF0020012008BDF8B52DEDB3
:1062B000028B054603F06EFE03F06AFD0446B8B398
:1062C000FFF7F8F890F8093393B32846FFF7E0FF9B
:1062D000064668B30CF01EFDB02790F8F432F0EEDD
:1062E000087A07FB030090ED3B7AB4EEE77AF1EE13
:1062F00010FA1DD495ED1E8A0CF00CFD90F8F432C6
:10630000DFED1E7A07FB030090ED3C0A98EE270AAA
:1063100014F004FDB0EEC00ADFED197AB4EEE70A1E
:10632000F1EE10FA08DC344662F03CFCC5F8680176
:106330002046BDEC028BF8BD05F5B67017F044FFA2
:10634000B0EE408A0CF0E6FC90F8F4329FED0D7A46
:1063500007FB0303D3ED3B7A67EE877AB4EEE78A57
:10636000F1EE10FADFD562F01DFCD5F86841001B94
:10637000B0F5FA6F8CBF00240124D9E7E02E654206
:1063800000003442CDCC4C3F0A4B1B6810B5DB6A91
:10639000044693F89C305BB962F004FCD4F87C317D
:1063A000C01A44F61F6398428CBF0020012010BD24
:1063B0000020FCE7B4250030F8B52DED068B04462F
:1063C0000CF0A8FC064603F0E5FD054606F0C2FB0E
:1063D000002840F0AD802046FFF768FF002800F05D
:1063E000AA802846FFF784FCD4F8E830984200F0F1
:1063F00020812846DFED969AFFF77AFCD4F8E83042
:10640000C31A284607EE903AF8EE677A67EEA99A23
:10641000FFF76EFC94F8BC30C4F8E800F3B92846E6
:1064200003F0C8FCD0B104F1280795F846232846AC
:10643000394603F035FBD4ED1D0AB0EE401A38465C
:1064400094ED1C0A15F006F90023C4F89030C4F846
:106450008C30C4F88830012384F8BC3020462946AB
:10646000FFF77EFE96F8F402B0EE408A06EB0010CD
:10647000D0F8A030C4F8EC3004F1B00094ED12AACA
:1064800017F0A2FE6368DFED737A28EE0AAA93ED97
:10649000007AB0EE409AB4EEE77AF1EE10FA01D548
:1064A000C3ED007A2046B0EE490AFFF7B1FE6368FB
:1064B00060EE0A8A93ED000A68EE808AFFF7CCFE50
:1064C000204668EE808AC4ED248AFFF75DFF38B16C
:1064D000B2EE007AD4ED247A67EE877AC4ED247A9E
:1064E000F0EE007AF4EEE79AF1EE10FA12D5B7EE7C
:1064F000C90A9FED557BB4EEC70BF1EE10FA09D532
:10650000DFED557A2AEE27AAD4ED2A7AEAEE297A27
:10651000C4ED2A7AB0EEC88A9FED500A94ED397A1C
:10652000DFED4F7A28EE008AA7EE278A84ED398ABC
:10653000BDEC068BF8BDFEF7BDFF90F80933002BCC
:1065400077D02046FFF7A4FE002872D096F8F422F8
:1065500006EB0213D3F8A010D4F8EC308B4268D0CD
:10656000B025F0EE087A05FB026292ED3B7AB4EEBC
:10657000E77AF1EE10FA5CDBCB1AC4F8EC109FED71
:10658000391A07EE903A96F8F43294ED1E0A05FB9C
:106590000363F8EE677ADFED349A93ED3C9A67EE89
:1065A000A99A29EE019A39EE400AB7EEC00A14F012
:1065B00021FCF7EEC08BB0EE680A8BF02DFC94F84E
:1065C000BC30B0EE408AF3B1F3EE047AF4EEE79A11
:1065D000F1EE10FA17DC96F8F402F2EE027A05FBFF
:1065E000006090ED3B7AB4EEE77AF1EE10FAFFF638
:1065F00043AFB0EEE80ADFED1D7AB4EEE70AF1EE44
:1066000010FAFFF639AFB0EE491AD4ED1D0A94ED39
:106610001C0A04F1280015F01DF89FED158A0123CE
:1066200084ED248A84ED238A84ED228A84F8BC30A8
:1066300022E7BDEC068B04F188009FED0E0ABDE851
:10664000F84017F019BA00BF000000481857D63FAD
:10665000BD378635CDCC4C3D0AD7233CCDCC4C3E06
:10666000CDCC4C3F35FA8E3C6F12833A1904863FED
:1066700000000000EC51783F0C2303FB010130B512
:1066800001F1C0038BB0144604AD93E8070085E820
:10669000070094E8070083E807002846FFF7D8F9C9
:1066A00007AB58B194E8070083E807009DED070A9F
:1066B000DDED080A9DED091A0BB030BD95E8070025
:1066C000F2E7000010B52DED028BDFED0E8AB0EE83
:1066D000408A044660EEA88AB0EE680A8AF0C0FDDF
:1066E00020EE480A84ED5B0AB0EE680A8BF094FB5A
:1066F00020EE480A0023BDEC028B84ED5C0AC4F84E
:10670000743110BD35FA8E3CF0B52DED028BD0F80A
:106710003031044685B00D468B60D0F83431CB6003
:1067200001F0D6FB06460CF0F5FAA369074693F98B
:106730000030022B53D1FDF7A9FB02284FD997F85F
:10674000F432B02202FB0373D3F8E0100022284693
:1067500002F070FB94ED501A94ED4F0A2846B7EE04
:10676000C11AB7EEC00A02F063FE94F8443183B355
:106770009FED258A62F016FA01AA97F8F4120646F0
:1067800038468DED018A0BF085FAD4F83801F0EE29
:10679000480A9FED1E0AB6EE001A361A4FF48760BB
:1067A00007EE906AF8EE677A27EE800A14F03AFB5B
:1067B000DDED017A04F5847030EE270A8DED010AD3
:1067C00016F026FF2846B7EEE01AB7EEC00A02F030
:1067D0002FFE94F8440105B0BDEC028BF0BD707C37
:1067E000242303FB006696ED0B8AFEF763FED0EDD3
:1067F0009C7A9FED077AF8EEE77AE8EE077AFDEEED
:10680000E77A17EE901AA1E7000000006F12833AB2
:106810000000C842F8B5036F00F14C050E4607466C
:106820000B6001F10C04436F4B60836F8B600FCDE5
:106830000FC40FCD0FC407F1B0022B68236006F11F
:10684000300307CA83E8070007F1940206F13C030E
:1068500007CA83E8070007F11C0206F1480307CACC
:1068600083E8070006F160013846FFF74DFF86F820
:106870007000F8BD30B589B004460D46684602F098
:10688000D3FA69462046FFF761F818B9002420467C
:1068900009B030BD04A802F0C7FA204604A9FFF7EA
:1068A00033FF04460028F1D004A9684602F0E2FC58
:1068B00085ED000AC5ED010A85ED021AE7E7000043
:1068C0001FB500230C4601A9019302930393FFF720
:1068D000D1FF08B1039B236004B010BD30B585B073
:1068E00000230C4601AD0193029329460393FFF761
:1068F000C1FF034618B195E8030084E80300184679
:1069000005B030BDF8B506460F461546FDF746F909
:10691000044690B13946FDF711F970B12046394669
:10692000FDF710F9044640B1FDF738F93946FDF797
:106930000BF985ED000A2046F8BDFEF7BBFD90F887
:10694000083343B13046FFF7A3FC044618B1D6F82C
:1069500064312B60EFE7D6F8643100242B60EAE75E
:1069600070B52DED048B1646FFF7CCFF054670B3CE
:10697000FEF7A0FD90F930424CB30CF0CBF9FDF7D7
:1069800085FA012823D9E4B207EE904AB8EE678A67
:106990000CF0C0F9B02290F8F43296ED009A02FBA8
:1069A0000300D0ED3B8AFEF771FF40F2614029EE13
:1069B000000A38EE281A78EEC80A14F033FAB0EE5E
:1069C000408AFEF763FFC8EE007AC6ED007A2846DB
:1069D000BDEC048B70BD000008B503F0DBFABDE828
:1069E000084003F0D5B9000010B5044617F09CF834
:1069F00050B904F10C0017F097F828B904F1180009
:106A0000BDE8104017F090B8012010BD38B500F176
:106A1000280504462846FFF7E7FF28B12046012154
:106A2000BDE83840FFF7E0B9B7EE007AD4ED107A50
:106A3000F4EEC77AF1EE10FA06D5BFEE007AF4EE66
:106A4000C77AF1EE10FA12DC2046FFF721FB284648
:106A5000FFF7CAFF0028E1D1D4ED107AB2EE047A34
:106A6000F0EEE77AF4EEC77AF1EE10FAD6DC38BD34
:106A700010B5044617F0A8FB2046BDE8104017F0FB
:106A80000FB800002DE9F04F044600274FF0000832
:106A900004F1F00B04F1280A2DED028BA3B0B0EE47
:106AA000408A5E460A970B970C97FFF785FC13F018
:106AB00013FC054695F8F1315FFA88F1022BA8BF67
:106AC00002238B423AD92846019112F02DF8019900
:106AD00080B310AB13AA284613971497159712F09A
:106AE00015FB9DED100AB5EEC00AF1EE10FA21DD9E
:106AF00013A816F07DFF1CA950468DED1C0ACDEDA4
:106B00001D0A8DED1E1A14F0E1FB8DED160AB0EE94
:106B1000480A16A8CDED170A8DED181A16F058FF81
:106B20001CA930468DED1C0ACDED1D0A8DED1E1AF7
:106B300016F06EFF08F101080C36BBE70C2395F840
:106B4000EC14504603FB015101F5007114F0BEFB3B
:106B500084ED070A94ED450AC4ED080A30EE088A70
:106B600084ED091A84ED458A0CF0D4F80646FEF748
:106B7000A1FC90F8093320460293FFF789FB80B10E
:106B80003046FDF783F902280BD996F8F422B0239A
:106B9000616903FB026391F9001093F802018842D6
:106BA00060DA94ED457ADFEDCB7AB4EEE77AF1EE78
:106BB00010FA61D494ED598AFEF76EFF38B1FCF7F4
:106BC000EDFF90F85611FCF7BFFFB0EE408A236C42
:106BD000B0EE480A626B1CA8A16A1E931D921C911C
:106BE00016F0F6FE04F5B6710AA88DED0A0ACDED91
:106BF0000B0A8DED0C1A16F00BFF61F0D3FF00238A
:106C0000019084F82C312046FFF742FB00286AD01F
:106C100096F8F422B02101FB0262D2F8E430C4F805
:106C2000303196F8F43201FB0363D3F8E830C4F84E
:106C3000343161F0B7FF0123C4F83801C4F83C7166
:106C4000C4F8407184F84431D4F81831002B5DD178
:106C5000019B04F5847423610AAB93E8070084E880
:106C6000070009E006EB0212D2F8A0200192019978
:106C7000D4F818218A4204D123B0BDEC028BBDE8C0
:106C8000F08F03F582730DF1280C93E8070094F858
:106C90002C318CE807001BB904F5847383E80700E6
:106CA0000123604604F5B67184F82C3116F07AFEA3
:106CB0001CA904F14C008DED1C0ACDED1D0A8DEDD3
:106CC0001E1A14F031FBB5EEC00A8DED1C0ACDED95
:106CD0001D0A8DED1E1AF1EE10FAD8BF9FED7E0A47
:106CE00084ED590A8FE794ED457AD4ED4F7ADDEDC6
:106CF0000A6AE6EE877ADDED0B6AC4ED4F7AD4EDD1
:106D0000507AE7EE267AC4ED507A9DE7D4ED457AC5
:106D1000724BF5EEC07A0D970E970F93F1EE10FAC5
:106D2000AAD99FED6F7A94F82C3167EE877AB7EE87
:106D3000007AC7EE278A1BB9029B002B00F0C380A4
:106D4000E36804F584710AA893ED008A16F02AFE20
:106D50008DED1C0A1CA828EE888ACDED1D0A8DED4C
:106D60001E1AB0EE480A16F033FE16A90DA8CDED96
:106D7000170A8DED160A8DED181A16F049FE0DA8AA
:106D8000FFF776FE0DA816F0E9FE20B161F00AFFCC
:106D9000C4F8780170E701231822002116A8039394
:106DA0008EF01EF8182200211CA88EF019F80DF1A3
:106DB000700805F20E534FF000099FED478A4FF01F
:106DC000FF37059395F8F1315FFA89F1022B1A46E6
:106DD000A8BF02228A4240F28B808B4204916BD979
:106DE000059B13F80930002B66D0B0EE680A5846B0
:106DF00016F042FEDDE90331002B66D00C2222ABF7
:106E0000204602FB0933A3F11802069304925A4666
:106E1000FFF732FC069B03ED060A049BC3ED010A53
:106E200083ED021A4046FEF713FE002844D1404687
:106E3000FFF71EFE404616F091FE00283CD10C23C1
:106E40000DA9404603FB09F222AB13440792A3F1BC
:106E500030020693049216F04BFE069B0DA94046A5
:106E600003ED0C0A049BC3ED010A83ED021A16F030
:106E70002BFE22AB079A03EB890303ED1A0A16AB2C
:106E8000981817F0A1F97A1C04D0B4EEC08AF1EE7C
:106E900010FA03DDB0EE408A4FFA89F722AB03EB1C
:106EA000870353ED1A7AF5EE407AF7EE007AF1EEA9
:106EB00010FA48BFB0EE678A09F1010908F10C0821
:106EC0000BF10C0B7EE7029B66E79BE8070088E866
:106ED0000700A7E7CDCC4C3E00000000000080BFBB
:106EE0000AE81C41CDCC4C3ECDCC4C3FCDCC4C3DEA
:106EF0007B1C3FF44BAF204684F81C71FFF7D6F99A
:106F000060B12046FFF7C4F9002840F0378122AA7B
:106F10000C2303FB0723002243F8282C16AA07EBB7
:106F2000470895F8EB3402EB880895F8F0219A426F
:106F300040F23F812B4493F80C35002B00F039814F
:106F400095F8EC3495F8F1219A4240F232812B44C5
:106F500093F80E35002B00F02C810C2322AA414619
:106F6000504603FB072714F0DFF907ED0C0A47ED45
:106F70000B0A07ED0A1A404616F0D6FD002840F02D
:106F80002481404616F0EAFD002840F01E815FEDA6
:106F90002B7A04F1B00094ED387A28EE278A5FED61
:106FA0002E7AA7EE278A84ED388A17F00DF9A368A8
:106FB0005FED327AB0EE408A93ED007AB4EEE77A74
:106FC000F1EE10FA00F105812046B0EE480AFFF715
:106FD0001FF9404616F0FCFCA3688DED130A13A8B8
:106FE000CDED140A8DED151A93ED000A16F0F0FCA4
:106FF000204684ED1F0AC4ED200A84ED211AFFF714
:10700000C3F928B1B2EE000A04F17C0016F034FD99
:10701000029BC3B33046FCF739FF012833D996F8F9
:10702000F402B023F0EE087A03FB006696ED3B7A9B
:10703000B4EEE77AF1EE10FA25D595F8EC040C23BE
:10704000F1EE0C7A03FB005595ED807AB4EEE77A09
:10705000F1EE10FA17DB94ED1D7A9FED606BB7EE41
:10706000C77AB4EEC67BF1EE10FA0CDD9FED5D6BD6
:10707000B4EEC67BF1EE10FA05D5B6EE000A04F1C7
:107080007C0016F0F9FCB7EEC88A9FED587BB4EE91
:10709000C78BF1EE10FA22D59FED560A404616F046
:1070A00097FC10A88DED100A94ED450ACDED110A5C
:1070B0008DED121A16F08CFC13A904F1A0008DEDD1
:1070C000130ACDED140A8DED151A16F0A1FCD4EDBE
:1070D0002B7A94ED457A77EE877AC4ED2B7AF1EE30
:1070E000047A94ED2B7A0025B4EEE77AF1EE10FAEB
:1070F0003BDB13F0F1F8DFED407A94ED2B1A40F210
:10710000C53094ED280A21EE271AF1EE410A8DEDE3
:10711000031ACDED020A13F085FE40F2C6309DED54
:10712000031ADDED020A84ED280A94ED290A13F012
:1071300079FE40F2C7309DED031ADDED020A84EDC1
:10714000290A94ED2A0A13F06DFE04F1A00104F15E
:10715000940084ED2A0A16F05BFCC4F8A850C4F829
:10716000A450C4F8A050C4F8AC501822002104F177
:10717000F0008DF035FEC4F8145169E5E368F7EED0
:10718000000A93ED000A13F00DFD00283FF4BFAE96
:1071900094ED1C0AB0EEC00A8AF03EFE0C2322AA2F
:1071A00003FB072353ED0A7A27EE800A03ED0A0A50
:1071B000B4E60C2322AA03FB0727002347F8283C48
:1071C00047F82C3C47F8303CD5E62046FFF71EFC3C
:1071D000DCE5C3ED007AF7E6AFF30080000000368F
:1071E00052C1E0BF0000003652C1E03F000000483D
:1071F0001857D63F728A0E3C5B821839F0B52DEDD8
:10720000048B9FB0044613F067F800F59F6390ED80
:107210007F8AD3ED007AF4EE487AF1EE10FA48BF97
:10722000B0EE678ADFED557AB4EEE78AF1EE10FA38
:107230000CDD1822002104F1F0008DF0D1FD0023B7
:10724000C4F814311FB0BDEC048BF0BD204614AD62
:10725000FEF768FD2046FEF71BFFB0EE480A204609
:1072600004F14C06FFF70EFC2046FFF7CFFBFEF7BC
:1072700021F904F1280100F5347214A814F0A4F8DF
:107280000FCD0FC60FCD0FC62B6804F1740204F1A9
:10729000700104F14C00336004F1780314F03AFA01
:1072A00094ED1E8AB0EE480A89F0DAFF84ED6B0A8D
:1072B000B0EE480A8AF0B0FD204684ED6A0AFEF777
:1072C00025FDFEF7F7F804F5C071FDF7FDFE61F04E
:1072D00069FCD4F8B031C31A632BB3D9C4F8B00138
:1072E0003EF0F6FA054661F065FCDFED257A94ED97
:1072F0001E0A074694ED1C8A0E4694ED1D9A20EE58
:10730000270A28EE278A29EE279A13F0F1FC94ED3C
:107310005D7AB7EEC00A1B4BB7EEC88AB7EEC77AE4
:10732000194AB7EEC99A0193184B28461849009399
:10733000184B8DED127B94ED5C7AB7EEC77A8DED2C
:10734000080B8DED107B94ED5B7AB7EEC77A8DED6F
:10735000069B8DED0E7B94ED397AB7EEC77A8DEDF5
:10736000048B8DED0C7B94ED387AB7EEC77ACDE9BE
:1073700002768DED0A7B3DF0EBFE63E7CDCC4C3E13
:10738000E02E6542D5D10B08A6D10B08DFD10B0842
:1073900028D00B089CD10B08094A0123D2ED057AAD
:1073A000D8B2F4EEC07AF1EE10FA02DD0138C0B2C4
:1073B000704701331432082BF0D10720704700BF0B
:1073C000C4D20B080C4B1422DFED0C6AF0EE407AAD
:1073D00002FB003090ED047A90ED010AB0EEC76A2E
:1073E000B4EEE66AF1EE10FA5EBFD0ED006A77EE19
:1073F000E67AA7EE270A7047C4D20B0800000034D3
:1074000010B504463648F0EE407A012103462DEDD2
:10741000068B90ED077ACAB2F4EEC77AF1EE10FA55
:1074200023DD013AD2B2142101FB023393ED027A3B
:1074300087EE870ADFED2B7AB4EEE70AF1EE10FA59
:1074400019DA3CF0D5FBA7224FF480113CF088FB01
:10745000637C2422D4ED257A02FB034393ED0B0ACF
:1074600030EE270ABDEC068B10BD0131143008291F
:10747000CFD10722D7E793ED049A93ED008AB0EEBF
:10748000C97AD3ED019ADFED188A9FED18AAB4EE00
:10749000E77AF1EE10FA12D58AF0E2F968EEE98A9D
:1074A000F0EE487A88EE8A7AE0EE077A9FED107A5D
:1074B00067EE876A77EE677A86EEA70AD2E768EE0C
:1074C000C98AC8EE8A0A8AF0E9FA89EE897AF7EE63
:1074D000007A30EE670AF0EE487AE7EE007AE5E7E8
:1074E000C4D20B0800000034CB868F430AE81C414D
:1074F0003CFEC14ADFED257A254920EE277A30EEA1
:10750000270A08B587EE005A2DED028BB0EE450A2A
:10751000FFF742FF142303FB001140B2FFF752FFB5
:10752000DFED1C7AD1ED045A91ED038AB0EEE57AD5
:10753000B4EEE77ADFED187AF1EE10FA12D520EE0C
:10754000270A9FED167AC7EE007A91ED000A35EE14
:10755000400A27EE800A8AF009F928EE000ABDECFD
:10756000028B08BD65EEA75ADFED0D7AC7EEA50ABE
:10757000F7EE007A70EEA70AD1ED017A80EE270AC5
:10758000F1EE600A8AF08AFAE7E700BF3CFEC14AE2
:10759000C4D20B0800000034CB868F430AE81CC11C
:1075A0000AE81C4108B5FFF7A5FFDFED097AB4EE44
:1075B000E70ADFED087ABDE80840F1EE10FA20FE98
:1075C000270ADFED057A87EE800A8AF04DBE00BFFC
:1075D00000000034BC77E936CDCC9C3F10B52DEDD2
:1075E000028BF0EE608A0446FFF70AFFB0EE408A95
:1075F0002046B0EE680AFFF703FF30EE480ABDEC04
:10760000028B10BD427C2421D0ED257A01FB0202C1
:1076100092ED0B0A30EE270AFFF7C4BF38B52DED07
:10762000088BB0EE409A0546F0EE609A1524B0EE55
:10763000408ADFED1DAA9FED1DAA9FED1DBA013CFA
:10764000A4B25CB3F0EE490A2846B0EE480AFFF750
:10765000C5FF70EE698AF0EE490A284638EE2A0A1C
:10766000FFF7BCFFB0EEE87A70EE697AB4EECA7A42
:1076700077EEE87AF1EE10FA10D468EEAA8A40F2BA
:107680006310B0EE4B1AF0EE4A0A88EEA70A38EE05
:10769000400A13F0C7FBB0EE408AD0E7B0EE480ACC
:1076A000BDEC088B38BD00BFCDCCCC3D0AD7233C08
:1076B00000247449002343608360C3600361436115
:1076C0008361C361002380F82030704790F8202048
:1076D000531C00EB8202DBB2062B80F8203082EDD7
:1076E000010A84BF002380F8203070474FF0FF3339
:1076F00010B5436104460D4BA8300360002380F8A9
:107700002030FFF7D7FF0A4B04F58670C4F8A83085
:1077100060F0E6F9074B204607491C6039F09AFBF8
:10772000D4F890302046C4F8943010BD9CD40B0897
:10773000ACD40B08AC66003044D50B08A83008B5B3
:1077400040F064FADFED027A20EE270A08BD00BFA0
:1077500000007A4490ED3C0ADFED057AB0EEC07A85
:10776000B4EEE77AF1EE10FA48BF90ED3D0A7047AB
:107770000000003473B5D0F8A43004460E4663B15F
:1077800061F010FAD4F8A430C01A42F20F73984294
:1077900003D894ED280A02B070BD114B1D687DB16D
:1077A00095F856112846FCF7CDF948B101AA95F88D
:1077B00056112846FCF7BCF910B19DED010AEAE725
:1077C0002421DFED087A01FB064494ED0A0AB4EEA9
:1077D000E70AF1EE10FA58BFB0EE670ADBE700BF28
:1077E000A466003000000C4208B561B10378022B9A
:1077F00002D9064861F0A8F95A1C027000EB830018
:107800004160012008BD0846FCE700BF64D30B08B7
:107810002DE9F84305460E469146002400F13C0848
:107820002B78A34211DD00234A46314601200FF098
:1078300051FA242307460021634358F803000FF050
:1078400059FA874204D00134EAE70020BDE8F88302
:107850000120FBE7054B1B682BB141694A1C02D094
:1078600018463DF059BE0020704700BF8C690030BB
:1078700002290BD8242303FB010191F8390030B110
:1078800091F83A0018B191F83B007047002070471A
:107890002DE9F047044661F085F942F210730027A4
:1078A000D4F8F8604FF0240942F2107A861B9E4209
:1078B00088BFC4F8F800FDB2237CAB421CD929462E
:1078C0002046FFF7D5FF70B109FB0548D4ED250A26
:1078D000204698ED0D0AD8ED097A30EE270AFFF719
:1078E0009DFE88ED0C0A564504D909FB0540303051
:1078F00039F086FC0137DEE7617C2046FFF73AFF6E
:1079000084ED3D0ABDE8F08770B5044686B061F0AD
:1079100049F90546D4F89830C31AB3F57A7F4DD3A8
:1079200094ED257ADFED326AB0EEC76A314BD4EDC3
:10793000247A1B68B4EEE66ADB6AF1EE10FA93F87B
:107940009C6030D5B0EEE76AB4EEE66AF1EE10FA6C
:1079500029D502A801F068FA86BBFDF7ABFD02A9A4
:10796000FDF7B2FB50B3DDED037A9FED237AF8EE1D
:10797000E77A67EE877AC4ED257AC4F89850FDF768
:1079800099FDFDF769F92046FFF782FF48F024FAD8
:1079900094ED257A194A0621B7EEC77A8DED007B62
:1079A00041F02AF90AE037EE676AF7EE005AB0EEC6
:1079B000C66AB4EEE56AF1EE10FA01DC06B070BDFD
:1079C000B0EEE76AB4EEE66AF1EE10FAF6D4002EF5
:1079D000D1D02046903080ED007A39F011FC48F08B
:1079E000FBF9074A012106B0BDE8704041F004B937
:1079F00000000034B42500300AD7233CA5D30B087F
:107A000080D30B08F0B52DED048B85B004464FF400
:107A1000537200F5867103A800250FF0E7FAD4ED44
:107A2000227AD4ED236A24229FED786A37EEE67A33
:107A3000637C02FB0343B0EEC77AB4EEC67AF1EE84
:107A400010FAC1BF9FED727A67EE877A9FED717A67
:107A5000E6EE877AC4ED237A93F83960E9B22378A9
:107A60008B4206D904EB81030135586863F01EFA96
:107A7000F4E70027DFED688A9FED688A9FED689A3A
:107A8000237CFDB2AB4264D9242303FB054393F866
:107A90003920002A5BD0D3ED0C7AF4EEE87AF1EECF
:107AA00010FA0BDBF4EE677AF1EE10FA06D6F0EE80
:107AB000E77AF4EE487AF1EE10FA04DD242303FBB2
:107AC00005435A6A1A63242303FB0543D3ED090ACD
:107AD000D3ED0D7A93F8382070EEA70AA2B993ED92
:107AE0000C0A2046FFF77AFDD4ED257A30EE670ABE
:107AF000B4EE400AF1EE10FA16D7242303FB054535
:107B0000002385F83A3022E0012A09BFD3ED0C7A30
:107B100093ED0B0A77EEE00AD4ED3B7A04BF80EEDA
:107B2000897A87EE270AE3E7F0EEC07A242303FB85
:107B30000545F4EE487AF1EE10FAE1DC012385F810
:107B40003A30D4ED237A37EE800A85ED0B0A0137FF
:107B500096E7627C20461146FFF78AFE48B1242151
:107B600004F1A80001FB0242D16992ED0B0A40F03A
:107B70002FF894F99C10277C002907DBB94205DA1D
:107B8000CAB220461146FFF773FE68B9002262743C
:107B9000D5B2AF4209D9294620460132FFF768FE27
:107BA0000028F5D0657400E062742046FFF7ACFE53
:107BB0002046FFF74FFE10B1204664F083F9637C46
:107BC000242505FB034393F83930B34216D03DF02A
:107BD0007FFE4FF6FF713DF09FFC78B1607C05FBA6
:107BE000004494F83930002B14BF00220422019283
:107BF0003DF06EFE019A12213DF020FC03A80FF02B
:107C000017FA05B0BDEC048BF0BD00BF0AD7233CCA
:107C10000AD7A33C48E17A3F00000034FFFF7F7F92
:107C2000002019462DE9F04F04460F4687B0007C2E
:107C300004F13A0300220121D5B22433A84205D928
:107C4000013203F8231C03F8241CF5E76F4B1E6870
:107C5000F06A03685B68984740B148F0BDF86C4A29
:107C6000062107B0BDE8F04F40F0C6BF48F0B4F8B9
:107C7000684A06210A2540F0BFFF002303A904F14A
:107C80008800039339F0C6FE60F08CFF80462046E2
:107C9000FFF7B8FE60F086FFA0EB0800B0F5FA7FB2
:107CA00002D95D4801F0A4F8B06A0A2103685B6854
:107CB0009847617C2046FFF7DBFD0028E7D0B06ADB
:107CC000013D642103685B68984715F0FF05DBD12F
:107CD000524B05951B888DF80650ADF80430CDE960
:107CE0000355052560F05EFF80462046FFF78AFEBB
:107CF00060F058FFA0EB0800B0F5FA7FD1D8617CA6
:107D00002046FFF7B5FD0028EFD094F810B00DF134
:107D10000C08A14601AA4FF0000A5FFA8AF18B45D0
:107D200016D92046FFF7A4FD50B1D8ED007A99EDA1
:107D3000097A137877EE877A0133C8ED007A1370E9
:107D40000AF1010A08F1040809F124090132E4E703
:107D5000B06A013D642103685B68984715F0FF0530
:107D6000C0D1A9464FF02408237C5FFA89F6B342BC
:107D700026D906AB334413F8143C33B908FB064646
:107D800086F83B3009F10109EEE7002FFAD006AA88
:107D900007EE903A2046D4ED250A02EB8602F8EE73
:107DA000E77A12ED030A80EE270AFFF737FC08FB9B
:107DB000064002A98DED020A303039F02BFEE1E7D2
:107DC00000264FF02408DFF85C902046617CFFF726
:107DD000D1FC84ED3D0A237CF7B2BB420FD908FBEE
:107DE000074393F83B3043B1013547F0F5FF7B1C67
:107DF0004A46EDB2062140F0FFFE0136EBE70DB931
:107E000007484FE707B0BDE8F08F00BFB42500304A
:107E1000C0D30B08EBD30B0801D40B08E48D0B087F
:107E20003DD40B081BD40B0808B5037C022B02D9E8
:107E3000034860F089FE5A1C0274184608BD00BF52
:107E40005CD40B0838B50246057C0024E1B28D42B3
:107E500006D910460134FFF70BFD0028F6D138BDD6
:107E6000281E18BF0120FAE770B50D4609780446B0
:107E7000072906D8027E437E22B901228A40134395
:107E8000437670BD002BFCD000262278F3B29A42D4
:107E9000F7D904EB83032946013658680368DB6889
:107EA0009847F2E737B50D460192FFF7CBFF0199EE
:107EB000044630B904482A46044B0068C06A0FF0F3
:107EC0006FFA204603B030BDB42500300B4C0D08CE
:107ED000014B1868704700BFAC66003010B504460F
:107EE000006810B103685B689847204610BD000029
:107EF000002213B50B680A6001A9019363F028FB07
:107F0000044601A8FFF7EAFF204602B010BD0000BA
:107F1000002213B50B680A60022201A9019364F0E4
:107F200005FD044601A8FFF7D9FF204602B010BDA9
:107F3000002213B50B680A60012201A9019364F0C5
:107F4000F5FC044601A8FFF7C9FF204602B010BDAA
:107F5000002213B50B680A6001A9019364F0E6FCE6
:107F6000044601A8FFF7BAFF204602B010BD00008A
:107F700010B50446006810B103685B689847204656
:107F800010BD00002DE9F04F8FB0D0F8003104464D
:107F9000344D0893344B05F1D80A1B685868059393
:107FA00003689B68984794F99D300690002BA2BF08
:107FB000012606FA03F306932B68089A1A420BD09F
:107FC00000274FF0010BB9460BFA07F3069A13424C
:107FD00006D10137202FF7D10C355545ECD12DE0D6
:107FE000F9B26B682A7A204609910793FFF710FCD3
:107FF0000999804628B3CDE90A990B9B0DA9204623
:108000000D93079BCDE90B99984701462046FFF752
:10801000EBFB0DA8FFF762FF0CA8FFF75FFF0BA8B3
:10802000FFF7A6FFB8F1000F02D00AA8FFF7A0FFE4
:108030002378032B02D0237C032BCAD10FB0BDE8D9
:10804000F08F059B042258680368CDE90182074A36
:1080500000920A461B6801460BA81E462B7AB047C1
:10806000CBE700BF34D60B08B4250030801A0600D9
:1080700070B5D0ED247A01239FED647A8AB0F0EEDA
:10808000E77A04460376F4EEC77AF1EE10FA09D4E3
:108090009030002309A90590099339F0BBFC05989D
:1080A00039F0AEF80026772220463146E663266690
:1080B000C4F88460FFF7ACFB054600283FD0CDE94B
:1080C0000666079A002309A920460992CDE90733DD
:1080D00064F080FF01462046FFF786FB09A8FFF702
:1080E000FDFE08A8FFF7FAFE07A8FFF741FF15B14C
:1080F00006A8FFF73DFF2378032B59D0237C032BE1
:1081000056D094F99D10002928DA2046FFF73AFF4F
:10811000D4F80031DA045DD40025637EEAB2EB4086
:10812000DB075DD40135082DF7D1237823B1237CFB
:1081300013B16368002B3BD1354800F059FE354B35
:1081400004221B6859680B68CDE90102324A00928B
:1081500002461E6807A87723B047B2E77722C9B264
:108160002046FFF755FB054620B30023CDE9063333
:10817000079B002209A920460993CDE9072264F054
:10818000D5FB01462046FFF72FFB09A8FFF7A6FE07
:1081900008A8FFF7A3FE07A8FFF7EAFE15B106A897
:1081A000FFF7E6FE2378032B02D0237C032BACD110
:1081B0000AB070BD174B04221B6859680B68CDE9E3
:1081C0000102154A07A8009294F89D201E687723A3
:1081D000B047CDE7637E002B9ED1012363769BE7FA
:1081E0003820059201F030F9064618B1059A21466B
:1081F00064F03AFC31462046FFF7F6FA2378032B69
:10820000D6D0237C032B8DD1D2E700BF00000034F1
:1082100070D40B08B4250030801A060090F884351D
:10822000934207D900EB8200D0F85C0510B10368D7
:108230009B6A1847002070472DE9F3416E460546BA
:1082400004460F4600F5C87886E80C00114B45F847
:10825000043B28462C3500F0D1FCA845F9D104F5A3
:10826000B163C4F8807596E8030083E80300089BB7
:1082700020460949C4F8903538F0ECFD074B1A68E0
:1082800012B1074860F060FC20461C6002B0BDE8F7
:10829000F08100BF3CD90B0804D80B08B066003051
:1082A00048D70B082DE9F041A2B00C4607A937F0DA
:1082B00079FF002856D000210D220CA80BAD0591A6
:1082C000ADF818100B918CF08BFD611C2A4B0A95B0
:1082D000C9B21F680129F86A47D1284B062205A9AF
:1082E0000FF05EF8264B002411222946019305ABBE
:1082F0008DF819400093F86A224B0FF051F804AA48
:108300000DF10F0128468DF83C40049439F052FAE3
:1083100040B3062610ACDFF86C8048221A4910A83A
:108320008CF014FD226829460C34531E049AC2F3C3
:10833000513202EB831214F8083C8DF8243054F8C3
:10834000043C08921122019305AB00934346F86A5E
:108350000FF026F8B7EE000A002107A838F0D0F891
:10836000013EDFD122B0BDE8F08100910622074B2B
:1083700005A90FF015F8B5E7B42500309FC40B0828
:1083800079D70B0873D70B08E88D0B086CD70B084F
:108390002DE9F04F90F8848585B00446B8F1000FC0
:1083A0004BD17F2304F5C87504F25C57261D80F875
:1083B000943504230DF10F012A308DF80F3039F078
:1083C00065FB5FFA88FA1C22FF2128468CF008FD25
:1083D00085F863A096F92690B9F1150F6AD03FDCB5
:1083E000B9F1090F5AD02BDCA9F10303DBB2012B41
:1083F00047D9386850B1A96EC5F8649031B1394B8E
:1084000043F8281038F032FF38F028FF0AF101094C
:1084100057F8040B5FFA89F940B103689B689847E5
:108420005146204684F88495FFF73CFF08F1010887
:108430006C352C36B8F1090FC3D105B0BDE8F08F0B
:10844000B9F10A0FD5D1302000F0FEFF834610B3FA
:1084500033462A462146CDF800A066F037F91AE0E7
:10846000B9F1190F32D0B9F11C0FC2D15C2000F064
:10847000EBFF834678B133462A46214664F056FE28
:1084800009E0442000F0E0FF834620B133462A464D
:10849000214664F0A5FFC7F800B0AAE7382000F035
:1084A000D3FF83460028F6D033462A46214665F09E
:1084B000F9FBF0E7782000F0C7FF83460028EAD0F8
:1084C00033462A46214665F055FCE4E7482000F093
:1084D000BBFF83460028DED033462A46214666F09D
:1084E00073F9D8E7B466003090F884358B4283BFC7
:1084F0006C2303FB010090F8E101002070470000AD
:1085000090F884358B4283BF6C2303FB010090ED10
:108510006B0A9FED010A70470000000090F8843557
:108520008B4206D900EB8100D0F85C0508B165F0FC
:10853000F5B89FED010A70470000000010B490F8F4
:1085400084450A468C4214D900EB8104D4F85C457A
:108550007CB1E468246A640603D55DF8044BFFF738
:10856000DDBF6C2101FB020393ED6B0A5DF8044B48
:1085700070479FED010AF9E70000000090F884358C
:108580008B420BD900EB8100D0F85C0538B1C36891
:108590001B6A1A4214BF0120002070470020704758
:1085A00070B590F8843504460E461546934201D8BE
:1085B000002070BD00EB8203D3F85C050028F7D0E3
:1085C00003689B6998470028F2D06C2202FB05449F
:1085D000D4F8B0313360ECE770B590F884350446D8
:1085E0000E461546934201D8002070BD00EB820371
:1085F000D3F85C050028F7D003689B6998470028EA
:10860000F2D06C2202FB0544D4ED6D7AF4EE677A69
:10861000F1EE10FAE8D6C6ED007AE6E770B590F80C
:10862000843504460E461546934201D8002070BD9D
:1086300000EB8203D3F85C050028F7D003685B6980
:1086400098470028F2D06C2202FB0544D4F8B831D8
:108650003360ECE790F8843593420ED900EB820347
:10866000D3F85C355BB16C2303FB020292F8F00196
:1086700030B1D2F8EC310B607047002070471846DB
:108680007047000008299DBF2C2303FB01004068B0
:1086900000207047474B1B682DE9F04F2DED028BF2
:1086A000DB6A87B0044693F89C30002B7DD04FF0F6
:1086B0000009DFF814A1DFF814B19FED3F8A5FFADB
:1086C00089F594F88435AB426FD904EB8503D3F870
:1086D0005C05002853D003685B6B98476C23074602
:1086E00003FB054393F8E031834248D2032857D86F
:1086F000DFE800F04502484F304E4FF0000847F0E9
:108700006BFB94F884256B1C0421AA4289BF6C2260
:10871000B0EE487A02FB054292ED6B7A6C2202FBC6
:108720000545B7EEC77A524695ED6D6A0096B7EEED
:10873000C66A8DED027B8DED046B40F05DFA01237E
:1087400084F895358BF80B3085F8E071D4F89035C6
:108750004BB3002255B25957481C03D0414502F192
:108760000102F7D194F99435AB4208DBD4F88C358B
:1087700042463146D4F88805984784F8945509F163
:1087800001099CE72C230E4E03FB054393F92D8032
:10879000B5E72C230B4E03FB054393F92E80AEE780
:1087A0000026B046ABE71D46DCE707B0BDEC028B08
:1087B000BDE8F08FB4250030000000008DD70B0815
:1087C0006E590D0884D70B089CD70B082D67003015
:1087D00090F884358B4207D900EB8100D0F85C0516
:1087E00010B10368DB6918470020704708299CBF57
:1087F0006C2303FB010000F5C870704790F88435C6
:10880000934207D900EB8200D0F85C0510B10368F1
:108810005B6A18470020704790F884358B420DD969
:1088200000EB8103D3F85C3543B16C2303FB0101FA
:10883000012081ED740A81F8CC0170470020704757
:10884000F8B5002402460E462C272546E1B292F8E0
:1088500084358B4210D902EB8103D3F85C354BB1E0
:1088600007FB01239B689E4204D11046FFF7D4FF0B
:108870002843C5B20134E9E72846F8BD2DE9F04F99
:10888000002493B005460E46174621462F2206A81F
:10889000059405F25C598CF0A3FA05F12A0A4FF011
:1088A0002C0B05F5FA730BFB04F259F8040BE5B237
:1088B0001AF9021030B951B90134092CF3D14FF033
:1088C000010813E06C2262439A58914212D001359C
:1088D0001448154B4FF000080068EDB20193324682
:1088E00000953946114BC06A0EF05AFD404613B050
:1088F000BDE8F08F05A93322039364F0EFFF05A9CB
:108900008046039B0028D7D10135064801913246A5
:10891000EDB20068054B39460095C06A0EF040FD87
:10892000E4E700BFB4250030D2D70B08C4D70B084A
:108930002DE9F04F06468DB00027DFF87C90DFF878
:108940007CA0DFF87CB096F88435FCB2A3422ED927
:108950006C2505FB046595F8E83133B395F8E9110A
:1089600019BB4FF00108202204A8444489F819805B
:108970008CF036FA4AF2104307EE904A03AA4C21D3
:108980005046F8EEE77AADF828302423CDED037A8F
:1089900042F050F847F020FA9BF80030054A0421D5
:1089A000009440F029F985F8E9810137CBE70DB053
:1089B000BDE8F08FDCD70B082D670030886A0030E7
:1089C000E8220030304B2DE9F04F1E6885B0044698
:1089D00046B1D0F8801530463CF09EFD10B13046CF
:1089E0003BF000FD4FF000084FF02C0A4FF06C0BED
:1089F00060F0D8F801905FFA88F594F88435AB42BE
:108A000039D904EB8507D7F85C0588B30AFB054321
:108A10000BFB054993F92A20D9F8F4118A4227D192
:108A200032B30268D2689047D7F85C050268126BCF
:108A3000904799F8E12112B1019BC9F8E431BEB128
:108A4000D4F8801530463CF067FD88B160F0B2F88C
:108A500002460B46CDE902102946D7F85C0565F0C1
:108A600083FC2946D7F85C05DDE9023265F0FAFCA3
:108A700008F10108BFE72046FFF70CFE204605B0CD
:108A8000BDE8F04FFFF754BF8C6900302DE9F04787
:108A90004FF0000804468946012647464FF06C0A0D
:108AA0002DED028BB0EE408A94F884355FFA88F59C
:108AB000AB421AD929FA05F3DB070AD504EB850383
:108AC000D3F85C0578B10368B0EE480A9B6B984711
:108AD00006400AFB054508F1010895F8E0319F4280
:108AE00038BF1F46E0E70646F3E727B97F23A4F81F
:108AF0009435034BDF723046BDEC028BBDE8F08746
:108B00002D67003090F884358B4207D900EB810047
:108B1000D0F85C0510B10368DB6B18470020704784
:108B20000B46114690F884259A4207D900EB830042
:108B3000D0F85C0510B103681B6C18477047000043
:108B400070B504460E460025E9B294F884358B4290
:108B500005D9324620460135FFF7E2FFF4E770BD44
:108B60002DE9F843024690F88455002400F12A06C6
:108B70002C2700F5FA784FF06C09E1B28D420FD93D
:108B800007FB04F309FB04F0F35658F80000834296
:108B900009D11BB11046FFF7A7FC10B10134ECE777
:108BA0000120BDE8F8830020FBE7000010B590F835
:108BB000842504468A4217D96C2202FB010393F8EC
:108BC000E031022B03D004D9032B18BF0023184631
:108BD00010BDFFF797FF48B92046FFF7C1FF0028F7
:108BE0000CBF06230123F2E70023F0E70623EEE79C
:108BF000014B1868704700BFB066003010B50446DE
:108C0000024938F027F9204610BD00BFBCD90B0837
:108C100010B50446203051F0E3FA044B20460449D5
:108C20001C6038F017F9204610BD00BFD866003030
:108C300050DB0B082DE9F3410546B7EE000A002290
:108C4000022137F073FD284665F026FE51F042FB05
:108C5000234B04461E68F06A03685B6A98470B461C
:108C6000022102462046009151F0D0FAB5F94A702F
:108C7000002F13DDD6F82C80BCB2D8F80030404667
:108C80005B68984728B198F84D3013B1C92FA8BF39
:108C9000C824B06A214603685B68984720220021F7
:108CA00095F9490012F026F9C4B254F0EFF954F0E6
:108CB00053F970B9B06A013405210368E4B25B6806
:108CC0009847072CF1D9074802B0BDE8F0415FF0A2
:108CD00027B8072CF7D885F8494002B0BDE8F081E5
:108CE000B4250030BCDA0B0810B5044665F08AFDE7
:108CF0002046BDE8104065F0B5BD00002DE9804874
:108D00001446284B012293B005460E464FF000084A
:108D1000DFF89490DFF894A0DFF894B01A705FF059
:108D200041FFD9F80030A0EB08020746039341F257
:108D300087339A421FD903985346342205A9B8466F
:108D4000CDE90056C06A0EF02BFB214605A804941D
:108D50005EF0D6FF03985B46342205A9CDE90056A4
:108D6000C06A0EF01DFB049447F036F8049B05AA78
:108D700002213FF027FF47F02FF846F051FA47F065
:108D80002BF848F02FFA0A2105A80EF015F9039BDD
:108D90000521986A03685B68984705A80EF018F9E2
:108DA000BDE700BFDC660030B425003029710C0837
:108DB0007D6E0D080FB400B595B0002116AA05A868
:108DC000049152F8043B03923C2201938CF008F882
:108DD000054A4021019B04A85EF03AFF039A04A9CA
:108DE0000248FFF78BFF00BFD4DA0B08EADA0B0862
:108DF0000FB407B504AA034852F8041B0192FFF709
:108E00007DFF00BFFCDA0B081022044908B58BF087
:108E10008DFFB0FA80F0400908BD00BFE066003069
:108E2000102200218BF0DCBF10B50446FFF7F8FFDD
:108E3000204610BD0378022A416023F00D03037021
:108E400008D0032A0AD0012A03D1DBB243F0010380
:108E500003707047037843F00803F9E7037823F0C1
:108E6000050343F00503F3E773B504460E461546C4
:108E70000193FFF7D5FF2046069A0199C4E90265E0
:108E8000FFF7D8FF02B070BD0078420704D4030793
:108E900004D400F00100704703207047022070479F
:108EA000F0B587B004461546FFF7EEFF88420F463F
:108EB000064605D163682B600126304607B0F0BD39
:108EC00000230328019301D0032913D13AF082F93A
:108ED00008B90026F1E7012301AA214639F0BAFFBB
:108EE0000028F6D0DDED017A9FED337A67EE877AC0
:108EF000CDED017A032E32D8DFE806F00209162400
:108F00006468032FE5D8DFE807F02C2E3C49FCF716
:108F1000D1FA90F87C32DB07DBD56468FCF7CAFA3B
:108F2000D0F870321C44ECE702A8FFF779FFFCF799
:108F3000C1FA02A9FCF7C8F806460028BDD064684B
:108F4000039BEFE7D4ED017A9DED017AF8EEE77A25
:108F500077EE877AFDEEE77A17EE904AD1E70024A4
:108F6000CFE72C60A8E7FCF7A5FA90F87C6216F032
:108F70000106AED0FCF79EFAD0F87032E41A2C60ED
:108F80009BE702A8FFF74CFFFCF794FA02A9FCF755
:108F90009BF80646002890D0039BEFE707EE904A27
:108FA0009DED017AF8EEE77A77EEC77AFDEEE77A83
:108FB000C5ED007A80E700BF0000C84273B501AA82
:108FC00005460E46FFF76CFF044620B13246019974
:108FD0002846FFF72FFF204602B070BD13B5144698
:108FE00001AAFFF75DFF48B1DDED017A9FED047A3C
:108FF000F8EEE77A67EE877AC4ED007A02B010BD2A
:109000000AD7233C07EE900A9FED0C0AF8EEE77AA8
:1090100008B527EE800A88F023F9DFED097AB4EE6F
:10902000E70AF1EE10FA02DDB7EEC00A08BD9FEDC7
:10903000010BFBE700000040E17A843F50E0EF3095
:109040000AD7233C10B50446806812F0D5F820B149
:10905000E068BDE8104012F0E3B810BD0D4B83424C
:109060004FF000038B4106DA00F1255000F5311076
:1090700000F5E0507047084B98424FF0FF3371EB1A
:109080000303BEBF00F1564000F5130000F5244075
:10909000704700BF00D2496B002EB69490EA010FD2
:1090A00001D4401A7047C317401A63EBE1710D4BAE
:1090B00083424FF000038B4106DA00F1255000F5A2
:1090C000311000F5E0507047074B98424FF0FF33E6
:1090D00071EB0303BEBF00F1564000F5130000F52D
:1090E0002440704700D2496B002EB69470B52DED28
:1090F000028B84B004460D466846FFF791FEFCF7EC
:10910000D9F96946FBF7E0FF064628B3A368029A3F
:10911000DFED148A9B1A039907EE903AF8EEE77A8E
:1091200067EEA87AC5ED007AE068FFF7B7FF08EEB2
:10913000100AA068B8EEC88A024428EE288A02EB1A
:10914000D2725010B7EEC88AFFF75CFF28EE000B12
:10915000B7EEC00B85ED010A304604B0BDEC028BC2
:1091600070BD00BFF67C8E3F002337B50C4601AAC8
:10917000022105460193FFF793FE10B9002003B0CA
:1091800030BD21462846FFF7B1FF0028F6D0DDEDBF
:10919000017AF8EEE77AC4ED027AF0E738B50C46CA
:1091A00002462DED028BC168E068FFF777FF9568F6
:1091B000A46808EE100A6019641B00EBD070401020
:1091C000FFF720FF07EE904AB8EEC81BB8EEE77B2A
:1091D00087EE006BBDEEC60B10EE103A5B4200EE60
:1091E000103AB8EEC00B88F051FF9FED087B30EECF
:1091F000070BB5EEC00BF1EE10FA03D59FED057B22
:1092000030EE070BBDEC028B38BD00BF00000060E4
:10921000FB21F93F00000060FB2119400B4630B5EF
:109220002DED028B8C6885B0D0E90251D868FFF72C
:1092300035FF08EE100A6019641B00EBD070401077
:10924000FFF7E0FEB8EEC86A9FED095A07EE904AB4
:1092500026EE056AF8EEE75AB7EEC66A26EE006B10
:1092600025EE850AF7EEC60B05B0BDEC028B30BDCE
:109270008262363CF0B50D4606462DED028B8C68B9
:1092800089B0D0E90271E868FFF708FF08EE100A1C
:10929000E019E41B00EBD0704010FFF7B3FEB8EE0E
:1092A000C86ADFED0F4A736826EE246A6A689FED8C
:1092B0000D1A9B1AB7EEC66A07EE903A26EE006BBF
:1092C000B8EEE75A07EE904AF8EEE75AF7EEC60B0B
:1092D00025EE011A25EEA40A09B0BDEC028BF0BD03
:1092E0008262363C0AD7233C0B4630B52DED028B0B
:1092F0008C6889B0D0E90251D868FFF7CFFE08EE3C
:10930000100A6019641B00EBD0704010FFF77AFE62
:1093100007EE904AB0EE401BB8EEE76BB8EEC87BA4
:109320009FED050B27EE007B26EE000B27EE011BC1
:1093300009B0BDEC028B30BD0000004050CC863F30
:1093400084B004B0FFF7D0BF10B52DED048B846856
:109350000B468A68111B224409EE101AC168D868AE
:1093600002EBD272FFF79AFE08EE100A5010B8EE28
:10937000C99BB8EEC88BFFF745FE28EE000B20EE28
:10938000000BA9EE090B88F0B1FE9FED037BBDEC4D
:10939000048B20EE070B10BD0000004050CC863F30
:1093A000094B984206DDC0F1D64000F5930000F568
:1093B000A4407047054B9842BEBFC0F1144000F571
:1093C000360000F53850704700E9A43500175BCA35
:1093D000F8B52DED048B9FED149BB0EE418B076823
:1093E00006460D4620EE090B28EE098BFDEEC07BEC
:1093F00017EE904A04EBD47007EB6000FFF702FE13
:1094000088EE007B3819FFF7CBFF306051EC170B6B
:10941000F7F7DCFA2B68C01841EBE371FFF71EFE8B
:109420002860BDEC048BF8BD00000040407556403C
:1094300000F10C010830FFF7CBBF00000148FFF737
:10944000EFBC00BFE06600300121884238BF08460B
:1094500085F07EBEFFF7F8BF08B185F07DBE70478E
:10946000FFF7FABF00214FF0FF33002210B543632E
:10947000044600F14003016041608160C16080F8F2
:10948000291000F50C70D9707C3343F8742C43F824
:10949000702C43F86C2C43F8682C43F8642C43F888
:1094A000602C43F85C2C43F8582C43F8542C43F8B8
:1094B000402C43F83C2C43F8382C43F8342C43F828
:1094C000302C43F82C2C43F8282C43F8242C43F858
:1094D000202C43F8102C43F80C2C43F8082C98420D
:1094E000D1D1214604F5177007F0C2FC044B1A686D
:1094F00022B9044920461C6037F0ACFC204610BD60
:10950000F0660030A4DD0B0873B5D0F84032044695
:109510000191994213D0D0F84432994218D0D0F832
:1095200048328B4216D102200AE0D4F8383253B3C5
:10953000D4F83C324BB34FF0030002B070BD0020B2
:1095400094F826308342F8D8431C84F82630F4E798
:109550000120F5E7D0F83462002EE6D194F84523D7
:109560003546B6009AB1A319C3F83412A319019A6B
:109570002846C3F8402294F82630AB429CBF6B1CAF
:1095800084F82630D9E70126E8E70226E6E704F565
:109590000D7001A9304438F04BFBE7E738B50446BD
:1095A0000D4638F0BBFA291D201D38F0B7FA05F139
:1095B000080104F1080038F08BFB05F1140104F1F7
:1095C000140038F085FB05F1200104F1200038F08B
:1095D0007FFB05F12C0104F12C0038F033FA05F182
:1095E000300104F1300038F03BFB05F13C0104F19F
:1095F0003C0038F06DFBAB6BA3636B6B636338BDF2
:109600002DE9F04300F14007A1B0002300250646F4
:1096100000F51078B9468DF807500393049305932D
:1096200006930793089309930A930B93109311934E
:1096300012931393149315931693179318931C93E3
:109640001D931E9358F8043BF3B1326F934222D01E
:10965000D6F8EC20934220D0D6F86821934213D15B
:109660000221EBB299420FD0C1EB411101A809EBE5
:1096700081042146FFF792FF39462046FFF78EFF0F
:1096800001A93846FFF78AFF01357C37032DD9D170
:1096900021B0BDE8F0830021E3E70121E1E700000C
:1096A0002DE9F04706460F461546804604464FF022
:1096B000000A39463046FFF727FFA26F5FFA8AF9A2
:1096C000BA420ED1C3B2022B0BD87C22012002FB7E
:1096D0000A6686F8420086F8433085F80090BDE8B7
:1096E000F0870AF1010A7C34BAF1030FE1D10024BA
:1096F00039463046FFF708FFD8F870205FFA84F942
:1097000012B9C3B2022B22D9013408F17C08032C10
:10971000EED100244FF07C0906F1420A394630466A
:10972000FFF7F2FE034609FB04F05FFA84F81AF82B
:10973000002012B9DBB2022B12D90134032CEDD177
:1097400096F82720042A14D918485FF0FDF97C20E8
:1097500000FB0464012084F8433084F84200BCE735
:109760000644012086F8433086F8420085F80080E0
:10977000B5E706F54470002150F8043BCCB2BB427B
:1097800008D1A24202D8631C86F8273003342C701B
:109790000020A4E733B9511CC43286F8271046F8DC
:1097A0002270F3E701310529E6D1F1E7E0DB0B0890
:1097B000C9B200EB8101D1F8403253B1426F9342FC
:1097C0000AD0D0F8F020934208D0D0F86C21934210
:1097D00006D04FF00300704700207047012070470B
:1097E0000220704759B190F82430032B07D05A1C3F
:1097F000063380F8242040F8231001207047002011
:10980000704700002DE9F8430F469146044600F5E5
:10981000BA7894F8425035B97C344445F9D10025E2
:109820002846BDE8F88300234A46394601200DF05A
:1098300051FA06460021206F0DF05CFA8642EBD10A
:10984000EEE700002DE9F043044685B000F5107600
:1098500000257C27DFF87080B14656F80C3CE9B251
:109860000436D9F80020934219D1C3B12046FFF73E
:109870009FFFC0B207FB004090F842307BB903A9BC
:10988000A9F10C00039338F0D3F946F0A5FA56F885
:10989000043C4246012100932B463FF0ADF90135CF
:1098A000032DD9D104F1700504F5F274296821B9AA
:1098B000AB6813B1284636F091FC7C35A542F5D152
:1098C00005B0BDE8F08300BFFCDB0B0838B50446EB
:1098D0001546FFF76DFFC0B2022808D87C23294641
:1098E00003FB0040BDE83840543038F0E1B938BDE2
:1098F00038B504461546FFF75BFFC0B2022808D80A
:109900007C23294603FB0040BDE83840603038F036
:10991000CFB938BD37B50D4604468DED010AFFF7C6
:1099200047FF022D07D8C0B27C2301A903FB0040EA
:109930006C3038F06FF803B030BD000038B5054624
:10994000FFF736FFC4B2022C13D8C4EB44144035E1
:109950000021A40004F10800284436F03FFC04F183
:10996000340104F1300029442844BDE8384038F07F
:109970005FB938BD70B505460E461446FFF718FFAF
:10998000C3B2022B0DD87C2000FB035394E80700E0
:10999000483383E8070031462846BDE87040FFF7AA
:1099A000CDBF70BD37B504461546FFF701FFC0B205
:1099B000022809D87C230DF107018DF8075003FB1D
:1099C0000040443038F0AAF803B030BD10B504466A
:1099D0000021FFF7B3FF01212046FFF7AFFF20462C
:1099E0000221BDE81040FFF7A9BF00001FB590F9A4
:1099F0003030044623B390F925300BB36846FFF7A7
:109A000013FAFBF757FD6946FBF71AFBC0B1DDED12
:109A1000037A01239FED0B0AF8EEE70ADDED027AE7
:109A200084F84133F8EEE77AC0EE800A87EE800AC8
:109A300007F064FCDFED047A20EE270A84ED0B0AC0
:109A400004B010BD8096184B35FA8E3C024690F952
:109A5000250058B192F8440340B1114491F9300205
:109A600020B192F92800033818BF01207047000088
:109A700038B590F8263005465BB100242346E1B2A4
:109A80002846FFF7E3FF08B10133DBB20134032CB2
:109A9000F5D1184638BD000090ED0B0A7047000064
:109AA00038B50C46D1ED066A11460546FFF780FE33
:109AB00094ED076AC3B27C20D4ED087AB7EE007A41
:109AC00000FB0353D3ED270AA6EEE67AD3ED265A20
:109AD00026EE600A93ED255A67EEA00AA5EEA70AC6
:109AE000F0EE607AE5EE867AB1EE400A67EEE60ABD
:109AF000E5EE070A88F08CFB40F61C009FED081A83
:109B0000DFED080A11F08EF9D5ED0B7A30EE270A59
:109B1000B7EEC00A11F06EF9B7EEC00B38BD00BF4A
:109B2000DB0F4940DB0F49C02DE9F04190F82630AA
:109B300004460D468B4202D20020BDE8F081FFF7BB
:109B400037FE04F14006C0B2C0EB401006EB8000C7
:109B5000083014F039FBB0EEC00ADFED147AB4EE31
:109B6000E70AF1EE10FAE7D429462046FFF720FE77
:109B7000C5B27C2000FB05477B6F002BDCD0032D9A
:109B8000DAD000FB0560D7F87080303037F036FA55
:109B9000D7E91C32934201D1984505D07C2000FBC7
:109BA0000544C4F87080C7E70120C6E70000003410
:109BB0002DE9F74F04460E46174600F5107A4FF090
:109BC000000B5AF8049B5FFA8BF8B9F1000F26D00E
:109BD00041462046FFF73AFF08B341462046FFF7CB
:109BE000E7FD7C23C0B203FB004090F842505DB912
:109BF00008F101031B4A39463046DBB25EF028F813
:109C0000284603B0BDE8F08F5AF8102C914506D0D5
:109C1000154A3946304600255EF01AF8F0E70BF198
:109C2000010BBBF1030FCCD14FF000085FFA88F1B4
:109C300094F826308B420DD920460191FFF774FF2E
:109C4000054620B901992046FFF700FF20B908F129
:109C50000108EBE70125D3E7044A394630465DF0B9
:109C6000F7FFCDE724DC0B0839DC0B085EDC0B08C2
:109C70002DE9F04106464FF000082DED068B82B02D
:109C800090F84613FFF794FD06F14007C5B27C201B
:109C90009FED35AA00FB05759FED2F8B9FED309B47
:109CA00054355FFA88F396F826209A4251D919461E
:109CB0003046FFF7CBFE10B908F10108F1E719466D
:109CC0003046FFF775FDC4B27C2000FB0474D4ED70
:109CD000157A5434F0EEE77AF4EECA7AF1EE10FA1F
:109CE0000ED5D4ED017AF0EEE77AF4EECA7AF1EE11
:109CF00010FA05D5002002B0BDEC068BBDE8F0815E
:109D00002946204614F084FAB7EEC00AB4EEC80B18
:109D1000F1EE10FAEEDC2946204613F02BFDB7EEEB
:109D2000C00AB4EEC90BF1EE10FAE3DC2146284676
:109D300013F05EFC68468DED000ACDED010A13F0CC
:109D4000FDFCDFED0A7AB4EEE70AF1EE10FAB3DDBE
:109D5000D0E70120CFE700BF00000051FB21F93F11
:109D60000000003652C1F03F0000003400004843BC
:109D7000022910B5044608D8FFF71AFD7C23C0B2AB
:109D800003FB004494F8410010BD0020FCE70000F4
:109D900013B590F8461304460191FFF7E9FF30B17F
:109DA0000199204602B0BDE81040FFF74FBE02B057
:109DB00010BD0000F7B590F925500446002D73D072
:109DC00090F84453002D6FD090F84613FFF7D0FF62
:109DD00094F84133064613B92046FFF707FE0025E5
:109DE00094F82420EBB29A4207D90633013554F88F
:109DF000230003689B689847F2E75EF0D3FE0027D4
:109E0000224604F5BA7140F2F315D2F8A0307C3244
:109E1000C31AAB428CBF0023012302F83B3C9142A2
:109E200047EA0307F1D194F92830032B07D194F8BE
:109E30004033002B3BD0D4F83C03002849D167B114
:109E4000636B013309D03BF043FD616B3BF064FB76
:109E500018B13BF03DFD3AF015FC94F93032002B7F
:109E60003AD194F93132CBBB94F9323213B1022397
:109E700084F8463394F846132046FFF779FF86426C
:109E8000054611D03BF024FD4FF6FF713BF044FB3B
:109E900050B1002D14BF0022042201923BF018FDA6
:109EA000019A03213BF0CAFA284603B0F0BD012312
:109EB000042084F84033FFF7C7FA054610B1214665
:109EC00007F06CF894F92830C4F83C53032BB2D057
:109ED000B5E707F071F8B2E70023C9E70123C7E748
:109EE00038B590F925300446D3B190F84453BDB14C
:109EF000FFF75EFCC0B2022812D87C239FED0A7ADD
:109F000003FB0044D4ED1B7AF4EEC77AF1EE10FAAD
:109F100006D4B7EE087AF4EEC77AF1EE10FA00DD57
:109F20000025284638BD00BFABAA2A3F70B5D0F83F
:109F30000C5304460E4615F400350DD190F8443309
:109F40005BB90A78072A07D8012303FA02F290F8CE
:109F50004333134380F8433370BD94F82420EBB2AD
:109F60009A42F9D906333146013554F82300036883
:109F7000DB689847F1E7000038B5054670242B5997
:109F80001BB10021281936F029F97C34B4F5F27F91
:109F9000F5D138BD014B1868704700BFF06600303E
:109FA000504B2DE9F04F1F6804468BB000257868B0
:109FB0004FF00109DFF830A103689B68984780469D
:109FC00009FA05F313EA080F15D10135202DF7D151
:109FD000786800254FF00109DFF80CA10368DB6801
:109FE0009847804609FA05F313EA080F3FD1013577
:109FF000202DF7D129E0D4F80C3313F4805B20D165
:10A00000E9B20D2220460591FFF7FCFB05990646B3
:10A01000F0B1CDE907BB089B0022012109A8CDE9D9
:10A02000082304F059FE01462046FFF7DBFB09A890
:10A03000FDF79EFF08A8FDF79BFF16B107A8FDF7E7
:10A0400097FF94F82730052BBFD10BB0BDE8F08FF8
:10A05000786804220368CDF800A0CDE901620A46C1
:10A06000D3F800B001460D2308A8D847D3E7D4F8A9
:10A070000C3313F4805B20D1E9B20D222046059108
:10A08000FFF7C0FB05990646E0B1CDE907BB00220A
:10A09000089B09A81146CDE9082304F01DFE0146DE
:10A0A0002046FFF79FFB09A8FDF762FF08A8FDF710
:10A0B0005FFF16B107A8FDF75BFF94F82730052B6B
:10A0C00095D1C2E7786804220368CDF800A0CDE9F5
:10A0D00001620A46D3F800B001460D2308A8D8470C
:10A0E000D5E700BFB4250030801A0600B34B2DE938
:10A0F000F04FD3F8008004468DB00025D8F8040056
:10A100004FF0010903689B689847074609FA05F371
:10A110003B4240F092820135202DF7D1D8F804005F
:10A1200000254FF001090368DB689847074609FAE4
:10A1300005F33B4240F0C3820135202DF7D1D8F81A
:10A14000040000254FF0010903689B689847074603
:10A1500009FA05F33B4240F0F1820135202DF7D199
:10A16000D8F8040000254FF0010903689B68984760
:10A17000074609FA05F33B4240F01C830135202DC8
:10A18000F7D1D8F804000025DFF83CB203689B68DB
:10A19000984704900123049AAB40134240F0468351
:10A1A0000135202DF6D1D8F804000025DFF818B2CB
:10A1B0000368DB68984704900123049AAB4013427C
:10A1C00040F005840135202DF6D1D8F80400002593
:10A1D0004FF001090368DB689847074609FA05F361
:10A1E0003B4240F0BF840135202DF7D1D8F8040060
:10A1F00000254FF001090368DB689847074609FA14
:10A2000005F33B4240F0ED840135202DF7D1D8F81D
:10A21000040000254FF0010903689B689847074632
:10A2200009FA05F33B4240F01B850135202DF7D19B
:10A23000D8F8040000254FF0010903689B6898478F
:10A24000074609FA05F33B4240F04A850135202DC7
:10A25000F7D1D8F8040000254FF0010903689B6886
:10A260009847074609FA05F33B4240F079850135E6
:10A27000202DF7D1D8F8040000254FF0010903681C
:10A28000DB689847074609FA05F33B4240F0A4858E
:10A290000135202DF7D14A4B08AF04250893D8F893
:10A2A0000400002603689B68984783460123B34057
:10A2B00013EA0B0F40F0CB850136202EF6D1D8F8EB
:10A2C000040000260368DB68984783460123B340F7
:10A2D00013EA0B0F40F001860136202EF6D1013D26
:10A2E000013715F0FF05DAD1D8F804004FF0010965
:10A2F00003689B689847074609FA05F33B4240F01C
:10A3000030860135202DF7D1D8F8040000254FF014
:10A3100001090368DB689847074609FA05F33B42E1
:10A3200040F05B860135202DF7D1D8F804000025D8
:10A330004FF0010903689B689847074609FA05F33F
:10A340003B4240F086860135202DF7D1D8F8040035
:10A3500000254FF001090368DB689847074609FAB2
:10A3600005F33B4240F0B1860135202DF7D1154B66
:10A3700000250793D8F8040003689B689847834634
:10A380000123AB4013EA0B0F42D000275FFA85F997
:10A39000D4F80C3313F4803A32D107AB4946204647
:10A3A000DB5D1A460493FFF72DFA049B064600284E
:10A3B00000F0C786CDE908AA08E000BFB425003048
:10A3C0000C0D0E0F20212223801A0600099B00226B
:10A3D00001210BA80B93CDE9092204F06FFF014680
:10A3E0002046FFF7FFF90BA8FDF778FD0AA8FDF757
:10A3F00075FD09A8FDF7BCFD16B108A8FDF7B8FD6D
:10A4000094F82730052B00F048810137042FBFD185
:10A410000135202DB4D1D8F8040000250368DB688D
:10A42000984783460123AB4013EA0B0F38D000272F
:10A430005FFA85F9D4F80C3313F4803A28D107ABCE
:10A4400049462046DB5D1A460493FFF7DBF9049B7F
:10A450000646002800F08486CDE908AA0022099B60
:10A460000BA811460B93CDE9092204F027FF014602
:10A470002046FFF7B7F90BA8FDF730FD0AA8FDF756
:10A480002DFD09A8FDF774FD16B108A8FDF770FDB4
:10A4900094F82730052B00F000810137042FC9D133
:10A4A0000135202DBED1D8F80400002603689B6832
:10A4B000984782460123B34013EA0A0F31D0102592
:10A4C0005FFA86F9D4F80C3313F0080B20D12A4632
:10A4D00049462046FFF796F90746002800F04F86C8
:10A4E000CDE909BB0A9B002201210BA8CDE90A2373
:10A4F00001F04AFC01462046FFF774F90BA8FDF76E
:10A5000037FD0AA8FDF734FD17B109A8FDF730FDA6
:10A5100094F82730052B00F0C0800135EDB2142DE2
:10A52000D0D10136202EC5D1D8F80400002603680A
:10A530009B68984782460123B34013EA0A0F34D040
:10A5400014255FFA86F9D4F80C3313F4001B24D1D8
:10A550002A4649462046FFF755F90746002800F0ED
:10A560001E86CDE908BB099B002201210BA80B9395
:10A57000CDE9092202F01AF801462046FFF732F928
:10A580000BA8FDF7ABFC0AA8FDF7A8FC09A8FDF78E
:10A59000EFFC17B108A8FDF7EBFC94F82730052B6A
:10A5A0007BD00135EDB2182DCDD10136202EC2D190
:10A5B000D8F8040000260368DB6898478246012328
:10A5C000B34013EA0A0F34D014255FFA86F9D4F8A1
:10A5D0000C3313F4001B24D12A4649462046FFF7CA
:10A5E00011F90746002800F0ED85CDE908BB0022EF
:10A5F000099B0BA811460B93CDE9092201F0D6FF68
:10A6000001462046FFF7EEF80BA8FDF767FC0AA805
:10A61000FDF764FC09A8FDF7ABFC17B108A8FDF72E
:10A62000A7FC94F82730052B37D00135EDB2182D53
:10A63000CDD10136202EC2D12FE0D4F80C3313F047
:10A64000010A25D15FFA85FB1E2220465946FFF7F5
:10A65000D9F8064620B3CDE908AA099A00230121BA
:10A660000BA80B920822CDE9093303F0C7FA014683
:10A670002046FFF7B7F80BA8FDF730FC0AA8FDF756
:10A680002DFC09A8FDF774FC16B108A8FDF770FCB5
:10A6900094F82730052B7FF43EAD0DB0BDE8F08F68
:10A6A000D8F8041004220B68CDE90102B84A09A8C1
:10A6B00000925A46D3F800A01E23D047CDE7D4F825
:10A6C0000C3313F0010A24D15FFA85FB1E222046C9
:10A6D0005946FFF797F8064608B3CDE908AA099B43
:10A6E000002106220BA80B93CDE9091103F086FA8D
:10A6F00001462046FFF776F80BA8FDF7EFFB0AA806
:10A70000FDF7ECFB09A8FDF733FC16B108A8FDF72F
:10A710002FFC94F82730052B7FF40EADBDE7D8F859
:10A72000041004220B68CDE90102994A09A800929D
:10A730005A46D3F800A01E23D047D0E7D4F80C33F4
:10A7400013F4805A21D15FFA85FB0D222046594629
:10A75000FFF758F80646F0B1CDE909AA0A9B002296
:10A7600001210BA8CDE90A23082204F0B5FA01461D
:10A770002046FFF737F80BA8FDF7FAFB0AA8FDF70C
:10A78000F7FB16B109A8FDF7F3FB94F82730052B6A
:10A790007FF4E3AC81E7D8F8041004220B68CDE91C
:10A7A00001027B4A0AA800925A46D3F800A00D2362
:10A7B000D047D3E7D4F80C3313F4801A21D15FFAD1
:10A7C00085FB2C2220465946FFF71CF80646F0B1BF
:10A7D000CDE909AA0A9B002201210BA8CDE90A2391
:10A7E000082204F0A7FB01462046FEF7FBFF0BA85A
:10A7F000FDF7BEFB0AA8FDF7BBFB16B109A8FDF7E4
:10A80000B7FB94F82730052B7FF4B8AC45E7D8F8B0
:10A81000041004220B68CDE901025D4A0AA80092E7
:10A820005A46D3F800A02C23D047D3E7D4F80C33F2
:10A8300013F480773FD15FFA85F90C222046494610
:10A84000FEF7E0FF0646002800F08480CDE9067799
:10A85000079B4FF0000A692249462046CDF81CA00C
:10A860000A93FEF7CFFF0746002800F08180CDE96C
:10A8700008AA099B00220BA90AA8099201220B939E
:10A880001A2301F009F801462046FEF7ABFF0BA89A
:10A89000FDF76EFB09A8FDF76BFB17B108A8FDF7E4
:10A8A00067FB0AA8FDF764FB07A8FDF761FB16B17B
:10A8B00006A8FDF75DFB94F82730052B3FF4EDAEBD
:10A8C000D4F80C3313F480777FF46AAC5FFA85F91F
:10A8D0000C2220464946FEF795FF0646002859D02F
:10A8E000CDE90677079B4FF0000A682249462046CB
:10A8F000CDF81CA00A93FEF785FF0746002857D025
:10A90000CDE908AA099B00220BA90AA809920122F5
:10A910000B931A2300F0C0FF01462046FEF762FFAA
:10A920000BA8FDF725FB09A8FDF722FB17B108A826
:10A93000FDF71EFB0AA8FDF71BFB07A8FDF718FB98
:10A9400016B106A8FDF714FB94F82730052B7FF409
:10A9500027ACA2E6D8F8041004220B68CDF800B0AA
:10A96000CDE901024A461F6807A80C23B8476FE7E4
:10A97000D8F8041004220B68CDF800B0CDE901022C
:10A980004A46D3F800A009A86923D04771E700BF61
:10A99000801A0600D8F8041004220B68CDF800B025
:10A9A000CDE901024A461F6807A80C23B84799E77A
:10A9B000D8F8041004220B68CDF800B0CDE90102EC
:10A9C0004A46D3F800A009A86823D0479AE7D4F8EC
:10A9D0000C3313F480773DD15FFA85F90C222046C1
:10A9E0004946FEF70FFF0646002800F08180CDE9BA
:10A9F0000677079B4FF0000A692249462046CDF8AA
:10AA00001CA00A93FEF7FEFE074600287ED0CDE983
:10AA100008AA099B00220BA90AA80B931A230992E2
:10AA200000F03AFF01462046FEF7DCFE0BA8FDF7DA
:10AA30009FFA09A8FDF79CFA17B108A8FDF798FA44
:10AA40000AA8FDF795FA07A8FDF792FA16B106A82D
:10AA5000FDF78EFA94F82730052B3FF41EAED4F89C
:10AA60000C3313F480777FF4ADAB5FFA85F90C22D9
:10AA700020464946FEF7C6FE0646002855D0CDE9D9
:10AA80000677079B4FF0000A682249462046CDF81A
:10AA90001CA00A93FEF7B6FE0746002853D0CDE966
:10AAA00008AA099B00220BA90AA80B931A23099252
:10AAB00000F0F2FE01462046FEF794FE0BA8FDF7DB
:10AAC00057FA09A8FDF754FA17B108A8FDF750FA8C
:10AAD0000AA8FDF74DFA07A8FDF74AFA16B106A82D
:10AAE000FDF746FA94F82730052B7FF46BABD4E5DD
:10AAF000D8F8041004220B68CDF800B0CDE90102AB
:10AB00004A461F6807A80C23B84772E7D8F8041014
:10AB100004220B68CDF800B0CDE901024A46D3F813
:10AB200000A009A86923D04773E7D8F804100422CD
:10AB30000B68CDF800B0CDE901024A461F6807A8AE
:10AB40000C23B8479DE7D8F8041004220B68CDF811
:10AB500000B0CDE901024A46D3F800A009A8682355
:10AB6000D0479EE7D4F80C3313F0200A24D15FFAC3
:10AB700085FB1C2220465946FEF744FE064608B3D4
:10AB8000CDE908AA0022099B0BA811460B93CDE939
:10AB9000092203F031FC01462046FEF723FE0BA8F4
:10ABA000FDF79CF90AA8FDF799F909A8FDF7E0F966
:10ABB00016B108A8FDF7DCF994F82730052B7FF4CF
:10ABC00012AB6AE5D8F8041004220B68CDE9010243
:10ABD000B84A09A800925A46D3F800A01C23D047CF
:10ABE000D0E7D4F80C3313F0200A24D15FFA85FBA8
:10ABF0001E2220465946FEF705FE064608B3CDE95B
:10AC000008AA0022099B0BA811460B93CDE9092243
:10AC100003F0F2FB01462046FEF7E4FD0BA8FDF72A
:10AC20005DF90AA8FDF75AF909A8FDF7A1F916B1CF
:10AC300008A8FDF79DF994F82730052B7FF4E4AAC6
:10AC40002BE5D8F8041004220B68CDE90102994ADB
:10AC500009A800925A46D3F800A01E23D047D0E797
:10AC6000D4F80C3313F0200A25D15FFA85FB1C229F
:10AC700020465946FEF7C6FD064610B3CDE908AAA0
:10AC8000099A002301210BA80B920222CDE9093376
:10AC900003F0B2FB01462046FEF7A4FD0BA8FDF72A
:10ACA0001DF90AA8FDF71AF909A8FDF761F916B10F
:10ACB00008A8FDF75DF994F82730052B7FF4B5AAB5
:10ACC000EBE4D8F8041004220B68CDE90102794ABC
:10ACD00009A800925A46D3F800A01C23D047CFE71A
:10ACE000D4F80C3313F0200A25D15FFA85FB1E221D
:10ACF00020465946FEF786FD064610B3CDE908AA60
:10AD0000099A002301210BA80B920222CDE90933F5
:10AD100003F072FB01462046FEF764FD0BA8FDF729
:10AD2000DDF80AA8FDF7DAF809A8FDF721F916B150
:10AD300008A8FDF71DF994F82730052B7FF486AAA3
:10AD4000ABE4D8F8041004220B68CDE90102594A9B
:10AD500009A800925A46D3F800A01E23D047CFE797
:10AD6000D4F80C3313F0400A21D15FFA85FB0C2292
:10AD700020465946FEF746FD0646F0B1CDE909AA40
:10AD80000A9B002201210BA8CDE90A23062200F02C
:10AD900049FD01462046FEF725FD0BA8FDF7E8F822
:10ADA0000AA8FDF7E5F816B109A8FDF7E1F894F84F
:10ADB0002730052B7FF45BAA6FE4D8F80410042237
:10ADC0000B68CDE901023B4A0AA800925A46D3F823
:10ADD00000A00C23D047D3E7D4F80C3313F0400A7B
:10ADE00020D15FFA85FB0C2220465946FEF70AFD6A
:10ADF0000646E8B1CDE909AA00220A9B0BA8114634
:10AE0000CDE90A2300F00EFD01462046FEF7EAFCDC
:10AE10000BA8FDF7ADF80AA8FDF7AAF816B109A826
:10AE2000FDF7A6F894F82730052B7FF431AA34E417
:10AE3000D8F8041004220B68CDE901021D4A0AA8C3
:10AE400000925A46D3F800A00C23D047D4E7D4F898
:10AE50000C3313F0800A26D13B78F1B220461A4613
:10AE6000CDE90413FEF7CEFC8146DDE9041318B3E7
:10AE7000CDE909AA0A9B002201210BA8CDE90A23EA
:10AE80000C2203F087F901462046FEF7ABFC0BA825
:10AE9000FDF76EF80AA8FDF76BF8B9F1000F02D0C4
:10AEA00009A8FDF765F894F82730052B7FF404AA6C
:10AEB000FFF7F3BB801A0600D8F804004FF0040C2B
:10AEC000BF4AD0F800E000920A4601460AA8CDE940
:10AED000019CDEF800A0D047CCE7D4F80C3313F087
:10AEE000800A26D13B78F1B220461A46CDE90413F8
:10AEF000FEF788FC8146DDE9041308B3CDE909AA11
:10AF00000A9B002200210BA8CDE90A230C2203F0A2
:10AF100041F901462046FEF765FC0BA8FDF728F82D
:10AF20000AA8FDF725F8B9F1000F02D009A8FDF72E
:10AF30001FF894F82730052B7FF4CEA9FFF7ADBB9F
:10AF4000D8F804004FF0040C9D4AD0F800E00092BD
:10AF50000A4601460AA8CDE9019CDEF800A0D047C8
:10AF6000CEE7D4F80C3313F4004A20D15FFA85FB06
:10AF70000C2220465946FEF745FC0646F0B1CDE9C5
:10AF800009AA0A9B002201210BA8CDE90A2302F09D
:10AF900077FF01462046FEF725FC0BA8FCF7E8FFEB
:10AFA0000AA8FCF7E5FF16B109A8FCF7E1FF94F841
:10AFB0002730052B7FF4A5A9FFF76FBBD8F8041045
:10AFC00004220B68CDE901027D4A0AA800925A4684
:10AFD000D3F800A00C23D047D3E7D4F80C3313F4F4
:10AFE000004A20D15FFA85FB0C2220465946FEF725
:10AFF00009FC0646F0B1CDE909AA00220A9B0BA87C
:10B000001146CDE90A2302F03BFF01462046FEF738
:10B01000E9FB0BA8FCF7ACFF0AA8FCF7A9FF16B1E7
:10B0200009A8FCF7A5FF94F82730052B7FF47AA92F
:10B03000FFF733BBD8F8041004220B68CDE90102F6
:10B040005F4A0AA800925A46D3F800A00C23D047C2
:10B05000D3E7D4F80C3313F4007A20D15FFA85FBE0
:10B06000302220465946FEF7CDFB0646F0B1CDE929
:10B0700009AA0A9B002201210BA8CDE90A2303F0AB
:10B0800087FC01462046FEF7ADFB0BA8FCF770FFDE
:10B090000AA8FCF76DFF16B109A8FCF769FF94F840
:10B0A0002730052B7FF44FA9FFF7F7BAD8F8041023
:10B0B00004220B68CDE90102414A0AA800925A46CF
:10B0C000D3F800A03023D047D3E7D4F80C3313F4DF
:10B0D000007A20D15FFA85FB302220465946FEF7E0
:10B0E00091FB0646F0B1CDE909AA00220A9B0BA804
:10B0F0001146CDE90A2303F04BFC01462046FEF73A
:10B1000071FB0BA8FCF734FF0AA8FCF731FF16B15E
:10B1100009A8FCF72DFF94F82730052B7FF424A90C
:10B12000FFF7BBBAD8F8041004220B68CDE901027E
:10B13000234A0AA800925A46D3F800A03023D047E9
:10B14000D3E7D8F8041004200A68CDE901601C4850
:10B15000009009A8D2F800A04A46D047FFF736B9B8
:10B16000D8F8041004200A68CDE901601448009062
:10B1700009A8D2F800A04A46D047FFF76FB9D8F81F
:10B18000041004220B68CDE901020D4A0AA80092BE
:10B190004A46D3F800B02B46D847FFF7A3B9D8F8F2
:10B1A000041004220B68CDE90102054A09A80092A7
:10B1B0004A46D3F800B02B46D847FFF7D4B900BFB2
:10B1C000801A0600D8F8041004220B68CDE90102A9
:10B1D000044A09A800924A46D3F800B02B46D84743
:10B1E000FFF705BA801A060073B50446FEF77EFF26
:10B1F00094F82730052B35D0002594F84333E9B275
:10B20000EB40DA0719D40135082DF6D194F8273030
:10B21000052B27D02046FEF7C3FE94F8243013B147
:10B2200094F82630F3B9104B10491B6898690368ED
:10B230001B6802B0BDE870401847D4F80C339B037C
:10B240000CD42C200191FEF7FFF8064610B10199AD
:10B2500003F016FC31462046FEF7C4FA94F8273076
:10B26000052BD0D102B070BDB425003078DC0B08BE
:10B270002DE9F04F90F9253089B00446002B00F0FD
:10B280000481012300F50D75024600F5107180F868
:10B2900045332E462B46106F002859D0002384F8E2
:10B2A000453394F94430642B5BD094F9C030642B5F
:10B2B00000F08D8094F93C31642B00F08A80D4F842
:10B2C00034722FBB01A9204634F06CFF00B30C236D
:10B2D0000697694604A80593012304978DF8183052
:10B2E0006F4B8DF800700793BDF80430ADF8103047
:10B2F00035F0D6F89DF9001051B1022908DC38B1BB
:10B30000C9B27C23284603FB0141703136F0A8FC0A
:10B3100094F845B3BBF1000F5DD0236F0021A36704
:10B32000D4F8EC30C4F8F430D4F86831C4F8703193
:10B3300094F8273003F1C40204EB8202042B7CD87A
:10B3400052F8040B01331061DBB242F8041CF5E73C
:10B3500053F8040B0028A1D18B4202F17C029AD150
:10B360009FE70020662304A98DF810307C2303FB9F
:10B370000040443036F0B8FB04A9204634F012FFF8
:10B3800000289CD004238DF818300023CDE9013328
:10B39000039331230593694604A835F081F8059B92
:10B3A00028B108AA009902EB830242F8E01C01339D
:10B3B000332B0593EFD95BF08FF89DED031ADDED8C
:10B3C000020A66219DED010A5BF044F877E701204F
:10B3D000C8E70220C6E70127A94655F8043B23B178
:10B3E000AB600137042FF7D197E7AA46B8465FFA5A
:10B3F00088F3022BF5D8DAF8002055F8043C9A427D
:10B4000005D104A95046CDF810B036F029FC5AF801
:10B41000043B08F101020BB99046E8E704A906EBEA
:10B4200088000193CDF810B036F01AFC019B01A9F9
:10B430004846AB6036F014FCD3E794F8453313B9B3
:10B440002046FEF7DDF894F826300BB3154B642147
:10B450001B68986A03685B6898472046FEF7AAFC59
:10B4600094F8423003B9236794F8BE300BB9C4F89E
:10B47000EC3094F83A310BB9C4F86831FAF71AF89D
:10B48000FAF7A2F80123A4F8443309B0BDE8F08F1D
:10B490002046FFF7A9FE94F82630002BE0D0D5E730
:10B4A000149E0C08B425003070470000012070473E
:10B4B000012070474368986870470000054B10B53D
:10B4C00004460360806A10B103685B6898472046B1
:10B4D00010BD00BF38E10B08406803685B6A18477D
:10B4E00033B46C46406884E80C0003689D6A94E8B5
:10B4F0000C00AC4602B030BC6047000010B50446FA
:10B50000FFF7DCFF2046FDF7A7FF204610BD000037
:10B5100040680BF011BB0000012340680BF00CBB2E
:10B5200040680BF0E5BA00000A2240680BF08ABAC6
:10B5300040680BF09FBA000040680BF021BB000090
:10B5400090F82E2022B1002290F82D1001F06EB953
:10B550007047000073B5044605250026A06A0DF16A
:10B5600007028DF8076001210368DB68984778B10E
:10B570009DF807300C2B09D0102B05D0092B07D1D3
:10B5800084F8303002B070BD1523F9E71423F7E7D3
:10B59000013DE3D12846F5E710B4806A0822312145
:10B5A00003681C690123A4465DF8044B6047000052
:10B5B00010B4806A0122322103681C690023A4466A
:10B5C0005DF8044B60470000F0B50446806A85B022
:10B5D00003685B6998470546002800F08480A06AEC
:10B5E00003685B69984703689B689847A06A03688B
:10B5F0009B69984760B93D4B3D491B689869036852
:10B600001B6898472B6828460026DB68984767E048
:10B610002046FFF7CDFF0028F4D02046FFF79AFF21
:10B620000028EFD0A06A01210368DB6A9847204612
:10B63000FFF7B2FF30B92D4B2E491B68986903689C
:10B640001B68DEE7A06A0368DB69984730B9274BBF
:10B6500029491B68986903681B68D2E7A06A01271B
:10B6600094F8301084F82E7003685B6A9847A06ADB
:10B6700003689B6A984704F12D020146204601F0B9
:10B6800023F906460028BDD0A06A94F82D1003685F
:10B6900001919B6A984701990246204601F018F9EA
:10B6A00094F82C302BB13A4694F82D10204601F036
:10B6B00023F994F82F20204694F82D1001F03EF93C
:10B6C0002B682846DB689847A06A029442F2107102
:10B6D00003681D6A094B039304AB13E90C00A847E8
:10B6E000304605B0F0BD0646FAE700BFB42500308D
:10B6F000A4E00B08CAE00B08E9E00B08F5B7020864
:10B7000070B5002386B000250446806A6A468DF82D
:10B7100008501021059303930493CDE90055036865
:10B720009E680923B047A0B19DF8003013F00106D0
:10B7300015D194F831300133DBB2052B84F8313068
:10B7400007D12046FFF734FF2046FFF725FF84F896
:10B750003160A06A03681B6B984706B070BD9DF806
:10B76000083084F831501B07F3D4BDF901309FED48
:10B770001F6A06EE903ABDF90330F8EEE66A07EE6E
:10B78000103ABDF90530B8EEC77ACDED036AF0EE98
:10B79000E66A07EE903A8DED047AF4EEC66AF8EEAA
:10B7A000E77AF1EE10FACDED057A0DD5B0EEC77A55
:10B7B000B4EEC67AF1EE10FA06D5F0EEE77AF4EEC2
:10B7C000C67AF1EE10FAC4D49FED090A03A812F06C
:10B7D00053F9B2EE040A03A812F04EF90A2394F8C2
:10B7E0002D2003A9204601F00DF9B2E70000003436
:10B7F0009A99193EFFF784BF044B10B5044640F8F0
:10B80000043BFCF7B5FB204610BD00BF50E10B0820
:10B8100010B50446FFF7F0FF2046FDF71DFE204659
:10B8200010BD0000F7B503680F4616461BB900248B
:10B83000204603B0F0BD0024019304600820FDF70A
:10B8400003FE054620B1124B0360019B0194436047
:10B8500001A8FCF78DFB002DE9D03420FDF7F4FDA5
:10B8600004460028E3D000F0E1FE0A4BA562204622
:10B87000236084F82C7084F82F60FFF7A5FE05463E
:10B880000028D5D1236820462C465B689847CFE72F
:10B8900050E10B0838E10B082DE9F74F0468064624
:10B8A0000D4690469946002C6CD00B68002B49D071
:10B8B000236820465B6A984703689B689847012382
:10B8C000002128680DEB03020BF036F998B39DF8C0
:10B8D0000130EA2B2FD14FF0060ADFF8ECB000233D
:10B8E0008022062128680BF003F920B3DBF80070F2
:10B8F0000A21B86A03685B68984700230621286814
:10B900001A460BF0F5F8B0B1B86A0A2103685B6813
:10B9100098470123062128680DEB03020BF00CF970
:10B9200048B19DF8014014F040042FD00AF1FF3ACD
:10B930001AF0FF0AD3D1306803685B6A984703683E
:10B94000DB68984700241DE0022223460F21286867
:10B950000BF0CEF8B86A012103685B68984730683D
:10B9600003685B6A98470368DB68984733684A4610
:10B970003460414601A80193FFF754FF044601A833
:10B98000FCF7F6FA204603B0BDE8F08F22462346C6
:10B990000F2128680BF0ACF8B86A012103685B68D6
:10B9A00098470223214630680DEB03020BF0C4F8E0
:10B9B00004460028C8D0B869024903681B68984744
:10B9C000B9E700BF10E10B08B4250030002290F861
:10B9D0002C1000F02BBF000070B504468CB004267C
:10B9E000013E76B2731C4AD015236A465D21A06AD7
:10B9F0000BF0A2F80028F3D0152306AA5D21A06A57
:10BA00000BF09AF805460028EAD0152206A96846E8
:10BA100089F08CF90028E3D19DF800309DF81020C2
:10BA200084F82E309DF8073084F830309DF81430BB
:10BA300084F83A309DF8133084F83B309DF80F308D
:10BA400043EA02239DF80C20A3879DF8013084F877
:10BA50002F309DF8083084F83130039BC3F30F2357
:10BA600063869DF80B3043EA0223A386049BC3F34D
:10BA70000F23E386019BC3F30F23238707E0054BC6
:10BA8000002505491B68986903681B689847284684
:10BA90000CB070BDB425003084E10B082DE9FF41E6
:10BAA00004460023806A04258DF807300368DFF818
:10BAB00068815B6A984703689B689847A06A0A2177
:10BAC00003689B6C98470A220421A06A0AF0BAFF17
:10BAD000013D6DB26B1C32D000234B218222A06A43
:10BAE0000BF006F8D8F8006007460221B06A036838
:10BAF0005B689847002FEBD001234B21A06A1A46C0
:10BB00000AF0F6FF0746B06A022103685B689847AF
:10BB1000002FDDD001230DF107024021A06A0BF0B8
:10BB20000BF80028D4D09DF80720322A10D0002D21
:10BB3000CED1B069364903681D683223A847A06A90
:10BB4000002503685B6A98470368DB6898475BE0F9
:10BB50002046FFF741FF0028F1D001231722512191
:10BB6000A06A0AF0C5FF0028E9D052220123A06A8A
:10BB700011460AF0BDFF0028E1D0012338224C21F4
:10BB8000A06A0AF0B5FF0028D9D0A06A03685B6AF2
:10BB900098470368DB6898470521A06A0AF06AFFA6
:10BBA000A36A04F12C022046996800F08DFE054638
:10BBB00050B3A36A204694F82C109A6800F088FECF
:10BBC00094F8442094F82C10204600F0B7FE94F826
:10BBD00045302BB1012294F82C10204600F08CFE49
:10BBE000A06A022103689B6C9847A06A44F21B116B
:10BBF000029403689E6A074B039304AB13E90C009D
:10BC0000B0475CF0CFFF2064284604B0BDE8F08167
:10BC1000ACE10B0885BD0208B425003070B5858FF6
:10BC2000DB0090F93B60AD03B5FBF2F2A2F5804476
:10BC300004FB04F2D51190F83A200498D201A03008
:10BC4000624306FB0522521202F580124243121390
:10BC50004A4303EB623000B270BD000010B55300E0
:10BC6000448E5C43B0F93830C91A838F04F5004420
:10BC7000D31AB0F93620B0F9340053434FF40042E0
:10BC800000EB24409B10C3EBC133034993FBF0F05E
:10BC90000FF020F900B210BD0080FFFF10B52DEDB0
:10BCA000028B8AB004460823422105AA806A0AF062
:10BCB00043FF18B1BDF81A20D30719D4A06A0AF0BF
:10BCC0005FFF5CF06FFF236CC31AFA2B0CD90023C3
:10BCD00082224B212064A06A0AF00AFF01234B2133
:10BCE000A06A1A460AF004FF0AB0BDEC028B10BD30
:10BCF00094F930309208BDF9141020460093C91011
:10BD000094F92E300392FFF789FF94F9313008EE51
:10BD1000900ABDF916102046039A0093C91094F9B1
:10BD20002F30FFF77BFFBDF91810039A08EE100AB9
:10BD300049102046FFF792FF07EE900AF8EEE88AD6
:10BD400007A8F8EEE77AB8EEC88AB3EE000ACDEDA0
:10BD5000078ACDED097A8DED088A11F0A1FEB2EEC9
:10BD6000040A07A811F088FE5CF01CFF0A23206477
:10BD700007A9204694F82C2000F044FEA06A0AF09F
:10BD8000FFFEB1E7FFF78ABFF7B503680D46164619
:10BD90001BB90024204603B0F0BD002707604820EF
:10BDA000CDE90073FDF750FB044650B100F03EFCB6
:10BDB0000E4B84F844602360019B84F84550019742
:10BDC000A36201A8FCF78AF86846FCF787F8002C04
:10BDD000DFD02046FFF762FE05460028DAD123684F
:10BDE00020462C465B689847D4E700BFE4E10B0887
:10BDF000044B10B5044640F8283BFCF76FF820468A
:10BE000010BD00BFE4E10B0810B50446FFF7F0FFDA
:10BE10002046FDF721FB204610BD0000002290F8CF
:10BE20002C1000F003BD0000F8B504460D4617467F
:10BE30001E4600F0FBFB094B0022204623602B68C6
:10BE400084F82D70A36200232A6084F82E60236595
:10BE50006365A365E36523666366F8BDFCE10B08D3
:10BE6000F8B51C46093316466A46DB0800AF806AFF
:10BE7000A2EBC3039D46A31C6A460AF05DFE05467D
:10BE800028B122460DF10201304688F05FFF2846B6
:10BE9000BD46F8BD2DE9F34106460F4614465CF059
:10BEA00081FE114B0546D3F80080D8F82800012107
:10BEB00003685B68984701230DF1070207213046AC
:10BEC000FFF7CEFF60B19DF80730DA0702D4B7EB79
:10BED000531F05D05CF066FE431BA342E5D3002050
:10BEE00002B0BDE8F08100BFB42500302DE9F0417B
:10BEF00092B004460026DFF85C8202AF46F02002D2
:10BF000000235021A06AD2B20AF0F2FD002800F00E
:10BF10000C810325013D6DB26A1C00F00681D8F842
:10BF200000304FF49671986A03689B689847012324
:10BF30000DF1060255212046FFF792FF002800F080
:10BF4000F4809DF8063013F0E00F40F0EE80DB0740
:10BF5000E0D502230DF1060252212046FFF780FFB3
:10BF6000002800F0E280BDF8063001365BBA202ED2
:10BF700027F8023BC2D1BDF824309DF8261043F3C8
:10BF80000B021B099FED6B7A03F4706307EE902A96
:10BF9000BDF826200B43F8EEE77ADFED676A43F33E
:10BFA0000B039FED666AC4ED0C7A07EE903A02F43B
:10BFB00070639DF82820F8EEE77A134343F30B03F0
:10BFC000C4ED0D7A07EE903A9DF92230F8EEE77A4B
:10BFD000C4ED0E7A07EE903A9DF92930F8EEE77A33
:10BFE00067EE877A07EE103A9DF92A30B8EEC77AE5
:10BFF000C4ED0F7ADFED527A27EE267A84ED107ABF
:10C0000007EE103A9DF92B30B8EEC77AE7EE267AA4
:10C01000C4ED117A07EE903A9DF92330F8EEE77AF5
:10C0200067EEA67ADFED476AC4ED127A07EE903A22
:10C030009DF92C30F8EEE77A07EE103A9DF92E3094
:10C04000B8EEC77A67EE867A27EE267AC4ED137AC1
:10C0500084ED147A07EE103A9DF93030B8EEC77AC5
:10C0600007EE903A9DF92D30F8EEE77A27EE267A22
:10C0700067EEA67A84ED157A9FED337AC4ED167AD1
:10C0800007EE903A9DF92F30F8EEE77A67EE877A5F
:10C09000C4ED177A07EE903A9DF93130F8EEE77A61
:10C0A00006EE903ABDF9383067EE877AF8EEE66A28
:10C0B000C4ED187ADFED257AE6EE877A07EE103ABE
:10C0C0009DF93230B8EEC77ADFED216AC4ED197AF6
:10C0D000F3EE077AE7EE067A07EE103AB8EEC77A83
:10C0E00027EE267AC4ED1A7A84ED1B7A9DF9333057
:10C0F00007EE103A9DF93430B8EEC77A27EE267A6B
:10C1000084ED1C7A07EE103A9DF93530B8EEC77A07
:10C1100007EE903AF8EEE77A27EE267A67EEA67AEF
:10C1200084ED1D7AC4ED1E7A00E0002012B0BDE857
:10C13000F08100BFCDCC4C3E0000803B0000003BB6
:10C140000AD7233C0000003D0000803817B7D1B863
:10C150000AD7A33AB425003073B501230E460DF17A
:10C16000070206210446FFF77BFE18B90025284682
:10C1700002B070BD9DF80730013B012B0CD80023A5
:10C180000621A06A1A460AF0B3FC0028EED0062267
:10C1900000212046FFF77EFE002332460621A06ADA
:10C1A0000AF0A6FC05460028E0D0262231462046AB
:10C1B000FFF770FEDBE7000013B501230DF1070266
:10C1C00007210446FFF74CFE10B9002002B010BD55
:10C1D0009DF807301B070CD500230621A06A1A46DC
:10C1E0000AF086FC0028F0D0062200212046FFF746
:10C1F00051FE002307220621A06A0AF079FC0028DC
:10C20000E3D0132207212046FFF744FE0028DCD0AC
:10C21000002305220621A06A0AF06AFC0028D4D077
:10C22000172205212046FFF735FE0028CDD0012139
:10C230002046FFF791FFC9E7F7B50446806A052558
:10C240005A4F03685B6A984703689B689847A06ADF
:10C250000A2103689B6C98470A220421A06A0AF00D
:10C26000F1FB013D6DB26B1C00F096800023B622FD
:10C270007E21A06A0AF03CFC0028F2D03B686E46A2
:10C280001821986A03685B689847012332460021A9
:10C290002046FFF7E5FD0028E3D09DF80030332B62
:10C2A000DFD12046FFF722FE002875D00023802230
:10C2B0005021A06A0AF01CFC00286DD02046FFF730
:10C2C0007BFF002868D0002386222E21A06A0AF076
:10C2D0000FFC002860D0002324220421A06A0AF069
:10C2E00007FC002858D0002302220621A06A0AF089
:10C2F000FFFB002850D0142202212046FFF7CAFD80
:10C30000002307220521A06A0AF0F2FB002843D08F
:10C3100001212046FFF720FF00283DD0A06A03211D
:10C3200003689B6C9847A06A03685B6A9847036838
:10C33000DB6898471721A06A0AF09CFBA36A04F106
:10C340002C022046996800F0BFFA054608B3A36A9C
:10C35000204694F82C109A6800F0BAFA94F82E202F
:10C3600094F82C10204600F0E9FA94F82D302BB107
:10C37000012294F82C10204600F0BEFAA06A42F286
:10C38000107103689F6A0A4B0094019396E80C00B1
:10C39000B847284603B0F0BDA06A002503685B6A71
:10C3A00098470368DB689847F3E700BFB42500307F
:10C3B000A9C5020810B586B00C23312104466A468F
:10C3C000FFF74EFD002800F0DF809DF801309DF85A
:10C3D00000201B04DFED707ADFED705A03EB0223BF
:10C3E0009DF8022003EB02639DF803201B1206EE6A
:10C3F000903A9DF804301B04F8EEE66A03EB022342
:10C400009DF8052066EEA76A03EB02639DF80620FF
:10C410001B1207EE103A9DF807301B04B8EEC77ADE
:10C4200003EB02239DF8082027EE277ADFED5C7AE4
:10C4300003EB02639DF809201B1206EE103A9DF8EB
:10C440000A301B04B8EEC66A03EB02239DF80B20EA
:10C4500026EE276A03EB02631B1207EE903AF8EE12
:10C46000E77A67EEA57AF5EEC07AF1EE10FA40F3BE
:10C470008D80DFED4C5A77EEE57AF7EE005AD4ED79
:10C48000134A94ED0F5A0A2394ED1C4A03A974EE43
:10C49000A54AD4ED1D3A94F82C202046F0EE632AEC
:10C4A000A4EEA75AD4ED107AD4ED0C4A77EEA57A13
:10C4B000E7EEA64AD4ED1A7A75EE677A94ED145A2F
:10C4C000F0EE646AD4ED174AE5EE276AB0EE655ADD
:10C4D000A7EEA45AC6EE854A94ED115AD4ED0D6A22
:10C4E00035EE255AE5EE076A94ED157AB0EE655AF9
:10C4F000E7EE876A94ED187AA7EE875A86EE857A7A
:10C5000094ED125AD4ED0E6A35EE255AE5EE066A20
:10C5100094ED166A94ED195AE7EE866AB0EE656AF4
:10C52000A7EE856AF0EE657A86EE863A94ED1B6A90
:10C53000F0EE646AE6EE447AE6EE476A86EEA75AC3
:10C54000F0EE476AE4EE646AC6EEA75AD4ED1E6ABE
:10C55000D4EE262AE6EE636AB2EE046A27EE667A25
:10C5600065EE066AA2EEA47ACDED036A65EE866AF0
:10C57000CDED046AC7EE276A76EE837A67EE867A97
:10C58000CDED057A00F03EFA06B010BD44BFDFEDF8
:10C59000055A77EEA57A70E747ABE73B5B9E803A9A
:10C5A000F61BEB3B85EBCB41FFF704BF30B51346E1
:10C5B000026885B00D461AB90024204605B030BD8A
:10C5C00000210193039201607C20FCF73DFF0446AB
:10C5D00020B1019B2A4603A9FFF726FC03A8FBF71D
:10C5E0007DFC002CE8D02046FFF726FE05460028FB
:10C5F000E3D1236820462C465B689847DDE70000BE
:10C60000044B10B5044640F8283BFBF767FC204676
:10C6100010BD00BFFCE10B0810B50446FFF7F0FFAA
:10C620002046FCF719FF204610BD0000064B10B550
:10C6300004460360FDF7AEFC606004F108005BF0A7
:10C640004FFA204610BD00BF14E20B0873B5064632
:10C6500014467C2308467568C4EB4414019003FB20
:10C66000025305EB840493F8A81011F09BFA94F997
:10C67000403001983BB9736893F8291002B0BDE8C7
:10C68000704011F08FBA94F84410F7E737B57C2565
:10C690004468019105FB024595F8433004EB83049F
:10C6A000D4F850325BB15CF07DFA0199C5F8A00076
:10C6B000D4F8500203B0BDE8304003F0A9BF03B086
:10C6C00030BD00002DE9F04FC2EB421447680E4622
:10C6D00081464FEA840807F1400B15468BB008F1FC
:10C6E000080130460BEB8404594411F091F92946B6
:10C6F000D9F80400FDF7F4FB38B17C23304603FB86
:10C70000057393ED1B0A11F0B7F97C23DFED3C7A3A
:10C7100003FB057393ED156AD3ED166AB0EEC67A86
:10C72000B4EEE77AF1EE10FA0FD5B0EEE67AB4EE99
:10C73000E77AF1EE10FA08D594ED077AB0EEC77AF1
:10C74000B4EEE77AF1EE10FA1BD47C2303FB0573F9
:10C75000186E596E9A6EDB6D02900391049001A8D9
:10C76000079131468DED016ACDED056A069208927A
:10C7700009930EF0ABFD86ED000AC6ED010A86EDC9
:10C78000021A7C2308F13C0A08F1480803FB0577EC
:10C790000023DA44D844C7F89030C7F88C30C7F883
:10C7A0008830D9F8040090F9603263B15DB9414630
:10C7B00000F5177004F0CEFB414630460BB0BDE8E3
:10C7C000F04F11F025B990F93830012B0BD190EDD5
:10C7D0000F0A504611F0FCF884ED120AC4ED130A5A
:10C7E00084ED141AE8E7022BE6D1FCF701FA0022E7
:10C7F00001A9FBF7D5FE0028DED09DED010AE8E790
:10C800000000003410B57C24436804FB023407C9DF
:10C8100004F1940383E807005CF0C4F9C4F8A000B5
:10C820005CF0B8F9C4F8A40010BD0000F0B585B004
:10C8300007460D46164600F10801A92203A80AF092
:10C84000D5FB7C687C2303FB0543D3F8B82022B9D1
:10C8500003A80AF0EDFB05B0F0BDBEB196ED007A7D
:10C86000D3ED2B7A67EE877AC3ED2B7AD3ED2C7A52
:10C8700096ED017A67EE877AC3ED2C7AD3ED2D7AA7
:10C8800096ED027A67EE877AC3ED2D7A7C2607EE65
:10C89000902A06FB0541B8EE670AAC3108460191C3
:10C8A00011F0FEF801992A463846FFF7ABFF06FB68
:10C8B00005410023C1F8B430C1F8B030C1F8AC3044
:10C8C0000023C1F8B830C3E74068FCF7E9BE0000B8
:10C8D000F7B506467C2740680D461446019207FBD3
:10C8E000010001A9703035F09BF9716807FB05154F
:10C8F0006C6703B0F0BD000007B57C23406803FB04
:10C90000010393F94030022B0BD000F14003C1EB3F
:10C9100041100DF107018DF8072003EB800035F081
:10C92000D9F803B05DF804FB43687C2202FB0131B7
:10C9300091F94000003818BF0120704743687C20FF
:10C9400000FB013181F8A82070470000F8B50546CA
:10C9500008460F4611F002F910B100242046F8BD38
:10C96000384611F0E1F804460028F6D16B6893F9D7
:10C9700038637EB1384611F027FC95ED087ADFED7B
:10C980001E7AF0EEC76AF4EEE76AF1EE10FA03D50C
:10C9900085ED080A0124E1E777EE407AF6B230EE41
:10C9A000076AF0EEE77AC7EE866A07EE906A9FEDB7
:10C9B000136AF8EE677A26EE866AF4EEC67ADFED41
:10C9C000107AF1EE10FA47BFB2EE046A6B6AB0EE6D
:10C9D000676A012441BF013366EE866A6B6287EEA7
:10C9E000A66AF7EE007A20EE060A77EEC67AA7EE80
:10C9F000270A85ED080AB1E700000034000048432B
:10CA0000CDCCCC3D2DE9F74304460E4615461F46D6
:10CA1000FFF71CFE31462A462046FFF737FE314617
:10CA200020462A46FFF74EFE31462046FFF78EFF8E
:10CA300028B39B2204F1080101A84FF07C090AF0F9
:10CA4000D5FA6468314609FB054808F1AC08404650
:10CA500010F0DEFF09FB0542D2F8B8100131C2F830
:10CA6000B8104FB1B94207D34908B0EE000A4046AA
:10CA7000C2F8B81011F014F801A80AF0D9FA03B0FE
:10CA8000BDE8F08310B50446FCF792FEC0B2403416
:10CA9000C0EB401004EB800010BD0000F8B5044668
:10CAA00000F51777084E04F5147555F8040B08B116
:10CAB00004F0CAF8BD42F8D133680121986A0368CE
:10CAC0005B689847EFE700BFB425003008B5FFF773
